:1000000000080020431D03004F1D03004F1D030087
:10001000EDC402004F1D03004F1D03004F1D0300E0
:100020004F1D03004F1D03004F1D03004F1D030014
:100030004F1D03004F1D03004F1D03004F1D030004
:100040004F1D03004F1D03004F1D03004F1D0300F4
:100050004F1D03004F1D03004F1D03004F1D0300E4
:100060004F1D03004F1D03007D3601008D68010008
:10007000816801004F1D03004F1D03004F1D030049
:100080004F1D03004F1D03004F1D03004F1D0300B4
:100090004F1D030095C702004F1D03004F1D0300B5
:1000A0004F1D0300AF330200953302004F1D0300C4
:1000B0004F1D0300075302004F1D0300C7590200E4
:1000C0008359020081590200B9530200C559020048
:1000D000855902008959020087590200591C030002
:1000E000055A02004F1D03004F1D03004F1D030062
:1000F0004F1D03009F5401004F1D03004F1D0300BF
:100100004F1D03004F1D03004F1D03004F1D030033
:100110004F1D03004F1D03004F1D03004F1D030023
:100120004F1D03004F1D03004F1D03004F1D030013
:100130004F1D030000000000000000000000000050
:10014000401E00D0FCE77047000000000000F03FB8
:1001500000000000000024400000000000005940A2
:100160000000000000408F40000000000088C340F5
:1001700000000000006AF8400000000080842E416A
:1001800000000000D01263410000000084D79741B6
:100190000000000065CDCD41666E692D00000000B5
:1001A000666E692B00000000207B696E7465726EBC
:1001B000616C5F6572726F723A25647D00000000A9
:1001C0007B282573297D00007B6572726F723A006F
:1001D0007B6572726F72436F64653A25647D0000BF
:1001E0000100000005000000020000030000000004
:1001F00000000000000000000B0000000B000000E9
:1002000002000000000020200000000003000000A9
:100210008C8C3C000000000000000000000000008A
:1002200001260000040000000000000000010000A2
:10023000000000004552524F523A204E6F206D6F21
:10024000726520737061636520746F2073746F72C0
:100250006520636C6920636F6D6D616E64732069E6
:100260006E2052414D2E0A005468652061726775F8
:100270006D656E74206973206E6F7420666F726D89
:10028000617474656420636F72726563746C790065
:100290004E6F20636F6D6D616E6420666F756E6466
:1002A000000000004D6178696D756D206E756D629E
:1002B0006572206F6620617267756D656E7473205C
:1002C000657863656564656400000000496E636F6E
:1002D000727265637420617267756D656E742074E7
:1002E00079706500496E636F7272656374206E7514
:1002F0006D626572206F6620617267756D656E74E0
:1003000073000000556E6B6E6F776E206572726FB2
:100310007200000075696E743800000075696E74B3
:100320003136000075696E7433320000696E7438BE
:1003300000000000696E743136000000696E74338D
:1003400032000000737472696E67000075696E7424
:10035000386F70740000000075696E7431366F700C
:100360007400000075696E7433326F7074000000A1
:10037000696E74386F707400696E7431366F7074A2
:1003800000000000696E7433326F7074000000006A
:10039000737472696E676F70740000006865786FBF
:1003A000707400006164646974696F6E616C000050
:1003B00077696C64636172640000000067726F7536
:1003C00070000000756E6B6E6F776E002E2E2E2003
:1003D0000000000068656C70000000000A25730AC8
:1003E000257325730000000025732008000000001D
:1003F000000000000000000002000000006A180079
:10040000000204000000000205000000640000007B
:10041000960000006400000096000000000000004C
:100420000000000000000000000000000100A00229
:100430000201020164000000B60000006400000038
:10044000C0000000000000000000000000000000EC
:100450000B010000C800FCFEB4008B087BC0FBFF52
:100460004D00E402E756FFFF2C00A20183EBFFFFE3
:100470001A000301B31A00001100A300552900005F
:100480000A005E005A28000006003A0021220000FF
:1004900004001800731600006400FCFEFFFF00005B
:1004A00000000000FFFF0000000000005A00F306FB
:1004B000A554FEFF2100A301A1FEFFFF1100A6002D
:1004C000832700000A006100DC26000006003B00D4
:1004D000F820000003001500AD1300000000FCFE32
:1004E000FFFF000000000000FFFF00000000000010
:1004F000FFFF000000000000FFFF00000000000000
:1005000040001806F4D200002C00B0023DBE0000EE
:100510001700F2000C7C00000C0041009E4200001D
:10052000000801B4540400000008015A98040000B7
:1005300000080040DC040000000000000000000093
:100540000080640001000080FF7F00000080FF7FCA
:10055000040200005258414354495645000000002F
:100560005458414354495645000000004C4E414503
:100570004E0000005041454E0000000052414341F2
:1005800043544956450000005054494441544100E9
:100590004652414D4544455445435400505245410F
:1005A0004D424C45444554454354000054494D493F
:1005B0004E47444554454354000000004652414DC7
:1005C0004553454E5400000053594E4353454E5435
:1005D00000000000454F46004343300043433100D4
:1005E00054050000010003316005000001000431E2
:1005F0006C050000010001317405000001000231AA
:100600007C05000001000031880500000100012E7A
:10061000900500000100072B9C0500000100072C3D
:10062000AC0500000100032DBC0500000100002CFA
:10063000C80500000100022DD40500000100052DB1
:10064000D80500000100012FDC0500000100022F89
:1006500069646C6500000000556E6B6E6F776E20EC
:100660006175746F2061636B2064656661756C747D
:100670002073746174652E00496E76616C69642024
:1006800069646C652074696D696E672E00000000F6
:10069000496E76616C6964207475726E61726F75F3
:1006A0006E642074696D696E6700000043616C6C54
:1006B00020746F205241494C5F49454545383032DE
:1006C0003135345F496E69742072657475726E6578
:1006D0006420616E206572726F7200003830322EB5
:1006E00031352E343A25732C727844656661756C09
:1006F0007453746174653A25732C7478446566612B
:10070000756C7453746174653A25732C69646C65F7
:1007100054696D696E673A25642C7475726E6172E6
:100720006F756E6454696D653A25642C61636B5412
:10073000696D656F75743A25642C64656661756CC6
:10074000744672616D6550656E64696E673A2573B3
:100750000000000044697361626C65640000000081
:10076000456E61626C65640054727565000000003E
:1007700046616C73650000003830322E31352E34FE
:100780003A2573004661696C656420746F20736557
:1007900074207768696368206672616D6573207480
:1007A0006F206163636570742E000000436F6D6D90
:1007B000616E644672616D653A25732C41636B46C8
:1007C00072616D653A25732C446174614672616D86
:1007D000653A25732C426561636F6E4672616D6583
:1007E0003A25732C4D756C7469507572706F736512
:1007F0004672616D653A2573000000004661696CC0
:10080000656420746F2028756E297365742070727A
:100810006F6D697363756F7573206D6F64652E00FE
:1008200050726F6D697363756F75734D6F64653A60
:10083000257300004661696C656420746F2028751B
:100840006E297365742050414E20436F6F72646946
:100850006E61746F722E000050616E436F6F726430
:10086000696E61746F723A25730000003830322E61
:1008700031352E3450616E49643A25730000000012
:100880003830322E31352E3453686F7274416464BF
:10089000726573733A2573003830322E31352E3439
:1008A0004C6F6E67416464726573733A2573000020
:1008B000FFFFFFFFFFFFFFFFFFFFFFFF0000000044
:1008C0000000000000000000000000000000000028
:1008D000000000003830322E31352E34416464720D
:1008E00065737365733A2573000000004461746199
:1008F0005265714C6174656E63793A25750000002C
:100900003830322E31352E34453A4661696C656493
:100910000000000031352E34455F47423836383A02
:1009200025732C31352E34455F456E6841636B3A33
:1009300025732C31352E34455F496D706C696369C0
:100940007442726F6164636173743A2573000000CE
:100950003830322E31352E34473A4661696C656441
:100960000000000031352E34475F47423836383AB0
:1009700025732C31352E34475F44796E616D696380
:100980004645433A25732C57692D53554E5F4D6F9D
:1009900064655377697463683A257300556E73759F
:1009A00070706F72746564004561726C7946703A5C
:1009B00025732C4461746146703A25730000000071
:1009C000696E76616C696420504852207479706554
:1009D0003A20256400000000696E76616C6964202D
:1009E0006E756D626572206F6620617267756D65E8
:1009F0006E74730050687253697A653A25642C509E
:100A000048523A30782578005048522077726974FD
:100A100065206661696C6564000000004D6F646567
:100A200020737769746368696E67206E6F742073D2
:100A30007570706F72746564206F6E20746869736E
:100A40002063686970206F72206D697373696E67C7
:100A50002050485220617272617900006363614DD9
:100A60006F64653A25750000434341206D6F6465EE
:100A700020756E737570706F72746564000000008D
:100A80005369676E616C206964656E746966696537
:100A90007220756E737570706F72746564000000FB
:100AA00064000000B600000064000000C000000008
:100AB0000000000000000000000000000000000036
:100AC0000100A0020202020200000000000000007B
:100AD0000000000000000000000000000000000016
:100AE000000000000B00000000000000FFFFFFFFFF
:100AF000220022008200820000000200FFFFFFFFB0
:100B00002200200082008000FFFFFFFFFFFFFFFFA9
:100B1000FFFFFFFFFFFFFFFFFFFFFFFFFFFFFFFFE5
:100B2000FFFFFFFFFFFFFFFF00220022FFFFFFFF8D
:100B3000222222208222822000220020FFFFFFFFAB
:100B4000222222208222822000820082FFFFFFFFD9
:100B5000228222808282828000820080FFFFFFFF4B
:100B60002282228082808080496E76616C69642056
:100B7000616464726573732066696C746572696E12
:100B80006720636F6E66696775726174696F6E2E38
:100B9000000000004164647265737346696C74659B
:100BA00072696E673A257300456E61626C65640018
:100BB00044697361626C6564000000003078252E22
:100BC000327820004669656C643A25752C496E645C
:100BD00065783A25752C4F66667365743A25752CD1
:100BE00053697A653A25752C416464726573733A6A
:100BF00025732C5374617475733A257300000000DB
:100C00004D61736B65642061646472657373206603
:100C1000696C746572696E67206E6F74207375708D
:100C2000706F72746564210041646472657373202F
:100C30006669656C64206F7220696E646578206FE8
:100C40007574206F662072616E6765210000000078
:100C5000546F6F206D616E79206164647265737387
:100C600020627974657320676976656E21000000E3
:100C7000436F756C64206E6F7420636F6E66696776
:100C800075726520616464726573732100000000F1
:100C9000436F756C64206E6F7420656E61626C6565
:100CA0002F64697361626C6520616464726573733B
:100CB0002100000069646C6500000000556E6B6ED9
:100CC0006F776E206175746F2061636B2064656659
:100CD00061756C742073746174652E00496E766161
:100CE0006C69642069646C652074696D696E672E37
:100CF00000000000496E76616C6964207475726E44
:100D000061726F756E642074696D696E67000000B2
:100D100043616C6C20746F205241494C5F436F6E8D
:100D20006669674175746F41636B20726574757293
:100D30006E656420616E206572726F720000000043
:100D4000727844656661756C7453746174653A2594
:100D5000732C747844656661756C74537461746542
:100D60003A25732C69646C6554696D696E673A2520
:100D7000752C7475726E61726F756E6454696D65F1
:100D80003A25752C61636B54696D656F75743A25EE
:100D9000750000004175746F41636B3A25732C52E6
:100DA000784175746F41636B5374617475733A2540
:100DB000732C54784175746F41636B53746174750F
:100DC000733A257300000000456E61626C65640033
:100DD00044697361626C6564000000005061757362
:100DE00065640000556E70617573656400000000F5
:100DF0004572726F722064697361626C696E6720FC
:100E00004175746F41636B0043616E63656C416350
:100E10006B3A25732C557365547842756666657216
:100E20003A257300547275650000000046616C73CA
:100E3000650000000000000000000000424C453A40
:100E400025730000456E61626C65640044697361DE
:100E5000626C6564000000005374617475733A2518
:100E600073000000424C45206D6F6465206E6F7406
:100E700020656E61626C6564000000004C6F6769FC
:100E800063616C4368616E6E656C3A25642C4163E6
:100E900063657373416464726573733A30782530A7
:100EA0002E38582C437263496E69743A3078253075
:100EB0002E38582C57686974656E696E673A2573C9
:100EC0000000000053657474696E67206368616E8A
:100ED0006E656C20706172616D65746572732066F9
:100EE00061696C6564000000496E76616C6964201C
:100EF0006164766572746973696E67206368616E98
:100F00006E656C004164766572746973696E6743DF
:100F100068616E6E656C3A25640000005068795314
:100F20007769746368546F52783A25730000000043
:100F30005369676E616C206964656E746966696582
:100F40007220756E737570706F7274656400000046
:100F5000021AFFEEDDCCBBAA020106100853696C31
:100F6000616273205241494C54455354496E737524
:100F70006666696369656E7420617267756D656E1A
:100F800074732E204D7573742070726F766964656A
:100F9000206368616E6E656C20686F7070696E6743
:100FA0002073657175656E63652E00004368616E20
:100FB0006E656C206D75737420626520612031361A
:100FC000206269742076616C75652E006E756D62A5
:100FD00065724F664368616E6E656C733A25642C6A
:100FE0006275666665723A307825782C537563634E
:100FF0006573733A25730000547275650000000034
:1010000046616C7365000000496E646578206D75FB
:101010007374206265203C2025750000696E64654C
:10102000783A25752C6F7074696F6E733A25752C3C
:10103000727373695468726573686F6C643A25647F
:1010400000000000696E6465783A25752C73796E2E
:10105000634465746563743A25752C707265616DBF
:10106000626C6553656E73653A25752C74696D699C
:101070006E6753656E73653A25752C74696D696E7C
:1010800067526553656E73653A25750053756363E2
:101090006573733A25730000436F756C64206E6F3F
:1010A00074207265616420525353492E20456E733B
:1010B000757265206368616E6E656C20686F707014
:1010C000696E672077617320636F6E6669677572FA
:1010D000656420616E6420656E61626C65642E00DB
:1010E000727373693A257300496E73756666696336
:1010F00069656E7420617267756D656E74732066C4
:101100006F7220737065636966696564206D6F64D2
:10111000650000004D697373696E672072737369AF
:101120005468726573686F6C6420617267756D6571
:101130006E7420666F72207370656369666965649A
:10114000206F7074696F6E00556E6578706563749A
:10115000656420657874726120617267756D656E73
:10116000747320666F722073706563696669656465
:10117000206D6F64652F6F7074696F6E730000006F
:10118000537563636573733A25732C4D6F64653AC9
:10119000307825782C506172616D657465723A25DE
:1011A000752C44656C61793A25642C4F7074696FB5
:1011B0006E733A25752C727373695468726573681F
:1011C0006F6C643A256400004E6F206368616E6E38
:1011D000656C7320696E2072616E676520666F753D
:1011E0006E6400004572726F7220696E2052414930
:1011F0004C5F4765744368616E6E656C4D657461E4
:10120000646174612C206368616E6E656C20636F2D
:101210006E66696720696E76616C69642E000000F5
:101220006368616E6E656C496E6465783A25752CED
:101230006368616E6E656C3A25752C6672657175B2
:10124000656E63793A25752C727373693A2573005C
:101250002B2D2D2D2D2D2D2D2D2D2D2D2D2D2D2DC0
:101260002D2D2D2D2D2D2D2D2D2D2D2D2D2B0A0000
:101270007C20525353492064426D20627920436898
:10128000616E6E656C204E756D626572207C0A0021
:10129000252D3464000000002025732064426D0A6F
:1012A000000000004368616E6E656C204E756D62D3
:1012B00065720A0052657065617465645478436FA5
:1012C000756E743A257500004E6565642061742062
:1012D0006C65617374203620706172616D65746530
:1012E000727320666F7220424C4520686F702063D5
:1012F0006F6E6669672E00005241494C2063686139
:101300006E6E656C206D7573742062652061207649
:10131000616C696420424C45206368616E6E656C47
:101320002E0000004C6F676963616C206368616E1A
:101330006E656C206D757374206265206120766126
:101340006C696420424C45206368616E6E656C2E4A
:101350000000000000000000FFFFFFFF0000000091
:101360000000000000000000FFFFFFFF0000000081
:10137000000000004E65774672657175656E637991
:101380003A257500257520487A206973206F757499
:10139000206F662072616E676520616E64206361F4
:1013A0006E6E6F74206265207365742061732074A3
:1013B0006865206672657175656E6379000000006E
:1013C0004E6F742063757272656E746C7920696EED
:1013D000206672657175656E6379206F76657272CD
:1013E000696465206465627567206D6F64652E00B1
:1013F00044697361626C6564000000004672657147
:1014000075656E6379204F76657272696465000058
:101410004E554C4C0000000044656275674D6F648A
:10142000653A257300000000256420697320616E11
:1014300020696E76616C6964206465627567206DF1
:101440006F6465210000000041646472657373205D
:101450003078252E3858206973206E6F742033320F
:1014600062697420616C69676E65640061646472AE
:101470006573733A3078252E38782C76616C7565F3
:101480003A3078252E38780043616C696272617455
:10149000696F6E733A257300456E61626C65640016
:1014A00046656174757265206E6F74207375707017
:1014B0006F7274656420696E20746869732074614A
:1014C000726765742E0000005065726970686572FD
:1014D000616C733A25732C4E6F746966696361742D
:1014E000696F6E733A25730053796D626F6C726128
:1014F00074653A25642C426974726174653A256496
:101500000000000043616E6E6F7420636F6C6C6549
:101510006374206D6F7265207468616E202564208D
:1015200072616E646F6D2062797465732E000000C5
:101530004572726F7220636F6C6C656374696E675D
:101540002072616E646F6D20646174612E00000012
:10155000252E3278000000004572726F7220707282
:10156000696E74696E672072616E646F6D2064616C
:1015700074612E004C656E6774683A25752C446161
:1015800074613A25730000004C656E6774683A25F3
:10159000752C446174615074723A3078252E387815
:1015A000000000002573205B70696E5D205B73692D
:1015B000676E616C5D205B6F7074696F6E735D0A3E
:1015C000000000000A50696E733A20416E79207065
:1015D000696E2066726F6D2050412C2050422C2085
:1015E00050432C20616E6420504420617661696C08
:1015F00061626C6520666F722064656275672C207D
:10160000627574206F6E6C7920313020746F746154
:101610006C2066726F6D20504120616E64205042D4
:101620002C20616E64203620746F74616C206672A9
:101630006F6D20504320616E642050440A0000000A
:101640000A50696E7320696E205573653A200A004E
:101650000A0A5369676E616C733A200A0000000041
:1016600020204F46460A2020435553544F4D5F508B
:101670005253203C736F757263653E203C736967FB
:101680006E616C3E0A2020435553544F4D5F4C49C8
:1016900042203C6576656E743E0A0000202025736A
:1016A0000A0000004E6F7420612076616C6964202E
:1016B00070696E206E616D65000000000A50696EF1
:1016C000206E6F7420696E20757365004E6F206DFB
:1016D0006F726520505253206368616E6E656C7343
:1016E00020617661696C61626C6520666F72205062
:1016F000412F5042000000004E6F206D6F72652038
:10170000505253206368616E6E656C732061766120
:10171000696C61626C6520666F722050432F504483
:10172000000000006E616D650000000068656C706F
:1017300000000000435553544F4D5F4C4942000098
:10174000496E76616C696420706172616D65746563
:1017500072732070617373656420746F20435553F6
:10176000544F4D5F4C494200435553544F4D5F50C9
:1017700052530000496E76616C6964207061726139
:101780006D65746572732070617373656420746F26
:1017900020435553544F4D5F5052530025732069D9
:1017A00073206E6F7420612076616C6964207369A8
:1017B000676E616C206E616D6500000050696E3A65
:1017C00025732C5369676E616C3A4F4646000000E2
:1017D00050696E3A25732C5369676E616C3A2573B4
:1017E0002C4368616E6E656C3A256400636F6465B6
:1017F0003A2564006E616D653A25732C73686966DD
:10180000743A25752C6D61736B3A257825303878DC
:101810002C7072696E74456E61626C65643A2573F2
:10182000000000006E616D653A5241494C5F4556BB
:10183000454E545F25732C73686966743A25752C80
:101840006D61736B3A30782578253038782C70725A
:10185000696E74456E61626C65643A2573000000C0
:10186000547275650000000046616C7365000000ED
:10187000656E61626C655072696E744576656E74F2
:10188000733A307825782530387800007072696EA8
:1018900074547841636B733A257300007072696EFB
:1018A0007452784572726F72733A257300000000AB
:1018B0007072696E745278467265714F66667365B0
:1018C00074733A25730000007072696E74696E67F4
:1018D000456E61626C65643A257300006170704DFD
:1018E0006F64653A25730000726164696F537461B7
:1018F00074653A25732C726164696F537461746501
:1019000044657461696C3A257300000076657269FC
:101910006679526164696F4362000000656E636FAF
:10192000646564416464726573733A307825303855
:10193000782C657870656374656456616C75653A7A
:101940003078253038782C61637475616C56616C21
:1019500075653A3078253038782C6469666665722A
:10196000656E6365417070726F7665643A257300C9
:10197000747275650000000066616C73650000009C
:1019800045787465726E616C20726164696F206362
:101990006F6E66696720737570706F7274206E6FFA
:1019A0007420656E61626C6564000000737563632A
:1019B0006573732C20646F6E65000000737563633C
:1019C0006573732C206F7065726174696F6E20731C
:1019D000757370656E64656400000000696E766101
:1019E0006C696420696E70757420706172616D65D8
:1019F000746572006461746120636F7272757074D3
:101A0000696F6E00766572696669636174696F6E8D
:101A10003A25732C746573744475726174696F6EC2
:101A200055733A25642C63616C6C6261636B436F20
:101A3000756E7465723A25640000000076657269FF
:101A40006669636174696F6E3A25732C746573748B
:101A50004475726174696F6E55733A2564000000B5
:101A60002417000000000000546F2072756E205093
:101A7000455220636F6D6D616E64732C20534C5F13
:101A80005241494C5F544553545F5045525F504F4B
:101A9000525420616E6420534C5F5241494C5F5454
:101AA0004553545F5045525F50494E206D757374D5
:101AB00020626520636F6E66696775726564206673
:101AC0006F72207573652E004572726F72206361AC
:101AD0006C6C696E67205241494C5F436F6E66695A
:101AE000674461746128292E000000004E756D4224
:101AF000797465733A25640042697473546F546550
:101B000073743A25752C42697473546573746564F3
:101B10003A302C50657263656E74446F6E653A306E
:101B20002E30302C525353493A25642C4269744567
:101B300072726F72733A302C50657263656E7442C4
:101B400069744572726F723A302E30302C53746162
:101B50007475733A5465737441626F72746564523C
:101B6000784F766572666C6F770000004269747317
:101B7000546F546573743A25752C426974735465B7
:101B8000737465643A25752C50657263656E744490
:101B90006F6E653A25732C525353493A25642C4293
:101BA00069744572726F72733A25752C5065726351
:101BB000656E744269744572726F723A25730000E3
:101BC000577269746554784669666F204572726F02
:101BD00072000000656C617073656454696D653AEC
:101BE000257500004572726F723A4E6F7420656EF3
:101BF0006F75676820696E707574732E0000000041
:101C00004572726F723A2573206973206E6F74206B
:101C1000612076616C696420706F72742E00000020
:101C20004572726F723A5468652070696E20796FE0
:101C3000752061726520636F6E6669677572696E83
:101C40006720697320756E617661696C61626C658D
:101C50002E20202020202020202020202020202076
:101C60002020202020202020202020202020506FF5
:101C70007274202573206861732074686520666F14
:101C80006C6C6F77696E6720706F7274206D617312
:101C90006B3A2025780000005374617475733A53D1
:101CA0007563636573732E0044697361626C656468
:101CB00000000000332D776972652D5350490000F4
:101CC000322D776972652D5541525400312D776957
:101CD00072652D55415254003F3F000025733A254F
:101CE00075000000526653746174653A25730000F4
:101CF0005241494C5F73746174655F6163746976C6
:101D0000650000005241494C5F73746174655F72F5
:101D1000780000005241494C5F73746174655F74D0
:101D2000780000005375636365737300496E7661D4
:101D30006C6964506172616D6574657200000000C9
:101D4000496E76616C6964537461746500000000CB
:101D5000496E76616C696443616C6C00556E6B6EA4
:101D60006F776E00557365725478436F756E743A71
:101D700025752C41636B5478436F756E743A2575E5
:101D80002C55736572547841626F727465643A259C
:101D9000752C41636B547841626F727465643A25A7
:101DA000752C557365725478426C6F636B65643A39
:101DB00025752C41636B5478426C6F636B65643A94
:101DC00025752C557365725478556E646572666C12
:101DD0006F773A25752C41636B5478556E64657244
:101DE000666C6F773A25752C5278436F756E743A2E
:101DF00025752C527843726345727244726F703A43
:101E000025752C53796E634465746563743A257542
:101E10002C4E6F52784275666665723A25750000E1
:101E2000547852656D61696E457272733A25752CEE
:101E3000526653656E7365643A25752C61636B5405
:101E4000696D656F75743A25752C61636B547846BE
:101E5000705365743A25752C61636B5478467046EF
:101E600061696C3A25752C61636B547846704164E6
:101E700064724661696C3A25750000004368616EC2
:101E80006E656C3A25752C4170704D6F64653A250E
:101E9000732C54696D696E674C6F73743A25752C99
:101EA00054696D696E674465746563743A25752C71
:101EB0004672616D654572726F72733A25752C5268
:101EC000784669666F46756C6C3A25752C52784F6A
:101ED000766572666C6F773A25752C41646472463C
:101EE000696C743A25752C41626F727465643A2589
:101EF000752C52784265616D733A25752C44617476
:101F00006152657175657374733A25750000000040
:101F100043616C6962726174696F6E733A25752CE6
:101F200054784368616E6E656C427573793A2575B5
:101F30002C5478436C6561723A25752C5478436350
:101F4000613A25752C547852657472793A25752C4E
:101F5000557365725478537461727465643A25756B
:101F60002C506150726F746563743A25752C5375EB
:101F700062506879303A25752C5375625068793112
:101F80003A25752C537562506879323A25752C5371
:101F90007562506879333A25752C7278526177539F
:101FA0006F7572636542797465733A307825782568
:101FB0003038780054785370616365436F756E7480
:101FC0003A25752C527842797465436F756E743A70
:101FD00025752C54784669666F5468726573686F0E
:101FE0006C643A25642C52784669666F5468726551
:101FF00073686F6C643A25642C54784669666F4147
:102000006C6D6F7374456D7074793A25752C5278C8
:102010004669666F416C6D6F737446756C6C3A25DA
:10202000752C52784669666F46756C6C3A25752C2E
:1020300052784F766572666C6F773A25752C5573BA
:1020400065725478556E646572666C6F773A257563
:102050002C41636B5478556E646572666C6F773A89
:10206000257500004170703A25642E25642E256484
:10207000000000005241494C3A25642E25642E256B
:10208000642E25642C686173683A3078252E3858A0
:102090002C666C6167733A3078252E325800000048
:1020A0005241494C3A25642E25642E2564000000D7
:1020B0004D756C746970726F746F636F6C3A2573D1
:1020C0002C4275696C743A25730000005472756572
:1020D0000000000046616C73650000006D6F646570
:1020E0003A25732C626175643A25752C70726F7491
:1020F0006F636F6C3A25752C726164696F436F6E04
:102100006669673A3078253032780000496E76612A
:102110006C69642076616C75652E204D7573742032
:102120006265206265747765656E202D32353520D5
:10213000616E64203235352E000000006C71694FED
:1021400066667365743A256400000000436F756C21
:1021500064206E6F74207265616420525353492E5F
:1021600020456E7375726520527820697320656E04
:1021700061626C6564000000727373693A25732CA8
:1021800065643135343A2575000000007273736957
:102190003A257300436F756C64206E6F742072650E
:1021A000616420525353492E20456E737572652029
:1021B00052582069732064697361626C65642E00F3
:1021C000436F756C64206E6F742072656164205279
:1021D0005353492E0000000054696D653A25640090
:1021E000496E76616C696420525353492E204D61CB
:1021F0006B652073757265207374617274417667C4
:10220000527373692072616E2073756363657373B3
:1022100066756C6C792E00004572726F7220736562
:102220007474696E672074686520727373694F6691
:102230006673657400000000727373694F6666739D
:1022400065743A2564000000726164696F527373AB
:10225000694F66667365743A25640000727373692A
:102260004F66667365743A25642C726164696F52B7
:102270007373694F66667365743A25642C746F7462
:10228000616C527373694F66667365743A256400B6
:1022900072737369446574656374546872657368B6
:1022A0006F6C6444626D3A25642C73746174757349
:1022B0003A257300456E61626C6564005253534960
:1022C000207468726573686F6C64206465746563FC
:1022D00074696F6E206973206E6F742073757070EF
:1022E0006F72746564206F6E207468697320636810
:1022F00069702E004572726F722073657474696E16
:1023000067207468652072737369446574656374CB
:102310005468726573686F6C642E000054696D6553
:102320003A2575005374617475733A537563636528
:1023300073732C43757272656E7454696D653A25BA
:10234000750000005374617475733A4572726F7250
:102350002C43757272656E7454696D653A2575000B
:10236000466561747572653A25732C436F6D7069AB
:102370006C6554696D653A25732C52756E54696DA0
:10238000653A2573000000005241494C5F53555097
:10239000504F5254535F4455414C5F42414E4400AC
:1023A0005241494C5F535550504F5254535F325035
:1023B0003447485A5F42414E440000005241494C64
:1023C0005F535550504F5254535F53554247485AEC
:1023D0005F42414E440000005241494C5F5355500A
:1023E000504F5254535F4F46444D5F5041000000E0
:1023F0005241494C5F535550504F5254535F414CDA
:102400005445524E4154455F54585F504F574552C2
:10241000000000005241494C5F535550504F5254F8
:10242000535F414E54454E4E415F444956455253C9
:10243000495459005241494C5F535550504F5254E2
:10244000535F4348414E4E454C5F484F5050494EB4
:10245000470000005241494C5F535550504F525471
:10246000535F4455414C5F53594E435F574F52445D
:10247000530000005241494C5F535550504F525445
:10248000535F45585445524E414C5F544845524D58
:102490004953544F520000005241494C5F5355502C
:1024A000504F5254535F415558414443000000007F
:1024B0005241494C5F535550504F5254535F505204
:1024C00045434953494F4E5F4C4652434F0000002D
:1024D0005241494C5F535550504F5254535F5241F3
:1024E00044494F5F454E54524F5059005241494C58
:1024F0005F535550504F5254535F524653454E53BD
:10250000455F454E455247595F44455445435449FC
:102510004F4E00005241494C5F535550504F52545A
:10252000535F524653454E53455F53454C454354C4
:102530004956455F4F4F4B00466561747572653A69
:1025400025732C436F6D70696C6554696D653A2510
:10255000732C52756E54696D653A25750000000044
:102560005241494C5F54585F504F5745525F4D4F51
:1025700044455F3250344749475F484947484553CF
:10258000540000005241494C5F54585F504F57452A
:10259000525F4D4F44455F5355424749475F484955
:1025A00047484553540000005241494C5F54585F1E
:1025B000504F5745525F4D4F44455F325034474965
:1025C000475F4850000000005241494C5F54585F3B
:1025D000504F5745525F4D4F44455F325034474945
:1025E000475F4D50000000005241494C5F54585F16
:1025F000504F5745525F4D4F44455F325034474925
:10260000475F4C50000000005241494C5F54585FF6
:10261000504F5745525F4D4F44455F5355424749D0
:10262000475F4850000000005241494C5F54585FDA
:10263000504F5745525F4D4F44455F5355424749B0
:10264000475F4D50000000005241494C5F54585FB5
:10265000504F5745525F4D4F44455F535542474990
:10266000475F4C50000000005241494C5F54585F96
:10267000504F5745525F4D4F44455F535542474970
:10268000475F4C4C500000005241494C5F54585F2A
:10269000504F5745525F4D4F44455F535542474950
:1026A000470000005241494C5F54585F504F574516
:1026B000525F4D4F44455F5355424749475F45463A
:1026C000465F333044424D005241494C5F54585F9D
:1026D000504F5745525F4D4F44455F535542474910
:1026E000475F4546465F323544424D005241494CB2
:1026F0005F54585F504F5745525F4D4F44455F53AD
:1027000055424749475F4546465F323044424D0097
:102710005241494C5F54585F504F5745525F4D4F9F
:1027200044455F4F46444D5F504100005241494C83
:102730005F54585F504F5745525F4D4F44455F4F70
:1027400046444D5F50415F4546465F333044424DFD
:10275000000000005241494C5F54585F504F5745AC
:10276000525F4D4F44455F4F46444D5F50415F457A
:1027700046465F323544424D000000005241494C0C
:102780005F54585F504F5745525F4D4F44455F4F20
:1027900046444D5F50415F4546465F323044424DAE
:1027A000000000005241494C5F54585F504F57455C
:1027B000525F4D4F44455F4F46444D5F50415F452A
:1027C00046465F4D415844424D0000005241494C3D
:1027D0005F535550504F5254535F50524F544F43D4
:1027E0004F4C5F424C4500005241494C5F424C45C2
:1027F0005F535550504F5254535F314D4250535FC9
:102800004E4F4E5F56495445524249005241494C41
:102810005F424C455F535550504F5254535F314DBA
:102820004250535F56495445524249005241494C27
:102830005F424C455F535550504F5254535F314D9A
:10284000425053005241494C5F424C455F535550F2
:10285000504F5254535F324D4250535F4E4F4E5F74
:1028600056495445524249005241494C5F424C45F9
:102870005F535550504F5254535F324D4250535F47
:1028800056495445524249005241494C5F424C45D9
:102890005F535550504F5254535F324D4250530086
:1028A0005241494C5F424C455F535550504F525432
:1028B000535F414E54454E4E415F53574954434830
:1028C000494E47005241494C5F424C455F53555079
:1028D000504F5254535F434F4445445F5048590052
:1028E0005241494C5F424C455F535550504F5254F2
:1028F000535F4354450000005241494C5F424C45F0
:102900005F535550504F5254535F5155555050419D
:10291000000000005241494C5F424C455F53555006
:10292000504F5254535F49515F53414D504C494EA3
:10293000470000005241494C5F424C455F5355509F
:10294000504F5254535F5048595F5357495443486E
:102950005F544F5F525800005241494C5F535550ED
:10296000504F5254535F50524F544F434F4C5F4956
:102970004545453830323135340000005241494C2C
:102980005F494545453830323135345F53555050F5
:102990004F5254535F434F45585F50485900000011
:1029A0005241494C5F494545453830323135345FF5
:1029B000535550504F5254535F455F535542534502
:1029C000545F4742383638005241494C5F494545CB
:1029D000453830323135345F535550504F5254538F
:1029E0005F455F454E48414E4345445F41434B0080
:1029F0005241494C5F494545453830323135345FA5
:102A0000535550504F5254535F475F5355425345AF
:102A1000545F4742383638005241494C5F4945457A
:102A2000453830323135345F535550504F5254533E
:102A30005F475F44594E4645430000005241494CB0
:102A40005F494545453830323135345F5355505034
:102A50004F5254535F475F4D4F444553574954437A
:102A6000480000005241494C5F49454545383032E5
:102A70003135345F535550504F5254535F475F5573
:102A80004E57484954454E45445F52580000000097
:102A90005241494C5F494545453830323135345F04
:102AA000535550504F5254535F475F554E57484906
:102AB00054454E45445F5458000000005241494C73
:102AC0005F494545453830323135345F53555050B4
:102AD0004F5254535F475F34425954455F4352430A
:102AE000000000005241494C5F49454545383032AD
:102AF0003135345F535550504F5254535F43414E1C
:102B000043454C5F4652414D455F50454E44494E0A
:102B1000475F4C4F4F4B5550000000005241494C0D
:102B20005F494545453830323135345F5355505053
:102B30004F5254535F4541524C595F4652414D45A7
:102B40005F50454E44494E475F4C4F4F4B555000E8
:102B50005241494C5F494545453830323135345F43
:102B6000535550504F5254535F455F4D554C544947
:102B7000505552504F53455F4652414D455300000A
:102B80005241494C5F494545453830323135345F13
:102B9000535550504F5254535F4455414C5F504130
:102BA0005F434F4E464947005241494C5F494545B6
:102BB000453830323135345F535550504F525453AD
:102BC0005F435553544F4D315F504859000000004A
:102BD0005241494C5F535550504F5254535F5052DD
:102BE0004F544F434F4C5F5A574156450000000029
:102BF0005241494C5F5A574156455F535550504FCB
:102C00005254535F524547494F4E5F50544900005C
:102C10005241494C5F5A574156455F535550504FAA
:102C20005254535F45445F50485900005241494C4B
:102C30005F5A574156455F535550504F5254535F5A
:102C4000434F4E435F504859000000005241494CE9
:102C50005F535550504F5254535F53515F50485932
:102C6000000000005241494C5F535550504F5254A0
:102C7000535F52585F5241575F4441544100000036
:102C80005241494C5F535550504F5254535F444941
:102C9000524543545F4D4F44450000005241494C5A
:102CA0005F535550504F5254535F414444525F4616
:102CB000494C5445525F414444524553535F424945
:102CC000545F4D41534B00005241494C5F535550A6
:102CD000504F5254535F4D464D0000005241494CF5
:102CE0005F535550504F5254535F454646000000C5
:102CF00063736D6100000000556E6B6E6F776E2020
:102D00004C4254206D6F6465207370656369666919
:102D100065642E004C62744D6F64653A6F666600A0
:102D20004C62744D6F64653A43534D41000000009E
:102D30004C62744D6F64653A4C4254004D696E426A
:102D40006F3A25752C4D6178426F3A25752C547277
:102D50006965733A25752C5468726573686F6C6485
:102D60003A25642C4261636B6F66663A25752C4484
:102D700075726174696F6E3A25752C54696D656F53
:102D800075743A25750000004D464D206973206E1C
:102D90006F742073757070706F72746564206F6EDD
:102DA000207468697320636869700000446174610D
:102DB000206F766572666C6F7773207478446174E7
:102DC000612062756666657200000000737461724E
:102DD000743A25752C656E643A2575005246536524
:102DE0006E7365205061796C6F61643A25730000E1
:102DF0004E6F742053657400496E76616C6964206F
:102E0000696E707574730000496E76616C69642038
:102E10006C656E67746820256400000054784C650A
:102E20006E6774683A25642C54784C656E677468D4
:102E3000205772697474656E3A2564004461746148
:102E4000206F766572666C6F77732061636B446187
:102E500074612062756666657200000054784C6586
:102E60006E6774683A25640046697865644C656EDF
:102E70006774683A256400006669666F00000000A8
:102E8000496E76616C69642044617461204D65749B
:102E9000686F642073656C656374696F6E2E0000E3
:102EA0004661696C656420746F2073756363657334
:102EB0007366756C6C792063616C6C205241494C6F
:102EC0005F44617461436F6E6669673A20256400F0
:102ED00054784D6574686F643A25732C52784D654B
:102EE00074686F643A25732C5278536F75726365FA
:102EF0003A2575004D6178205258204649464F20AA
:102F000073697A6520696E207468697320627569D7
:102F10006C642069732025752062797465730000E4
:102F200053657474696E67205258204649464F2095
:102F30006661696C65643B204D696E20525820467D
:102F400049464F2073697A652069732036342062C0
:102F5000797465730000000052784669666F5369A2
:102F60007A653A257500000044697361626C656496
:102F700000000000456E61626C656400547846692B
:102F8000666F4D616E75616C3A25732C5278466997
:102F9000666F4D616E75616C3A2573004D75737483
:102FA00020626520696E207278206669666F206DE8
:102FB000616E75616C206D6F646520286669666F4F
:102FC0004D6F6465546573744F7074696F6E7329C7
:102FD0002E000000020406005072653A25752C533D
:102FE000796E633A25752C456E643A25752C5072BE
:102FF00065416C743A25752C53796E63416C743A53
:1030000025752C456E64416C743A257500000000EE
:103010004E6F207061636B657420666F756E6420FF
:10302000696E207278206669666F2100446F4E6F6A
:103030007468696E67000000526573657400000073
:1030400054784669666F3A25732C52784669666FE4
:103050003A2573004D75737420626520696E207483
:1030600078206669666F206D616E75616C206D6F8A
:10307000646520286669666F4D6F64655465737476
:103080004F7074696F6E73292E0000005374617461
:1030900075733A4669666F205772697474656E007D
:1030A00054696D65416674657253796E63546F41FE
:1030B000626F72743A25640043616E2774207065F4
:1030C000656B206D6F7265207468616E20313020F1
:1030D000627974657300000052657175657374657B
:1030E00064206279746573206E6F7420696E20723B
:1030F00065636569766520627566666572000000C5
:10310000682F0000742F0000A5750100BB75010039
:10311000F37501002C300000383000005241494C5A
:103120005F54585F504F5745525F4D4F44455F3293
:1031300050344749475F4850000000005241494C15
:103140005F54585F504F5745525F4D4F44455F3273
:1031500050344749475F4D50000000005241494CF0
:103160005F54585F504F5745525F4D4F44455F3253
:1031700050344749475F4C50000000005241494CD1
:103180005F54585F504F5745525F4D4F44455F3233
:1031900050344749475F4849474845535400000069
:1031A0005241494C5F54585F504F5745525F4D4F05
:1031B00044455F4E4F4E45004368616E6E656C73CB
:1031C00020617265206E6F742076616C696420697D
:1031D0006E204465627567204D6F646500000000D5
:1031E0006368616E6E656C3A25640000496E7661B5
:1031F0006C6964206368616E6E656C2027256427A6
:10320000000000004F6666736574202564206F75AA
:1032100074736964652072616E6765206F66205BF8
:1032200025642C2025645D00436F756C64206E6FEF
:103230007420736574206672657175656E6379209C
:103240006F66667365740000667265714F666673BB
:1032500065743A2564000000737563636573733A9F
:1032600025732C6D6F64653A25732C766F6C7461D1
:1032700067653A25642C72616D7054696D653A25F5
:1032800064000000747275650000000066616C7374
:1032900065000000496E76616C69642050412065CC
:1032A0006E756D2076616C75652073656C656374F1
:1032B00065643A2025640000737563636573733A2F
:1032C00025732C706F7765724D6F64653A25732C8A
:1032D0006D696E506F7765724C6576656C3A2564E2
:1032E0002C6D6178506F7765724C6576656C3A2508
:1032F0006400000053756363657373004661696C15
:1033000075726500436F756C64206E6F7420736511
:103310007420706F77657220636F6E666967000056
:10332000706F7765724C6576656C3A25642C706FAA
:103330007765723A25640000436F756C64206E6F88
:10334000742073657420706F7765722E0000000022
:103350005377656570696E673A537461727465641A
:103360002C496E737472756374696F6E733A27714A
:103370002720746F2071756974206F722027656E25
:103380007465722720746F20636F6E74696E756543
:103390002E0000005041206E6F7420636F6E6669CE
:1033A00067757265642E0000506F7765724C6576A4
:1033B000656C3A25750000005377656570204162A1
:1033C0006F727465642E00005377656570696E676F
:1033D0003A436F6D706C6574650000004354554E40
:1033E000455849414E413A3078252E33782C435484
:1033F000554E45584F414E413A3078252E3378008E
:10340000496E76616C6964204354554E452076615F
:103410006C75652070726F766964656400000000E9
:103420004354756E6544656C74613A256400000010
:1034300050414354554E4554583A25642C5041430D
:1034400054554E4552583A25640000004572726F3B
:1034500072000000706143616C3A25730000000047
:10346000456E61626C65640044697361626C656499
:1034700000000000496E76616C69642073746174A9
:103480006573000054785472616E736974696F6E6D
:10349000733A25730000000052785472616E7369AC
:1034A00074696F6E733A257300000000537563638F
:1034B0006573733A25732C4572726F723A257300E7
:1034C000476574207278207472616E736974696FD5
:1034D0006E73206661696C65640000004765742046
:1034E0007478207472616E736974696F6E7320668C
:1034F00061696C656400000049646C65546F5278C2
:103500003A25752C5278546F54783A25752C4964B5
:103510006C65546F54783A25752C5478546F5278F2
:103520003A25752C52785365617263683A25752C7B
:1035300054783252785365617263683A25752C5419
:10354000783254783A25750053657474696E672033
:1035500074696D696E6773206661696C65640000EB
:103560005478206973206E6F7420696E2046494636
:103570004F206D6F6465000054784669666F54682B
:10358000726573686F6C643A25640000527846690E
:10359000666F5468726573686F6C643A25640000E6
:1035A0004D61736B3A30782578253038782C566128
:1035B0006C7565733A3078257825303878000000CE
:1035C0004D61736B3A307825782C56616C75657354
:1035D0003A30782578000000537563636573733A59
:1035E00025732C41637475616C44656C61793A256F
:1035F00064000000547275650000000046616C7341
:10360000650000005041206175746F206D6F646526
:103610002073686F756C6420626520656E61626CF2
:10362000656420746F2073657420636F6E666967CC
:10363000732E0000496E73756666696369656E7402
:1036400020617267756D656E74732E204D7573748D
:103650002070726F76696465206D696E2C206D61D3
:10366000782C206D6F646520616E642062616E64E9
:1036700020666F7220656163682050412061757417
:103680006F206D6F646520636F6E66696720656E7D
:103690007472792E000000005468657265206172B2
:1036A00065206E6F205041206175746F206D6F64CE
:1036B0006520636F6E666967732070726F766964E8
:1036C00065642E00546865205041206175746F2038
:1036D0006D6F646520636F6E6669677320617265E4
:1036E000206E6F7420636F6E666967757265642EF5
:1036F00000000000496E76616C6964206D6F64653E
:1037000020282564292073706563696669656400F3
:103710006E756D6265724F6650614175746F4D6F65
:103720006465456E74726965733A25642C537563DC
:10373000636573733A257300656E61626C653A2543
:10374000730000004C43443A2025732C204846580F
:103750004F3A2025732C20484652434F3A20257378
:103760002C20444344433A20257300005374617471
:1037700075733A256400000045787465726E616C5B
:1037800020726164696F20636F6E6669672073756C
:1037900070706F7274206E6F7420656E61626C65FC
:1037A00064000000766572696679526164696F0031
:1037B000526164696F206461746120636F72727515
:1037C0007074696F6E20646574656374656421004C
:1037D000524653656E73652057616B657570205056
:1037E00048593A257300000044697361626C65644E
:1037F00000000000456E61626C656400496E766190
:103800006C69642074696D65206D6F6465000000EB
:1038100063757272656E7454696D653A25752C64B2
:10382000656C61793A25752C726573756D6554699F
:103830006D653A2575000000466C617368207375EC
:1038400070706F7274206E6F7420656E61626C654B
:10385000640000006C6F636174696F6E3A25732CAD
:103860007374617475733A2573000000666C61733C
:103870006800000053756363657373004661696C8B
:10388000757265006C6F636174696F6E3A25732C95
:103890007374617475733A25732C736372697074F1
:1038A000436F756E743A25750000000074696D658C
:1038B00055733A25752C45787069726174696F6E1D
:1038C00054696D653A25752C497352756E6E696E33
:1038D000673A25732C4973457870697265643A2597
:1038E00073000000547275650000000046616C733F
:1038F0006500000053657454696D657220666169E6
:103900006C656400496E76616C6964206D756C74D9
:103910006954696D657220696E646578202D207325
:1039200074617274207769746820302E204E756D32
:10393000626572206F66206D756C746954696D657F
:1039400072732069732025640000000074696D653E
:1039500055733A25752C45787069726174696F6E7C
:1039600054696D653A25752C497352756E6E696E92
:10397000673A25732C4973457870697265643A25F6
:10398000732C4D756C746954696D6572496E64650C
:10399000783A2564000000007374617475733A25E9
:1039A000732C6E756D4D756C746954696D657273A9
:1039B0003A256400656E61626C65640064697361D8
:1039C000626C656400000000556E61626C65207475
:1039D0006F20636F6E666967757265207468652015
:1039E0006D756C746954696D65722E005365744D04
:1039F000756C746954696D6572206661696C656483
:103A0000000000004D756C746954696D6572207515
:103A10006E61626C6520746F2063616E63656C2EED
:103A2000000000004F66660047487A004D487A0063
:103A3000416E790048696768000000004C6F7700AC
:103A4000494E56414C49440044454641554C54006A
:103A5000505245414D424C455F5354415254000031
:103A6000505245414D424C455F53544152545F556D
:103A70005400000053594E435F454E44000000007F
:103A800053594E435F454E445F5554005041434B9C
:103A900045545F454E4400005041434B45545F45FB
:103AA0004E445F5554000000416E74656E6E613087
:103AB00000000000416E74656E6E61310000000010
:103AC00077616974466F7241636B3A25732C726536
:103AD0006D6F76654372633A25732C73796E635705
:103AE0006F726449643A25642C7478416E74656E13
:103AF0006E613A25732C616C74507265616D626CF5
:103B0000654C656E3A25732C6363615065616B5239
:103B10007373693A25732C6363614F6E6C793A2530
:103B2000732C726573656E643A2573005472756503
:103B30000000000046616C7365000000000000009A
:103B400000000000496E76616C69642074696D65DF
:103B5000206D6F646500000061626F727400000088
:103B6000747844656C61793A256400005478486F34
:103B70006C644F66663A257300000000456E616212
:103B80006C65640044697361626C656400000000E8
:103B9000526573756C743A25730000005375636346
:103BA000657373004661696C75726500496E766174
:103BB0006C69642043616C6C00000000496E7661A2
:103BC0006C696420537461746500000052657375FC
:103BD0006C743A25732C6269746C656E6774683A0C
:103BE00025752C73796E63576F7264313A256C7545
:103BF0002C73796E63576F7264323A256C750000CE
:103C000043616E2774207475726E206F6E2072652A
:103C10006365697665207768656E20696E205363F9
:103C2000686564756C6564527800000052783A25C6
:103C3000732C49646C653A25732C54696D653A257B
:103C400075000000436F756C64206E6F74206368AC
:103C5000616E67652072656365697665207374615E
:103C6000746520272564270043616E6E6F7420659C
:103C70006E746572205363686564756C6564527810
:103C8000207768656E206E6F7420696E2049646CC1
:103C9000652E0000496E76616C69642073746172F0
:103CA000744D6F646520737065636966696564004F
:103CB000496E76616C696420656E644D6F64652041
:103CC000737065636966696564000000436F756CB5
:103CD00064206E6F742073746172742073636865FE
:103CE00064756C656420726563656976652025641A
:103CF0000000000052784F7074696F6E733A46612D
:103D0000696C65640000000073746F7265437263D0
:103D10003A25732C69676E6F7265437263457272E0
:103D20006F72733A25732C656E61626C65447561C0
:103D30006C53796E633A25732C747261636B4162C4
:103D40006F727465643A25732C72656D6F76654188
:103D50007070656E646564496E666F3A25732C7287
:103D600078416E74656E6E613A25732C6672616D72
:103D7000654465743A25732C736B697044434361E1
:103D80006C3A25732C736B697053796E7468436158
:103D90003A257300496E76616C69642073747265AC
:103DA000616D206D6F6465004469726563744D6F69
:103DB0006465206E6F7420656E61626C65640000DE
:103DC00044697265637454783A2573004469726576
:103DD00063744D6F64652052782F5478206E6F7431
:103DE00020656E61626C65642027256427000000F1
:103DF000524653454E53452053656C65637469764E
:103E000065204F4F4B204D6F646520556E73757064
:103E1000706F727465640000524653454E534520DE
:103E2000456E6572677920446574656374204D6FD3
:103E3000646520556E737570706F727465640000F0
:103E4000454D3A257525732C53657269616C576130
:103E50006B6575703A25732C526653656E73653ABF
:103E600025732C526653656E73697469766974792B
:103E70003A25732C427574746F6E57616B6575705B
:103E80003A257300736C656570576F6B65000000B1
:103E9000454D3A257525732C53657269616C5761E0
:103EA0006B6575703A25732C526653656E73656445
:103EB0003A25732C5061636B657452783A25732CE4
:103EC000427574746F6E57616B6575703A25732C0B
:103ED000526655733A257500436F756C64206E6F9A
:103EE00074207374617274207265636569766520ED
:103EF000616674657220736C65657000496E7661E9
:103F00006C696420454D206D6F64652025752028FF
:103F100076616C696420302D342900005246534587
:103F20004E534520556E737570706F7274656400E2
:103F3000726653656E736564436865636B00000069
:103F4000526653656E7365643A25732C52665573D9
:103F50003A257500747854696D65506F733A25730E
:103F600000000000496E76616C69642054696D65DB
:103F7000506F736974696F6E202575202876616CA7
:103F8000696420302D25752900000000727854697D
:103F90006D65506F733A257300000000486F6C64C4
:103FA00052783A2573000000939F0100939F01000F
:103FB00087C9010087C90100A5C90100A5C9010081
:103FC000A9C90100A9C90100999F0100999F010099
:103FD000B7750100B7750100EF750100EF750100BD
:103FE00005760100057601005A2D57617665206E31
:103FF0006F742073757070706F72746564206F6E6B
:1040000020746869732063686970000052535349D3
:104010005F415645524147455F444F4E45000000C1
:1040200052585F41434B5F54494D454F5554000032
:1040300052585F4649464F5F414C4D4F53545F467F
:10404000554C4C0052585F5041434B45545F5245CC
:10405000434549564544000052585F505245414D32
:10406000424C455F4C4F53540000000052585F5083
:104070005245414D424C455F444554454354000030
:1040800052585F53594E43315F44455445435400A1
:1040900052585F53594E43325F4445544543540090
:1040A00052585F4652414D455F4552524F520000B3
:1040B00052585F4649464F5F46554C4C0000000041
:1040C00052585F4649464F5F4F564552464C4F57F0
:1040D0000000000052585F414444524553535F462C
:1040E000494C54455245440052585F54494D454F40
:1040F000555400005343484544554C45445F52587D
:104100002F54585F535441525445440052585F5302
:1041100043484544554C45445F52585F454E440022
:1041200052585F5343484544554C45445F52585F8D
:104130004D4953534544000052585F5041434B454D
:10414000545F41424F5254454400000052585F466C
:10415000494C5445525F50415353454400000000C0
:1041600052585F54494D494E475F4C4F53540000DD
:1041700052585F54494D494E475F44455445435456
:104180000000000052585F4348414E4E454C5F4886
:104190004F5050494E475F434F4D504C4554452F6B
:1041A00052585F445554595F4359434C455F5258E8
:1041B0005F454E44000000004945454538303231E6
:1041C00035345F444154412F5A574156455F4C5254
:1041D0005F41434B2F5F524551554553545F434F09
:1041E0004D4D414E442F54585F4D464D5F4255460C
:1041F0004645525F444F4E45000000005A57415615
:10420000455F4245414D000054585F4649464F5F67
:10421000414C4D4F53545F454D50545900000000E0
:1042200054585F5041434B45545F53454E54000032
:10423000545841434B5F5041434B45545F53454EA7
:104240005400000054585F41424F5254454400000E
:10425000545841434B5F41424F5254454400000083
:1042600054585F424C4F434B45440000545841431F
:104270004B5F424C4F434B454400000054585F5540
:104280004E444552464C4F5700000000545841439D
:104290004B5F554E444552464C4F570054585F4370
:1042A00048414E4E454C5F434C4541520000000092
:1042B00054585F4348414E4E454C5F425553590058
:1042C00054585F4343415F52455452590000000027
:1042D00054585F53544152545F434341000000001F
:1042E00054585F53544152544544000054585F534E
:1042F00043484544554C45445F54585F4D495353DA
:1043000045440000434F4E4649475F554E5343488E
:104310004544554C45440000434F4E4649475F5382
:1043200043484544554C454400000000534348452C
:1043300044554C45445F53544154555300000000CC
:1043400043414C5F4E4545444544000052465F534F
:10435000454E53454400000050415F50524F544574
:104360004354494F4E0000005349474E414C5F446F
:10437000455445435445440049454545383032315C
:1043800035345F4D4F44455357495443485F535468
:1043900041525400494545453830323135345F4D3E
:1043A0004F44455357495443485F454E440000002D
:1043B0004445544543545F525353495F5448524512
:1043C00053484F4C4400000068656C64527850724A
:1043D0006F63657373000000556E65787065637474
:1043E000656420696E76616C6964207061636B65D9
:1043F0007448616E646C6500556E657870656374B1
:1044000065642076616C6964207061636B657448D3
:10441000616E646C65000000726573657400000075
:104420004170703A25732C4275696C743A25732C6F
:1044300043617573653A3078257800005241494CE4
:104440007465737400000000556E6B6E6F776E00BC
:104450006173736572740000636F64653A25642C40
:104460006C696E653A25642C6D6573736167653A96
:1044700025730000417070656E64656420696E6626
:104480006F206D697373696E672066726F6D20525D
:1044900078207061636B657400000000526563658D
:1044A000697665204649464F20746F6F20736D61B1
:1044B0006C6C20666F722049522063616C69627275
:1044C0006174696F6E0000004572726F72207265D0
:1044D0006164696E67206261636B207061636B6504
:1044E00074207061796C6F616400000052656365CF
:1044F000697665206669666F20656E7472792068DA
:10450000617320696E76616C69642073746174757F
:104510007300000052656365697665206669666FA1
:1045200020656E74727920626164207061636B65CE
:1045300074206C656E67746800000000556E6162DF
:104540006C6520746F20636F6E6669677572652095
:10455000726164696F20666F722049522063616CDA
:104560006962726174696F6E000000005265616378
:1045700068656420756E6578706563746564207322
:1045800074617465207768696C652068616E646C1D
:10459000696E67205278206669666F206576656E61
:1045A000747300005265616368656420756E657898
:1045B00070656374656420737461746520776869DD
:1045C0006C652068616E646C696E672052584C455A
:1045D0004E206669666F206576656E747300000014
:1045E0005265616368656420756E65787065637493
:1045F0006564207374617465207768696C652068F0
:10460000616E646C696E67205478206669666F20FD
:104610006576656E74730000526561636865642039
:10462000756E657870656374656420737461746514
:10463000207768696C652068616E646C696E6720BC
:1046400054782041434B206669666F206576656E1D
:10465000747300004E6F206D656D6F727920746FFA
:104660002073746F7265207265636569766520706A
:1046700061636B65740000005061636B6574206C4E
:10468000656E677468206C6F6E6765722074686110
:104690006E20746865207265636569766520464999
:1046A000464F2073697A6500496E76616C696420B3
:1046B000726164696F20636C6F636B2070726573E5
:1046C00063616C65720000004572726F72207379CD
:1046D0006E6368726F6E697A696E672074686520B0
:1046E0005241494C2074696D656261736520616651
:1046F00074657220736C65657000000056434F202E
:104700006672657175656E6379206F75747369641F
:104710006520737570706F727465642072616E6766
:1047200065000000526164696F2061637469766599
:10473000207768696C65206368616E67696E6720C1
:104740006368616E6E656C7300000000496E76618F
:104750006C69642053796E74682056434F435452F9
:104760004C206669656C642063616C63756C617470
:10477000696F6E004E657374656420617474656D55
:10478000707420746F206C6F636B20746865207385
:10479000657175656E636572000000005253534980
:1047A00020617665726167696E6720656E61626C13
:1047B000656420776974686F757420612076616C18
:1047C00069642063616C6C6261636B00496E766141
:1047D0006C69642064796E616D6963206672616DD5
:1047E00065206C656E6774682073657474696E67A4
:1047F0002070726F7669646564202864666C426913
:1048000074732900556E61626C6520746F20736546
:10481000656420726164696F2070736575646F20D0
:1048200072616E646F6D206E756D62657220676572
:104830006E657261746F720054696D656F75742076
:104840006578636565647320454652333258473155
:104850002072656769737465722073697A650000F8
:10486000496E76616C69642074696D657220636855
:10487000616E6E656C20737065636966696564005E
:1048800054696D65722076616C7565206C61726724
:104890006572207468616E205241494C2074696DC4
:1048A00065626173650000004C425420636F6E6660
:1048B00069672065786365656473204546523332C5
:1048C0005847312072656769737465722073697A1D
:1048D000650000004465707265636174656420431F
:1048E000534D412F4C42542072657472792063619C
:1048F0006C6C6261636B20756E657870656374655E
:10490000646C792063616C6C65640000436F756C46
:1049100064206E6F742073796E6368726F6E697A4B
:1049200065205241494C2074696D65626173652050
:104930007769746820746865205254430000000051
:10494000436C6F636B20736F75726365206E6F7459
:104950002072656164790000417474656D707465DE
:104960006420746F20736574205241494C2074692F
:104970006D696E677320746F20696E76616C69640F
:104980002076616C756500004E554C4C2077617344
:1049900020737570706C69656420617320612052AA
:1049A00041494C5F48616E646C655F742061726759
:1049B000756D656E740000005363686564756C65A1
:1049C000642074696D6572206E6F742072756E6EEE
:1049D000696E670041504920696D70726F70657231
:1049E0006C792063616C6C6564207768696C652004
:1049F00070726F746F636F6C20696E616374697637
:104A0000650000004E6F20616374697665206861FF
:104A10006E646C6520616674657220737769746377
:104A200068000000526573657276656420666F7277
:104A30002066757475726520757365004E6F206110
:104A400063746976652068616E646C6520666F7258
:104A5000207363686564756C65642072780000007B
:104A6000496E76616C69642068616E646C6520666D
:104A70006F72207363686564756C65642074780078
:104A8000496E6163746976652068616E646C652047
:104A9000666F72207363686564756C6564207478F2
:104AA00000000000496E76616C696420636F6E6679
:104AB000696720696E64657820746F207377697404
:104AC000636820746F0000004E6F20616374697624
:104AD000652068616E646C6520666F722073696E14
:104AE000676C652070726F746F636F6C00000000FC
:104AF000546869732066756E6374696F6E2069739C
:104B0000206465707265636174656420616E642001
:104B10006D757374206E6F742062652063616C6CB8
:104B2000656400004D756C746970726F746F636FAB
:104B30006C207461736B2073746172746564207788
:104B4000697468206E6F206576656E7420746F20BE
:104B500072756E00496E76616C696420696E746569
:104B6000727275707420656E61626C65640000001D
:104B7000506F77657220636F6E76657273696F6EC2
:104B80002066756E6374696F6E732063616C6C650B
:104B900064206265666F7265206375727665732046
:104BA0007765726520696E697469616C697A65649C
:104BB000000000004469766973696F6E2062792095
:104BC0007A65726F0000000046756E6374696F6EDF
:104BD0002063616E6E6F742062652063616C6C652A
:104BE0006420776974686F7574206163636573739B
:104BF00020746F20746865206861726477617265E3
:104C000000000000506F696E7465722070617261FF
:104C10006D6574657220776173207061737365646C
:104C2000206173204E554C4C00000000496E7661A7
:104C30006C6964207461736B207479706520706195
:104C40007373656420746F205241494C5F536574DF
:104C50005461736B5072696F72697479000000005F
:104C600053796E746820726164696F20636F6E6639
:104C700069672062756666657220666F7220636878
:104C8000616E6E656C20686F7070696E6720746FFE
:104C90006F20736D616C6C00427566666572207082
:104CA000726F766964656420666F72205258204383
:104CB00068616E6E656C20486F7070696E67206900
:104CC0007320746F6F20736D616C6C00496E766138
:104CD0006C696420616374696F6E20776173206111
:104CE0007474656D70746564206F6E2061206D6FE3
:104CF00064756C6500000000546865207261646929
:104D00006F20636F6E66696720666F7220746869D2
:104D100073206368616E6E656C206973206E6F74BA
:104D200020636F6D70617469626C65207769746867
:104D3000206368616E6E656C20686F7070696E6765
:104D4000000000004368616E6E656C206368616EF0
:104D50006765206661696C65640000004174746574
:104D60006D7074656420746F207265616420696E73
:104D700076616C696420726567697374657200009E
:104D800043616E2774207265616420726567697380
:104D90007465722076616C75652066726F6D204E49
:104DA000554C4C207374617465000000444D5020D4
:104DB000726164696F20636F6E6669672063616307
:104DC00068696E67206661696C6564004E554C4C7D
:104DD0002077617320737570706C696564206173EE
:104DE0002061205241494C5F537461746554726173
:104DF0006E736974696F6E735F7420617267756D2D
:104E0000656E74004C444D41207472616E7366652A
:104E100072206661696C656400000000417474650D
:104E20006D7074656420746F2077616B6520757098
:104E3000207769746820696E76616C6964205254C9
:104E400043432073796E6320646174610000000045
:104E5000526164696F2073657175656E6365722058
:104E60006869742061206661756C7420636F6E647C
:104E70006974696F6E000000427573206661756C1D
:104E8000740000005468652063757272656E74204A
:104E9000726164696F20636F6E6669672063616E1B
:104EA0006E6F74206265207573656420776974681D
:104EB000207061636B65742066696C746572696EDD
:104EC00067000000526574696D696E6720636F6EDC
:104ED00066696775726174696F6E206572726F7250
:104EE0000000000054582043524320636F6E6669EF
:104EF0006775726174696F6E20697320636F727277
:104F0000757074005468652063757272656E7420E4
:104F1000504120636F6E66696720646F6573206E11
:104F20006F7420616C6C6F7720666F722074686993
:104F300073206F7065726174696F6E0054686520CC
:104F400073657175656E6365722073656C656374F6
:104F5000656420616E20696E76616C6964205041E1
:104F600000000000496E76616C69642F756E737580
:104F700070706F72746564206368616E6E656C201A
:104F8000636F6E66696700005468652064796E61BE
:104F90006D6963206672616D65206C656E6774680B
:104FA00020636F6E66696775726174696F6E2069E0
:104FB0007320696E76616C69640000004661696CFB
:104FC000656420746F20656E61626C6520454D31AB
:104FD0005020656E65726779206D6F646500000012
:104FE0004661696C656420746F2064697361626CEA
:104FF0006520454D315020656E65726779206D6F73
:10500000646500004661696C656420746F206469A2
:105010007361626C6520525443432073796E6368F8
:10502000726F6E697A6174696F6E00004D756C7491
:105030006974696D6572206C696E6B6564206C695A
:10504000737420636F727275707465640000000081
:10505000556E61626C6520746F20636F6E66696760
:1050600075726520726164696F20666F7220746565
:105070006D70657261747572652063616C696272CE
:105080006174696F6E000000496E76616C6964201E
:1050900045464620636F6E66696775726174696F15
:1050A0006E000000496E76616C696420524646507D
:1050B0004C4C20636F6E66696775726174696F6EC0
:1050C000000000005365637572652061636365735A
:1050D00073206661756C74005359535254433020E9
:1050E0006E6F742072756E6E696E670052616469CE
:1050F0006F20436F6E666967757261746F72206EA0
:105100006F74207570646174656400004661696C39
:10511000656420746F2073657420746865206576FB
:10512000656E7420666F7220636F6E666967757254
:1051300061626C65205253534920746872657368CC
:105140006F6C640074696D657243620054696D65CB
:10515000724578706972656443616C6C6261636BFF
:105160003A25752C436F6E6669677572656445787C
:105170007069726554696D653A257500747850617F
:10518000636B657400000000747853746174757308
:105190003A4572726F722C6572726F7252656173EA
:1051A0006F6E3A547820756E646572666C6F772006
:1051B0006F722061626F72742C6572726F72436FCE
:1051C00064653A30782578253038780074785374DF
:1051D000617475733A4572726F722C6572726F7278
:1051E000526561736F6E3A547820626C6F636B65C1
:1051F000642C6572726F72436F64653A30782578FB
:105200002530387800000000747853746174757329
:105210003A4572726F722C6572726F725265617369
:105220006F6E3A53636865645478206D6973736573
:10523000642C6572726F72436F64653A30782578BA
:1052400025303878000000007478537461747573E9
:105250003A4572726F722C6572726F725265617329
:105260006F6E3A5478206368616E6E656C2062756B
:1052700073792C6572726F72436F64653A3078256A
:105280007825303878000000747853746174757331
:105290003A4368616E6E656C436C65617200000034
:1052A000727841636B54696D656F7574000000001E
:1052B00061636B54696D656F75744475726174696F
:1052C0006F6E3A25640000006368616E676543682D
:1052D000616E6E656C000000464154414C2C2063A9
:1052E000616C6C20746F205241494C5F5374617241
:1052F0007452782829206661696C656420282575B8
:10530000290000007478456E6400000074785374BE
:10531000617475733A25732C7472616E736D697460
:105320007465643A25752C6C617374547854696D96
:10533000653A25752C74696D65506F733A25752C27
:105340006C617374547853746172743A25752C636C
:105350006361537563636573733A25752C66616980
:105360006C65643A25752C6C617374547853746160
:105370007475733A30782578253038782C747852E3
:10538000656D61696E3A25642C697341636B3A46B9
:10539000616C736500000000436F6D706C6574652F
:1053A000000000004572726F72000000506172745C
:1053B00069616C0074785374617475733A25732C49
:1053C0007472616E736D69747465643A25752C6CC2
:1053D000617374547854696D653A25752C74696DE0
:1053E00065506F733A25752C6661696C65643A2562
:1053F000752C6C61737454785374617475733A309E
:10540000782578253038782C697341636B3A54726B
:10541000756500006C656E3A300000006C656E3A90
:1054200025642C74696D6555733A25752C74696D06
:1054300065506F733A25752C6372633A25732C6639
:10544000696C7465724D61736B3A307825782C7293
:105450007373693A25642C6C71693A25642C706801
:10546000793A256400000000506173730000000069
:105470004661696C00000000697341636B3A2573F3
:105480002C73796E63576F726449643A25642C619A
:105490006E74656E6E613A25642C6368616E6E652C
:1054A0006C486F704964783A25642C6368616E6E4D
:1054B000656C3A25750000005472756500000000A7
:1054C00046616C736500000065643135343A2575BA
:1054D0002C6C71693135343A25750000667265713E
:1054E0004F66667365743A496E76616C6964000054
:1054F000667265714F66667365743A2564000000D4
:105500006C656E3A256400007B7061796C6F616434
:105510003A000000203078252E3278007072696ED3
:10552000745261696C4576656E747300556E6B6E6E
:105530006F776E205241494C204576656E74733A00
:105540003078257825303878000000006576656E63
:105550007400000074696D657374616D703A25752F
:105560002C6576656E744E616D653A5241494C5FAB
:105570004556454E545F257300000000536570206A
:10558000323720323032322030383A33343A3337FF
:10559000000000000C4000002040000030400000EF
:1055A00044400000584000006C4000008040000073
:1055B00090400000A0400000B0400000C04000004B
:1055C000D4400000E8400000F44000000C4100001E
:1055D00020410000384100004C41000060410000C3
:1055E0007041000084410000B8410000FC4100000F
:1055F0000842000020420000304200004442000007
:1056000050420000604200006C4200007C420000FA
:105610008C4200009C420000B0420000C0420000EA
:10562000D0420000E0420000EC42000004430000D1
:10563000184300002C430000404300004C4300008E
:105640005843000068430000784300009443000082
:10565000B04300006170704D6F646500546F6E65FB
:1056600000000000504E3900313053747265616D96
:1056700000000000546F6E6550686173654E6F697D
:105680007365000052616D7053747265616D000046
:10569000546F6E6553686966746564004E6F6E651D
:1056A0000000000053747265616D0000436F6E74FA
:1056B000696E756F757354780000000044697265F7
:1056C00063744D6F646500005061636B657454785A
:1056D000000000005363686564756C65645478006D
:1056E0005363685478416674657252780000000014
:1056F00052784F766572666C6F7700005478556EFD
:10570000646572666C6F7700547843616E63656C94
:1057100000000000526653656E73650050455200EC
:10572000424552005363686564756C656452780045
:1057300025733A456E61626C6564000025733A45D5
:105740006E61626C65642C53747265616D4D6F643B
:10575000653A25732C54696D653A25750000000083
:1057600025733A456E61626C65642C25733A446911
:105770007361626C65642C53747265616D4D6F6406
:10578000653A25732C54696D653A25750000000053
:1057900025733A456E61626C65642C25733A4469E1
:1057A0007361626C65642C54696D653A25750000FF
:1057B00043616E27742025732025732064757269F8
:1057C0006E67202573000000656E61626C650000E5
:1057D00064697361626C65005C5600006456000089
:1057E0006856000074560000845600009056000071
:1057F0009C560000A45600005C560000AC56000009
:10580000BC560000C8560000D4560000E056000008
:10581000F0560000FC560000085700001457000026
:105820001C57000020570000245700000000000013
:105830000000000000000000010000000000000067
:105840000200000000010102010202030102020342
:10585000020303044E65656420746F20626520694D
:105860006E202573206D6F64652C206E6F7420256B
:10587000732C20666F72207468697320636F6D6D7E
:10588000616E640049646C650000000052784163F9
:105890007469766500000000547841637469766528
:1058A00000000000496E61637469766500000000C5
:1058B000556E6B6E6F776E0041637469766500009C
:1058C0004E6F4672616D65004E65656420746F2091
:1058D000626520696E20257320726164696F207390
:1058E0007461746520666F72207468697320636FD9
:1058F0006D6D616E640000004175746F0000000002
:10590000416E74656E6E613000000000416E74651A
:105910006E6E6131000000007278457272466D74DF
:10592000000000007278457272466C74000000003E
:10593000727845727241627400000000727845729C
:10594000724F76660000000072784572724372638F
:105950000000000072785061636B65740000000005
:1059600072784572723F3F3F000000005A576176DF
:10597000654265616D4672616D6500006E6F6465BC
:1059800049643A307825782C6368616E6E656C489E
:105990006F704964783A25642C6C724265616D3A87
:1059A00025732C6C724265616D5478506F77657207
:1059B0003A25642C6265616D527373693A256400FF
:1059C0006D756C746954696D657243620000000006
:1059D00054696D65724578706972656443616C6C79
:1059E0006261636B3A25752C436F6E6669677572E9
:1059F000656445787069726554696D653A25752CE2
:105A00004D756C746954696D6572496E6465783A58
:105A100025640000676574417667527373690000FE
:105A2000436F756C64206E6F7420726561642052E0
:105A30005353492E00000000727373693A257300B6
:105A40006D69737365645261696C41707045766508
:105A50006E747300636F756E743A257500000000F4
:105A6000726164696F00000046726571487A3A2578
:105A7000752C4D6F64756C65496E666F3A3078258C
:105A80003038782C4D6F64756C654E616D653A25C4
:105A9000730000000000000073797374656D0000EE
:105AA00046616D696C793A25732C46616D233A2500
:105AB000752C436869705265763A25752E25752CCC
:105AC000736469643A25752C506172743A30782594
:105AD00030387800454652333258473231000000A2
:105AE0005266506174683A25640000004572726F16
:105AF0007220616C6C6F636174696E6720524D52E5
:105B0000206D656D6F72792E00000000417267751F
:105B10006D656E7420636F756E7420646F6573209D
:105B20006E6F74206D61746368206E756D6265724E
:105B3000206F6620617267756D656E74732E00004C
:105B40004E756D626572206F6620617267756D6556
:105B50006E74732067726561746572207468616E1B
:105B6000206C6F63616C206275666665722E000042
:105B70004572726F722077726974696E6720746FF4
:105B8000207374727563747572652E00436F6D6D4A
:105B9000616E645374617475733A537563636573AE
:105BA00073000000496E636F7272656374206E75D6
:105BB0006D626572206F6620617267756D656E74C7
:105BC000730000004572726F7220757064617469B1
:105BD0006E672073747275637475726500000000DF
:105BE0004E65656420746F20626520696E2049648B
:105BF0006C6520726164696F2073746174652066DE
:105C00006F72207468697320636F6D6D616E6400DC
:105C10000A5241494C746573740A0000527820435B
:105C20006F756E743A202530356C750054782043BA
:105C30006F756E743A202530356C75004368616E5F
:105C40006E656C3A202564002020205478202020A6
:105C5000202052780000000000186C6C10CE38082C
:105C6000600C0000000000007C307C7CC6FE7CFEE6
:105C70007C7C000070001C7C7C7C7E7C7EFEFE7C3C
:105C8000C63C78C606C6C67C7E7C7E7C7EC6C6C602
:105C9000C6C6FE7C007C10000C00060060003800C8
:105CA000060000060C0000000000000000000000DC
:105CB0000000003018188C000000000000186CFE76
:105CC000FC6A2C1830186C18000000C0C638C6C614
:105CD000C606C6C0C6C61818387C38C6C6C6C6C6EC
:105CE000C60606C6C618306606EECEC6C6C6C6C608
:105CF00018C6C6C6C6C6C00C066038000C00060032
:105D000060000C00061830060C00000000000000C7
:105D100018000000000000181830D6000000000035
:105D2000001848FE162E2C18183038180000006095
:105D3000C63060C0C6060660C6C618181C7C70C691
:105D4000F6C6C606C6060606C618303606FEDEC607
:105D5000C6C6C60618C6C6C66CC6600C0C606C000B
:105D6000043C3E3C7C3C3C3C3E0000660C6E3E3CB1
:105D70003E3C363C186666C666667E181830620081
:105D8000000000000018006C7C10DC001830FE7E63
:105D90001C7E0030C6303070FE7E7E307CFC000001
:105DA0000E00E070F6FE7E06C61E1EF6FE18301EC1
:105DB00006D6F6C67EC67E7C18C6C6D638FC300C23
:105DC0001860C6000060660666660C6666183036A7
:105DD0000CD6666666666E067C6666C63C66300CE9
:105DE0000060000000000000000000FED0E8660037
:105DF0001830387E1C7E1C18C63018C0C0C0C618AB
:105E0000C6C018181C7C703076C6C606C60606C604
:105E1000C618303606C6E6C606B6C6C018C6C6FEE2
:105E20006CC0180C30600000007C6606667E0C7C3E
:105E30006618301E0CD666663E56063C186666D658
:105E4000187C18181830000000000000001800FE30
:105E50007EAC660030186C1818001C0CC6300CC6DE
:105E6000C0C6C60CC6C61818387C380006C6C6C6DA
:105E7000C60606C6C618366606C6C6C60666C6C6C0
:105E800018C66CEEC6C00C0C606000FE00666606AC
:105E900066060C60661836360CC666660626066010
:105EA00018663CD63C600C1818300000000000005A
:105EB0000018006C10E6DC00600C00180C001C06DA
:105EC0007C78FE7CC07C7C067C7C000C70001C30E6
:105ED0007CC67E7C7EFE06FCC63C1CC6FEC6C67C1E
:105EE00006DCC67C187C38C6C67EFE7CC07C00FE04
:105EF000007C3E3C7C3C0C3E66701C6638C6663CB2
:105F0000065C063E707C18FC663E7E301818000069
:105F10000000000000000000000000000000000081
:105F20000000000000000000000000000000000071
:105F30000000000000000000000000000000000061
:105F40000000000000000000000000000000000051
:105F50000000000000000000000000000000000041
:105F60000000000000000000000000000000000031
:105F70000000000000000000585C000020030164E5
:105F800008080200010000001E00000305000000D8
:105F90000000000040420F0005010000000000006A
:105FA00000000000000000008000800001010000EF
:105FB000E0C810003C060200436F6E74726F6C20E4
:105FC0005241494C206576656E74732E00000000C6
:105FD0006576656E74734D61736B3C33313A303E58
:105FE0001F6576656E747356616C7565733C3331ED
:105FF0003A303E1F6576656E74734D61736B3C3647
:10600000333A33323E0A2020202020202020202036
:10601000202020202020202020205B75696E7433F2
:10602000326F70745D206576656E747356616C7541
:1060300065733C36333A33323E1F00005265736558
:1060400074732074686520545820616E642052581F
:1060500020636F756E746572732E0000436F6E74EB
:10606000726F6C204C45447320616E64204C434435
:10607000207065726970686572616C732E00000033
:106080005B303D44697361626C655D20313D456EF6
:1060900061626C651F000000436F6E74726F6C204C
:1060A0006173796E6368726F6E6F7573207374615C
:1060B000747573207072696E7473202872785061E1
:1060C000636B65742C7478456E642C7478457272B9
:1060D0006F72292E00000000303D44697361626CCC
:1060E00065205B313D456E61626C655D1F0000009F
:1060F00053686F772077686574686572206E6F7477
:10610000696669636174696F6E73206F7220706570
:10611000726970686572616C732061726520656E6A
:1061200061626C65642E0000476574207665727349
:10613000696F6E20696E666F726D6174696F6E2E25
:106140000000000047657420766572626F736520F9
:1061500076657273696F6E20696E666F726D6174B9
:10616000696F6E2E00000000536574205054492062
:1061700070726F746F636F6C20666F72204E6574FF
:10618000776F726B20416E616C797A65722E0000B8
:10619000303D437573746F6D20323D546872656194
:1061A0006420333D424C4520343D436F6E6E656341
:1061B0007420353D5A696762656520363D5A2D5712
:1061C0006176651F00000000476574205054492027
:1061D000636F6E66696775726174696F6E2E000019
:1061E000436F6E74726F6C20616C6C207072696E9C
:1061F00074696E6720696E205241494C74657374EE
:106200002C2065786365707420434C492E00000093
:10621000436F6E74726F6C2072656365697665207A
:106220006D6F64652E000000436F6E66696775725E
:1062300065207363686564756C6564207265636569
:106240006976652E00000000737461727454696D84
:106250006555731F2772656C273D52656C617469C3
:1062600076652027616273273D4162736F6C757498
:10627000651F656E6454696D6555731F2772656C83
:10628000273D52656C6174697665202761627327CA
:106290003D4162736F6C7574651F72785472616EE4
:1062A00073456E6453636865643A205B305D2F31DB
:1062B0000A202020202020202020202020202020F4
:1062C00020202020205B75696E74386F70745D200B
:1062D00068617264456E643A205B305D2F311F0047
:1062E00053686F772F436F6E6669677572652072AA
:1062F000656365697665206F7074696F6E732028B9
:106300005241494C5F52585F4F5054494F4E732988
:106310002E00000072784F7074696F6E7356616C56
:106320007565733A206269746D61736B206F6620C6
:10633000656E61626C6564206F7074696F6E731F47
:10634000000000005472616E736D697420706163A7
:106350006B65747320776974682063757272656EFB
:1063600074205458206F7074696F6E732E00000093
:106370006E756D626572206F66207061636B657407
:10638000732C20303D636F6E74696E756F7573206A
:10639000756E74696C206E6578742027747820306F
:1063A000271F000053616D6520747820636F6D6D49
:1063B000616E642E205468697320636F6D6D616E29
:1063C0006420697320646570726563617465642E0E
:1063D000000000005363686564756C65206120549B
:1063E00058207769746820737065636966696564AD
:1063F0002064656C617920616674657220656163F3
:10640000682052582E00000064656C617955733A1B
:1064100020303D44697361626C651F0053686F777B
:106420002F436F6E666967757265207472616E7353
:106430006D6974206F7074696F6E732028524149C2
:106440004C5F54585F4F5054494F4E73292E0000F3
:1064500074784F7074696F6E7356616C7565733ABA
:10646000206269746D61736B206F6620656E616276
:106470006C6564206F7074696F6E731F000000009C
:10648000436F6E666967757265206669786564201A
:106490006C656E677468207061636B6574206F70E3
:1064A00065726174696F6E2E000000006669786520
:1064B000644C656E6774683A207061796C6F6164D2
:1064C0002062797465731F005365742074686520B9
:1064D0007472616E736D697420706F7765722E20AF
:1064E00054686520726164696F206D7573742062F1
:1064F000652049444C452E00706F7765723A2064E0
:106500006563692D64426D20756E6C657373202719
:10651000726177272069732061646465641F277244
:106520006177273D756E69747320617265207261B1
:106530007720706F776572206C6576656C1F000040
:1065400047657420746865207472616E736D697438
:1065500020706F77657220696E20646563692D64B1
:10656000426D2E00536574207472616E736D697490
:1065700020504120636F6E66696775726174696F40
:106580006E2E000070614D6F64651F6D696C6C69E3
:10659000766F6C74731F72616D7054696D6555739D
:1065A0001F00000047657420746865207472616E76
:1065B000736D697420504120636F6E6669677572F0
:1065C0006174696F6E2E0000476574206D696E20DE
:1065D000616E64206D617820706F7765724C6576AE
:1065E000656C20666F72206120706F776572206D18
:1065F0006F64652E00000000706F7765724D6F64E8
:10660000651F0000436F6E74726F6C206175746F4C
:106610006D617469632050412073656C65637469B2
:106620006F6E206261736564206F6E2074686520F0
:10663000545820706F776572206C6576656C2E00FB
:10664000303D44697361626C6520313D456E616225
:106650006C651F00436F6E66696775726520656EB5
:10666000747269657320696E20746865206465665C
:1066700061756C74205041204175746F204D6F64BA
:106680006520706C7567696E2E000000737461720E
:106690007420496E6465781F6D696E206D61782085
:1066A0006D6F64652062616E643A205041206175AF
:1066B000746F20636F6E66696720656E74726965BA
:1066C000731F0000537765657020545820706F77F2
:1066D000657220666F7220746865206375727265DA
:1066E0006E7420504120627920746F6E696E67204D
:1066F00061742065616368206C6576656C2E0000AE
:1067000041646A7573742074686520686172647787
:106710006172652773204C51492076616C75652044
:10672000666F722072656365697665642070616367
:106730006B6574732E0000006F66667365743A2093
:106740007369676E65642076616C756520746F206F
:106750006164640A20202020202020202020202086
:106760002020202020202020546865207265737529
:106770006C74696E67204C514920697320636170A5
:106780007065642077697468696E20302E2E32350A
:10679000352072616E67652E1F000000476574200A
:1067A0005253534920696E2064426D2E204974274C
:1067B0006C6C20626520696E76616C696420696624
:1067C0002072656365697665722069736E2774202F
:1067D00072656164792E00005B303D646F6E2774D2
:1067E00020776169745D20313D7761697420666F3F
:1067F000722076616C696420525353492069662087
:10680000706F737369626C651F0000005377656574
:106810007020706F77657220627920746F6E696E78
:1068200067206C6F772F6869676820696E20612028
:106830007371756172652077617665206661736832
:10684000696F6E2E000000006C6F77506F77657275
:106850003A20646563692D64426D1F6869506F77E3
:1068600065723A20646563692D64426D1F706572BC
:10687000696F6455731F000053746172742041473F
:1068800043205253534920617665726167696E6790
:106890002E0000006176657261676554696D65550B
:1068A000731F6368616E6E656C3A20696620646967
:1068B00066666572656E74207468616E20637572B9
:1068C00072656E74206368616E6E656C1F000000F7
:1068D00047657420414743205253534920617665F0
:1068E000726167696E6720726573756C742E000043
:1068F000436F6E74726F6C20746F6E65207472617A
:106900006E736D697373696F6E2E0000303D44695C
:106910007361626C6520313D456E61626C651F611B
:106920006E74656E6E613A205B305D2F310A2020F7
:106930002020202020202020202020202020202057
:1069400020205B75696E7433326F70745D206D6FDB
:1069500064653A205B305D2F313D70686173654E30
:106960006F6973651F000000436F6E74726F6C2057
:1069700073747265616D207472616E736D69737387
:10698000696F6E2E00000000303D44697361626CD7
:106990006520313D456E61626C651F73747265617F
:1069A0006D4D6F64653A205B313D504E395D20324C
:1069B0003D3130313020333D70686173654E6F6911
:1069C000736520303D746F6E650A202020202020E2
:1069D00020202020202020202020202020205B7527
:1069E000696E7433326F70745D20616E74656E6EA3
:1069F000613A205B305D2F311F0000005072696EDC
:106A000074207468652063757272656E7420737487
:106A10006174757320636F756E746572732E0000F8
:106A20005072696E74207468652063757272656E49
:106A300074204649464F2D72656C6174656420630D
:106A40006F756E746572732E00000000436F6E7474
:106A5000726F6C207472616E736D697420686F6CF4
:106A6000642D6F66662028626C6F636B696E6720A9
:106A70006F66207472616E736D697473292E0000E5
:106A80005365742074686520696E7465722D706139
:106A9000636B65742064656C617920666F72207227
:106AA000657065617465642054582E0064656C617E
:106AB000794D696C6C697365636F6E64731F000058
:106AC0004765742074686520696E7465722D706105
:106AD000636B6574206D696C6C697365636F6E645C
:106AE0002064656C617920666F72207265706561E3
:106AF0007465642054582E005365742054582070D7
:106B000061636B6574207061796C6F616420627978
:106B100074657320666F7220667574757265207473
:106B200072616E736D6974732E0000006F66667318
:106B300065741F6279746530206279746531202E26
:106B40002E2E1F004C696B6520736574547850615C
:106B5000796C6F61642C20627574206C657373208E
:106B6000766572626F73652E0000000053657420B5
:106B7000686F77206D756368206461746120746F3D
:106B8000206C6F616420696E746F20746865205496
:106B900058204649464F20666F72207472616E73AA
:106BA0006D697474696E672E0A20202020202020D1
:106BB000202020202020202020202020204163741D
:106BC00075616C207061636B6574206C656E6774B1
:106BD00068206D61792076617279206261736564E5
:106BE000206F6E20726164696F20636F6E666967E3
:106BF00075726174696F6E2E000000006C656E67BF
:106C0000746842797465731F000000005072696EE9
:106C100074207468652063757272656E74205458B0
:106C2000207061796C6F6164206461746120616EB1
:106C3000642062797465206C656E6774682E00004C
:106C40005065656B2061742074686520737461728F
:106C500074206F6620746865207265636569766567
:106C6000206275666665722E0000000062797465A8
:106C7000733A20312D31301F6F66667365743A2088
:106C80005B305D1F0000000047657420746865205C
:106C900063757272656E74205241494C2074696D3F
:106CA0006520696E206D6963726F7365636F6E64D2
:106CB000732E0000536574207468652063757272CA
:106CC000656E74205241494C2074696D652E000038
:106CD00074696D6555731F00436F6E74726F6C201D
:106CE0007468652064617461206D6574686F647395
:106CF00020666F7220545820616E642052582E0016
:106D000074784D6574686F643A2027706B74272F10
:106D1000276669666F271F72784D6574686F643ADD
:106D20002027706B74272F276669666F271F5241D3
:106D3000494C5F527844617461536F757263655F4B
:106D40007420283E30206E65656473206669666F26
:106D5000206D6F6465290A2020202020202020201B
:106D600020202020202020202020205B75696E74A8
:106D7000386F70745D205241494C5F54784461749F
:106D800061536F757263655F7420283E30206E65B5
:106D90006564732070696E672D706F6E6720627511
:106DA00066666572291F000053657420746865204B
:106DB0007265636569766520627566666572206CCA
:106DC000656E6774682E00006C656E677468427942
:106DD0007465733A2072616E67652036342D52589F
:106DE0005F4255464645525F53495A451F000000D1
:106DF00053657420746865205458204649464F20D6
:106E0000416C6D6F737420456D7470792074687275
:106E10006573686F6C642E007468726573686F6C5C
:106E20006442797465733A2062656C6F7720776885
:106E300069636820746865206576656E7420747275
:106E40006967676572731F005365742074686520F5
:106E50005258204649464F20416C6D6F737420464E
:106E6000756C6C207468726573686F6C642E0000BA
:106E70007468726573686F6C6442797465733A20E4
:106E800061626F7665207768696368207468652041
:106E90006576656E742074726967676572731F002A
:106EA0004D616E75616C20636F6E74726F6C206FD4
:106EB000766572205241494C746573742046494688
:106EC0004F20616374696F6E732E00007478466999
:106ED000666F3A20313D4D616E75616C20303D41E9
:106EE00075746F6D617469631F72784669666F3A75
:106EF00020313D4D616E75616C20303D4175746F80
:106F00006D617469631F00005265616420616E6485
:106F1000207072696E742062797465732066726F76
:106F20006D2072656365697665204649464F207716
:106F300068656E20696E206D616E75616C206D6F85
:106F400064652E00617070656E646564496E666F7D
:106F50003A20313D696E636C756465207061636BC6
:106F60006574206D657461646174611F6279746514
:106F700073546F526561641F5B303D646F6E27749C
:106F80005D20313D73686F772074696D657374613E
:106F90006D7073207769746820617070656E6465C8
:106FA00064496E666F1F000054727920746F206C04
:106FB0006F6164206461746120696E746F20617612
:106FC00061696C61626C65205458204649464F20C7
:106FD00073706163652E0000526573657420746878
:106FE00065207472616E736D697420616E642F6FB9
:106FF000722072656365697665204649464F2E00AA
:1070000074783A20313D7265736574205458204677
:1070100049464F1F72783A20313D7265736574207E
:107020005258204649464F1F0000000049646C65D5
:107030002074686520726164696F2073686F727470
:107040006C792061667465722052582073796E6382
:1070500020776F726420646574656374696F6E2E47
:107060000000000061626F72744F6666736574554C
:10707000731F0000436F6E74726F6C207072696EC4
:1070800074696E67206F662054582041434B20700E
:1070900061636B6574732E00436F6E66696775720A
:1070A0006520616E205258204368616E6E656C20C9
:1070B000486F7070696E672073657175656E636582
:1070C0002E0000006368616E6E656C20686F704D05
:1070D0006F646520706172616D2064656C617955C3
:1070E000733A206120686F70277320636F6E666942
:1070F000672C0A2020202020202020202020202053
:10710000202020202020202020202020202020207F
:1071100020202072657065617420666F7220616442
:10712000646974696F6E616C20686F7073202E2EB5
:107130002E0A202020202020202020202020202057
:10714000202020202020557365206E6F20617267FB
:10715000756D656E747320746F20676574205A2D89
:107160005761766520726164696F20636F6E66692E
:10717000672064656661756C74732E1F00000000E3
:10718000436F6E74726F6C205258206368616E6E2C
:10719000656C20686F7070696E67207072657669C3
:1071A0006F75736C7920636F6E666967757265645D
:1071B0002E0000005B303D44697361626C655D20A8
:1071C000313D456E61626C651F5B303D436F6E748F
:1071D000696E75655D20313D52657374617274200E
:1071E00073657175656E63651F000000436F6E66A1
:1071F0006967757265206F7074696F6E7320666F52
:1072000072206120686F702E2055736520636F6E49
:107210006669675278486F7070696E67206166743E
:1072200065722E00686F70496E6465781F6F7074A8
:10723000696F6E731F727373695468726573686FD8
:107240006C643A2064426D20666F72207468652019
:107250007468726573686F6C64206F7074696F6EA8
:107260001F000000436F6E666967757265206D755B
:107270006C74692D73656E736520666F7220612072
:10728000686F702E2055736520636F6E6669675254
:1072900078486F7070696E672061667465722E0041
:1072A000686F70496E6465781F73796E63446574A6
:1072B00065637455731F707265616D626C655365AB
:1072C0006E736555731F74696D696E6753656E7370
:1072D0006555731F74696D696E67526553656E738A
:1072E0006555731F000000004765742074686520B1
:1072F0006C6174657374205253534920666F722019
:107300006120686F7070696E67206368616E6E657A
:107310006C2E0000686F70496E6465781F00000075
:10732000486F70206163726F7373206120636861BE
:107330006E6E656C2072616E676520746F20736578
:1073400065207468652052535349206469737472D0
:1073500069627574696F6E2E00000000313D5368DC
:107360006F772041534349492D4172742067726100
:10737000706820286E6F6E2D706172736561626C2B
:1073800065206F7574707574291F6D696E4368612F
:107390006E6E656C3A205B305D2D36353533350ABF
:1073A00020202020202020202020202020202020DD
:1073B000202020205B75696E7431366F70745D20FB
:1073C0006D61784368616E6E656C3A20302D5B3676
:1073D000353533355D0A2020202020202020202034
:1073E000202020202020202020204368616E6E6510
:1073F0006C2072616E6765206973206C696D6974B9
:107400006564206279207468652050485920616E57
:107410006420627920686F7070696E6727730A2034
:10742000202020202020202020202020202020205C
:107430002020204D41585F4E554D4245525F4348F4
:10744000414E4E454C532E1F00000000436F6E66A8
:1074500069677572652052582044757479204379A4
:10746000636C696E67206F6620746865207265635F
:1074700065697665722E0000686F704D6F64651FD8
:10748000706172616D65746572287329207B7379F0
:107490006E63557320707265616D55732074696DEC
:1074A000696E67557320726574696D696E6755738F
:1074B0007D1F64656C617955731F6F7074696F6EA1
:1074C000730A20202020202020202020202020207F
:1074D0002020202020205B696E7433326F70745D31
:1074E00020727373695468726573686F6C643A20B4
:1074F00064426D20666F72207468652074687265DE
:1075000073686F6C64206F7074696F6E1F00000089
:10751000436F6E74726F6C205258206475747920BA
:107520006379636C696E672070726576696F7573D5
:107530006C7920636F6E666967757265642E0000F2
:10754000447574794379636C696E673A20303D44C1
:10755000697361626C6520313D456E61626C651FC7
:107560005363686564756C656457616B6575703AE3
:10757000205B303D44697361626C655D20313D453F
:107580006E61626C651F0000204765742074686539
:107590002064656661756C74205258206475747936
:1075A000206379636C6520636F6E666967757261CD
:1075B00074696F6E2E00000053657420616C7465F1
:1075C000726E61746520545820707265616D626CD2
:1075D00065206C656E6774682C20656E61626C65F1
:1075E00064207669612074784F7074696F6E732EB1
:1075F00000000000707265616D626C6542697473B1
:107600001F0000005365742073796E6320776F72DA
:10761000647320616E64207468656972206C656EA5
:107620006774682E2054686520726164696F206DEC
:10763000757374206265206F66662E0062697473CC
:107640003A20322D33321F73796E63576F72643173
:107650001F73796E63576F7264323A205B73616D8A
:10766000652061732073796E63576F7264315D1F9B
:1076700000000000476574207468652073796E63AC
:1076800020776F7264206C656E67746820696E2065
:107690006269747320616E642076616C756528730D
:1076A000292E0000436F6E74726F6C207072696EC9
:1076B00074696E67206F66205258206572726F720F
:1076C000207061636B6574732E000000436F6E74ED
:1076D000726F6C207072696E74696E67206F6620BD
:1076E0005258206672657175656E6379206F6666A3
:1076F000736574732E0000005072696E7420746894
:10770000652064617461207261746573206F662006
:107710007468652063757272656E74205048592EC6
:107720000000000053746F707320616E20696E66F4
:10773000696E69746520707265616D626C65207434
:1077400072616E736D697373696F6E2E0000000055
:10775000536C65657020756E74696C205541525488
:1077600020696E707574206F722052462053656ECA
:107770007365642028696620656974686572206392
:107780006F6E66696775726564292E00656E657235
:1077900067794D6F64653A20302D345B68735D2CDA
:1077A00020666F7220454D31502075736520322060
:1077B0007769746820726164696F206F6E1F4C6511
:1077C000676163793A20526653656E736555730A33
:1077D00020202020202020202020202020202020A9
:1077E0002020202020202020202020202020202099
:1077F0002020202020202020526642616E643A2002
:10780000303D6E6F6E652C313D47487A2C323D4DD0
:10781000487A2C333D626F74680A20202020202093
:107820002020202020202020202020202020202058
:10783000202020206F722053656C65637469766523
:107840003A2053796E63776F72644279746573205E
:1078500053796E63776F726420526642616E641F63
:1078600000000000537461727420526653656E7399
:10787000696E672E000000004C65676163793A20ED
:10788000526653656E736555733B2053656C656333
:10789000746976653A2053796E63776F72644279C2
:1078A0007465731F4C65676163793A205266426163
:1078B0006E643A20303D6E6F6E652C313D47487ADC
:1078C0002C323D4D487A2C333D626F74680A20207B
:1078D00020202020202020202020202020202020A8
:1078E00020202020202020206F722053656C6563AB
:1078F000746976653A2053796E63776F72642052AB
:107900006642616E643A2061732061626F76651F22
:1079100000000000436F6E6669677572652052460D
:1079200053656E73652053656C6563746976652075
:1079300057616B6575702050485920666F722074CE
:1079400072616E736D697474696E672E0000000059
:107950004C6F6164205458204649464F2077697423
:107960006820526653656E73652053656C65637459
:10797000697665284F4F4B29204D6F6465207761EC
:107980006B65207061636B65742E000073796E63A4
:10799000776F72644E756D42797465733A20312D3C
:1079A000341F73796E63576F72643A2073656E7417
:1079B0002066726F6D206C6561737420746F206D2A
:1079C0006F7374207369676E69666963616E742092
:1079D000627974651F000000436F6E666967757297
:1079E00065207468652061646472657373732066D2
:1079F000696C7465722E00006D6174636854616215
:107A00006C651F6F6666736574302073697A6530C4
:107A1000206F6666736574312073697A6531202E34
:107A20002E2E0A2020202020202020202020202050
:107A300020202020202020456E746572206D6F72FA
:107A400065206F66667365747320616E6420736968
:107A50007A65732069662072657175697265642E36
:107A60001F000000436F6E74726F6C20616464725B
:107A70006573732066696C746572696E672E0000A9
:107A8000476574207468652063757272656E742032
:107A90007374617465206F662061646472657373CA
:107AA0002066696C746572696E672E005072696E2B
:107AB00074207468652063757272656E74206164E9
:107AC00064726573732066696C746572696E672091
:107AD0006164647265737365732E0000536574206E
:107AE000612073706563696669632066696C74659B
:107AF00072696E6720616464726573732076616C6D
:107B000075652E006669656C643A20302D311F66FC
:107B1000696C746572496E6465783A20302D331F44
:107B20006164647242797465302061646472427980
:107B3000746531202E2E2E20616464724279746542
:107B4000371F000053657420612073706563696698
:107B500069632066696C746572696E67206164642C
:107B600072657373206D61736B2E00006669656CBE
:107B7000643A20302D311F6269744D61736B1F00B0
:107B8000436F6E74726F6C206164647265737320EE
:107B900066696C746572696E6720666F7220612019
:107BA0007370656369666963206164647265737389
:107BB0002E0000006669656C643A20302D311F6626
:107BC000696C746572496E6465783A20302D331F94
:107BD000303D44697361626C6520313D456E616280
:107BE0006C651F0053746172742061205061636B77
:107BF0006574204572726F722052617465207465DD
:107C000073742E2027706572527820302030272020
:107C100073746F707320746573742E006E756D626B
:107C20006572206F66207061636B6574731F646595
:107C30006C617955731F0000476574207468652076
:107C4000504552207465737420726573756C74733B
:107C50002E20416C736F2073656520737461747599
:107C60007320636F6D6D616E642E00005365742028
:107C70006E756D626572206F66206279746573201F
:107C8000746F207265636569766520696E20424570
:107C900052206D6F64652E006E756D626572206F87
:107CA000662062797465733A20303D6D6178696D44
:107CB000756D2028353336383730393131291F007A
:107CC000436F6E74726F6C2042455220726563651B
:107CD000697665206D6F64652E000000476574202D
:107CE000737461747573206F662063757272656E4C
:107CF00074206F72206C6173742042455220746549
:107D000073742E0A202020202020202020202020D4
:107D10002020202020202020537461747573206956
:107D2000732072657365742062792073657442658F
:107D300072436F6E66696720616E6420626572527D
:107D40007820656E61626C652E00000053686F7765
:107D50002F53657420746865204C4254206D6F6405
:107D60006520666F72207472616E736D6974732E14
:107D700000000000276F6666272F2763736D612759
:107D80002F276C6274271F00476574207468652074
:107D900063757272656E74204C425420706172611A
:107DA0006D65746572732E00536574204C425420C7
:107DB000706172616D65746572732E006D696E42DB
:107DC0006F1F6D6178426F1F74726965731F636303
:107DD000615468726573686F6C641F6261636B6F76
:107DE000666655731F6475726174696F6E55731F93
:107DF00074696D656F757455731F00005365742049
:107E00003830322E31352E3420434341204D6F64BB
:107E1000650000006363614D6F646520303D52531F
:107E2000534920313D5369676E616C20323D525396
:107E300053497C5369676E616C20333D52535349FB
:107E4000265369676E616C20343D416C77617973AC
:107E5000207472616E736D69741F0000436F6E66EB
:107E6000696775726520616E6420656E61626C651C
:107E7000203830322E31352E34206D6F64652E005F
:107E800064656661756C7453746174653A20276922
:107E9000646C65272F277278271F69646C65546F9F
:107EA000527855731F7475726E61726F756E64547B
:107EB000696D6555731F61636B54696D656F75748A
:107EC00055733A20746F2041434B27732073796EAA
:107ED000632D6465746563741F64656661756C7495
:107EE00046503A205B305D2F31204672616D65202F
:107EF00050656E64696E6720666F7220706F6C6C7F
:107F00002041434B731F0000436F6E6669677572B3
:107F1000652074686520726164696F20666F7220E5
:107F2000322E342047487A203830322E31352E34E4
:107F30002E0A202020202020202020202020202049
:107F400020202020202055736520776974682065E3
:107F50006E61626C653830323135342E00000000BD
:107F6000616E744469763A205B303D4469736162A6
:107F70006C655D20313D456E61626C650A20202094
:107F800020202020202020202020202020202020F1
:107F9000205B75696E74386F70745D20636F6578EF
:107FA0003A205B303D44697361626C655D20313D10
:107FB000456E61626C650A20202020202020202050
:107FC00020202020202020202020205B75696E7436
:107FD000386F70745D2066656D3A205B303D446992
:107FE0007361626C655D20313D456E61626C650A4E
:107FF0002020202020202020202020202020202081
:10800000202020205B75696E74386F70745D20636A
:108010007573746F6D3A205B303D4E6F6E655D20F9
:10802000313D437573746F6D311F0000436F6E6691
:1080300069677572652074686520726164696F2074
:10804000666F7220383633204D487A203830322E11
:1080500031352E342047423836382E0A2020202051
:108060002020202020202020202020202020202010
:10807000557365207769746820656E61626C653838
:1080800030323135342E0000436F6E666967757289
:10809000652074686520726164696F20666F722064
:1080A000393135204D487A203830322E31352E3452
:1080B0002047423836382E0A202020202020202039
:1080C00020202020202020202020202055736520E3
:1080D0007769746820656E61626C6538303231355D
:1080E000342E0000436F6E66696775726520383004
:1080F000322E31352E3445206F7074696F6E732EB9
:10810000000000005241494C5F4945454538303236
:108110003135345F454F7074696F6E735F741F0043
:10812000436F6E666967757265203830322E31355F
:108130002E3447206F7074696F6E732E000000003C
:108140005241494C5F494545453830323135345FFD
:10815000474F7074696F6E735F741F00436F6E7466
:10816000726F6C206561726C7920616E642064614D
:108170007461206672616D652070656E64696E67FA
:10818000206C6F6F6B75702E000000006561726C63
:10819000793A20202020205B303D44697361626C75
:1081A000655D20313D456E61626C651F646174617F
:1081B0006672616D65733A5B303D44697361626CF0
:1081C000655D20313D456E61626C651F00000000F9
:1081D000436F6E74726F6C203830322E31352E340E
:1081E000206672616D6520747970652061636365D6
:1081F0007074616E63652E00636F6D6D616E643ABD
:1082000020303D52656A656374205B313D41636394
:108210006570745D1F61636B3A202020205B303DE8
:1082200052656A6563745D20313D416363657074B6
:108230001F646174613A20202020303D52656A65D8
:108240006374205B313D4163636570745D1F6265DB
:1082500061636F6E3A2020303D52656A6563742019
:108260005B313D4163636570745D1F6D756C74694E
:10827000707572706F73653A205B303D52656A6548
:1082800063745D20313D4163636570741F000000BD
:10829000436F6E74726F6C2070726F6D697363756B
:1082A0006F7573206D6F64652E000000436F6E74F0
:1082B000726F6C2077686574686572206E6F646594
:1082C00020697320612050414E20636F6F72646992
:1082D0006E61746F722E0000313D59657320303D20
:1082E0004E6F1F00536574207468652050414E2006
:1082F000494420666F7220612066696C74657269FA
:108300006E6720696E6465782E00000070616E49AA
:10831000641F66696C746572496E6465783A205BA7
:10832000305D2D321F000000536574207468652095
:1083300073686F7274206164647265737320666F12
:108340007220612066696C746572696E6720696E5F
:108350006465782E0000000073686F727441646475
:10836000721F66696C746572496E6465783A205B49
:10837000305D2D321F000000536574207468652045
:108380006C6F6E67206164647265737320666F72D0
:1083900020612066696C746572696E6720696E641D
:1083A00065782E006C6F6E67416464725F301F6C7D
:1083B0006F6E67416464725F311F6C6F6E674164FA
:1083C00064725F321F6C6F6E67416464725F331F4B
:1083D0006C6F6E67416464725F341F6C6F6E6741CF
:1083E0006464725F351F6C6F6E67416464725F36E0
:1083F0001F6C6F6E67416464725F371F66696C74CF
:108400006572496E6465783A205B305D2D321F00DD
:1084100053657420616C6C203830322E31352E3427
:10842000206164647265737320696E666F726D613A
:1084300074696F6E2E00000070616E4964301F73A6
:10844000686F727441646472301F6C6F6E67416450
:108450006472300A2020202020202020202020208C
:1084600020202020202020205B737472696E676FAB
:1084700070745D2070616E4964312073686F72742E
:108480004164647231206C6F6E67416464723120A4
:108490002E2E2E1F0000000053657420646174614D
:1084A0002072657175657374206576656E742070D1
:1084B000726F63657373696E67206C6174656E6358
:1084C000792E00006C6174656E637955731F00002E
:1084D00053657420504852202866697273742031A5
:1084E0002C2032206F722034206279746573292029
:1084F000696E2054782062756666657220616363D8
:108500006F7264696E6720746F0A2020202020201B
:10851000202020202020202020202020202020205B
:108520007468652027666F726D61742720696E70AC
:10853000757420706172616D657465722E0A2020F9
:10854000202020202020202020202020202020202B
:10855000202050485220276672616D654C656E6719
:10856000746827206669656C64206973206465728D
:10857000697665642066726F6D2054784C656E670D
:108580007468207365740A20202020202020202079
:1085900020202020202020202020202020707265F4
:1085A00076696F75736C79207769746820277365B5
:1085B0007454784C656E677468270A202020202048
:1085C0002020202020202020202020202020204685
:1085D0006F7220504852206669656C647320696E22
:1085E000666F2C20726566657220746F2038303299
:1085F0002E31352E3420737065636966696361744A
:10860000696F6E2E0000000050485220666F726D38
:108610006174203A20303D6D6973632049454545BA
:10862000383032313534206D6F64756C6174696F28
:108630006E732C205048522031627974650A2020D4
:10864000202020202020202020202020202020202A
:10865000202020202020202020202020202020201A
:1086600020202020202020313D53554E2046534BC2
:108670002C20504852203262797465730A202020E1
:1086800020202020202020202020202020202020EA
:1086900020202020202020202020202020202020DA
:1086A000202020202020323D53554E204F46444D5F
:1086B0002C20504852203462797465730A2020209F
:1086C00020202020202020202020202020202020AA
:1086D000202020202020202020202020202020209A
:1086E000202020202020333D53554E204F51505301
:1086F0004B2C20504852203462797465731F466FAA
:10870000722053554E5F4F46444D203A207261749B
:10871000650A20202020202020202020202020202A
:108720002020202020202020202020202020202049
:1087300020466F722053554E5F4F5150534B3A2095
:10874000737072656164696E674D6F64650A20209D
:108750002020202020202020202020202020202019
:1087600020202020202020202020202020466F7242
:108770002053554E5F46534B20203A206663735476
:10878000747970650A2020202020202020202020BD
:1087900020202020202020202020202020202020D9
:1087A00020202020466F72204C45475F4F51505388
:1087B0004B3A206E6F6E650A20202020202020205A
:1087C0002020202020202020202020205B75696E82
:1087D00074386F70745D20466F722053554E5F4F32
:1087E00046444D203A20736372616D626C65720A73
:1087F0002020202020202020202020202020202079
:108800002020202020202020202020202020204642
:108810006F722053554E5F4F5150534B3A20726147
:1088200074654D6F64650A202020202020202020C0
:108830002020202020202020202020202020202038
:10884000202020202020466F722053554E5F465333
:108850004B20203A2077686974656E696E670A203C
:108860002020202020202020202020202020202008
:108870002020202020202020202020202020466F83
:1088800072204C45475F4F5150534B3A206E6F6EEC
:10889000651F00005472616E736D69742061204D14
:1088A0006F646520537769746368207061636B65DA
:1088B00074207468656E207472616E736D697420C3
:1088C0007061636B657473206F6E20746865206ED1
:1088D00065772050485920776974682063757272F3
:1088E000656E740A202020202020202020202020B7
:1088F00020202020202020205458206F7074696F81
:108900006E7320446570656E64696E67206F6E20BB
:108910006D6F64655377697463684C69666520633D
:108920006F6E66696775726174696F6E2C2061661F
:1089300074657220616C6C20697465726174696F12
:108940006E73206172650A202020202020202020C4
:108950002020202020202020202020646F6E652CE5
:108960002069742065697468657220737461797315
:10897000206F6E20746865206E65772050485920FE
:108980006F722072657475726E7320746F207468D4
:10899000652062617365205048592E006E6577200E
:1089A0005068794D6F646549642C20692E652E20CE
:1089B0004944206F6620746865205048594D6F64A3
:1089C00065207765206172652073776974636869D3
:1089D0006E6720746F1F6E756D626572206F662002
:1089E0007061636B657473207472616E736D69740A
:1089F000746564206F6E20746865206E6577205002
:108A000048591F6E756D626572206F662074696DBE
:108A10006573207468652073657175656E63652084
:108A20002D6D6F646520737769746368207061636E
:108A30006B657420666F6C6C6F776564206279205B
:108A400064617461207061636B6574732D20697358
:108A50000A2020202020202020202020202020202C
:108A6000202020202072657065617465642C20646C
:108A7000656661756C7420697320312069662061B8
:108A80007267756D656E7420697320616273656EBF
:108A9000740A202020202020202020202020202098
:108AA0002020202020205B75696E7433326F707433
:108AB0005D2064656C61794D696C6C697365636F89
:108AC0006E6473206265666F726520737769746384
:108AD00068696E67206261636B20746F20626173E6
:108AE000652050485920616674657220616C6C2065
:108AF0007061636B6574732068617665206265657B
:108B00006E0A20202020202020202020202020202D
:108B10002020202020207472616E736D697474654A
:108B200064206F6E20746865206E65772050485908
:108B30002C2064656661756C74206973203020692F
:108B40006620617267756D656E742069732061625D
:108B500073656E742E204D756C746974696D6572E1
:108B60002069730A2020202020202020202020207F
:108B700020202020202020207573656420666F72DD
:108B80002064656C61792067726561746572207418
:108B900068616E20302E1F0052657475726E2074ED
:108BA0006F207468652062617365205048592061A8
:108BB0006674657220616C6C206461746120706100
:108BC000636B657473207472616E736D697373691E
:108BD0006F6E20666F72205458206F722061667429
:108BE00065720A2020202020202020202020202004
:108BF000202020202020204D4F44455F53574954CA
:108C000043485F5354415254206576656E74206129
:108C10006E64206D756C746974696D657220657819
:108C20007069726174696F6E206166746572206626
:108C3000697273742064617461207061636B657420
:108C40000A2020202020202020202020202020203A
:108C50002020202020726563657074696F6E206F1C
:108C60006E206E65772070687920666F722052588A
:108C70002E000000303D73746179206F6E206E65A8
:108C8000772050485920286E6F726D616C205769AB
:108C90002D53554E2046414E206265686176696FBE
:108CA00075722920313D72657475726E20746F2063
:108CB000626173652050485920287370656369614B
:108CC0006C2074657374206D6F6465291F0000004B
:108CD000436F6E74726F6C20424C45206D6F6465FB
:108CE0002E000000476574207468652063757272F9
:108CF000656E7420424C45206D6F64652E00000047
:108D0000436F6E666967757265206368616E6E6534
:108D10006C20706172616D65746572732072656C30
:108D20006174656420746F20424C452E0000000081
:108D30006C6F676963616C4368616E6E656C1F611F
:108D400063636573734164647220637263496E691F
:108D5000742064697361626C6557686974656E1F1D
:108D600000000000436F6E66696775726520424CB3
:108D70004520506879537769746368546F5278203E
:108D8000706172616D65746572732E20525820692E
:108D9000730A202020202020202020202020202096
:108DA000202020202020656E74657265642074691F
:108DB0006D6544656C7461557320616674657220DD
:108DC00073796E6320776F7264206F6620726563BB
:108DD0006569766564207061636B65742E000000C0
:108DE000303D44697361626C6520313D456E61625E
:108DF0006C651F7068792074696D6544656C746179
:108E000020706879736963616C4368616E6E656C2C
:108E10000A20202020202020202020202020202068
:108E200020202020205B75696E7433326F70745D72
:108E3000206C6F676963616C4368616E6E656C205E
:108E40006163636573734164647220637263496E26
:108E500069740A202020202020202020202020208B
:108E6000202020202020205B75696E7433326F70C3
:108E7000745D2064697361626C6557686974656EBE
:108E80000A202020202020202020202020202020F8
:108E900020202020205B75696E7433326F70745D02
:108EA00020657874726144656C617955731F0000A8
:108EB000436F6E66696775726520666F7220424CFB
:108EC00045206164766572746973696E672E00006F
:108ED0006164764368616E6E656C3A2033372D337A
:108EE000391F000053776974636820746F207468B9
:108EF0006520314D62707320424C45205048592EF8
:108F000000000000303D4C656761637920313D56BB
:108F1000697465726269205B636869702064656664
:108F200061756C745D1F0000537769746368207409
:108F30006F2074686520324D62707320424C45206A
:108F40005048592E000000005377697463682074FC
:108F50006F206120424C4520636F64656420504857
:108F6000592E00005241494C5F424C455F436F64AB
:108F7000696E675F742076616C75651F0000000084
:108F800053776974636820746F206120424C4520D8
:108F900073696D756C7363616E205048592E0000C3
:108FA00053686F772F436F6E74726F6C205A2D5712
:108FB000617665206D6F64652E000000303D446968
:108FC0007361626C6520313D456E61626C650A209B
:108FD0002020202020202020202020202020202091
:108FE0002020205B75696E74386F70745D206F701F
:108FF00074696F6E734269746D61736B1F0000005A
:10900000476574207468652063757272656E74209C
:109010005A2D57617665206D6F64652E0000000043
:1090200053657420746865205A2D576176652072E7
:109030006567696F6E2E0000726567696F6E3A2012
:10904000736565206C6973745A57617665526567FC
:10905000696F6E731F000000476574207468652097
:1090600063757272656E74205A2D57617665207231
:109070006567696F6E2E00004C697374207375709C
:10908000706F72746564205A2D5761766520726521
:1090900067696F6E732E00004765742074686520E1
:1090A0006261756472617465206F66207468652002
:1090B00063757272656E74205A2D576176652063F0
:1090C00068616E6E656C2E0053657473205A2D575F
:1090D000617665204E6F646549642E006E6F64652D
:1090E00049641F0053657473205A2D5761766520BB
:1090F000486F6D65496420616E64206974732068EF
:109100006173682E00000000686F6D6549641F6818
:109110006173681F00000000436F6E6669677572B7
:1091200065205A2D57617665206F7074696F6E7374
:109130002E0000006F7074696F6E734269746D6108
:10914000736B1F0053657420746865207472616EC0
:10915000736D697420706F77657220666F72206C12
:109160006F772D706F7765722041434B696E672E64
:109170000000000047657420746865206C6F7720DC
:10918000706F7765722076616C75657320286465F1
:1091900063692D64426D20616E6420726177292EAF
:1091A0000000000052756E20746865205A2D5761CA
:1091B0007665206265616D20646574656374696FAE
:1091C0006E20616C676F726974686D2E000000001C
:1091D000536574204D464D206D6F646520746F207B
:1091E000656E61626C6564206F7220646973616290
:1091F0006C656400476574207468652063757272DD
:10920000656E74204D464D206D6F6400536574206B
:10921000746865205241494C2074696D65722074F0
:10922000696D656F75742E0074696D656F75743A3C
:1092300020706572206D6F64651F2772656C273D15
:1092400052656C61746976652027616273273D41C0
:1092500062736F6C7574651F0000000043616E637C
:10926000656C20746865205241494C2074696D65B5
:10927000722069662069742069732061637469765D
:10928000652E00005072696E742063757272656E8F
:10929000742074696D657220636F6E66696775729C
:1092A0006174696F6E2E0000436F6E74726F6C2074
:1092B000746865206D756C746954696D65722041C0
:1092C00050492E0053657420612073706563696690
:1092D00069632074696D65722074696D656F75745A
:1092E0002E00000074696D65723A20302E2E284ED3
:1092F000554D5F4D554C54495F54494D4552532D82
:1093000031291F74696D656F75743A20706572201C
:109310006D6F64651F2772656C273D52656C6174C3
:109320006976652027616273273D4162736F6C75B2
:1093300074651F0043616E63656C20612073706506
:1093400063696669632074696D6572206966206966
:1093500074206973206163746976652E00000000D3
:1093600074696D65723A20302E2E284E554D5F4D32
:10937000554C54495F54494D4552532D31291F00D6
:1093800047657420696E666F726D6174696F6E20D7
:1093900061626F75742061207370656369666963CB
:1093A0002074696D65722E00446F206120626C6FBD
:1093B000636B696E672064656C617920666F7220EB
:1093C00061207370656369666965642074696D65A1
:1093D0002E00000064656C617955731F0000000069
:1093E000436F6E66696775726520616E6420656E95
:1093F00061626C65206175746F2D41434B20667509
:109400006E6374696F6E616C6974792E0000000080
:1094100064656661756C7453746174653A2027697C
:10942000646C65272F277278271F69646C65546FF9
:10943000527855731F7475726E61726F756E6454D5
:10944000696D6555731F61636B54696D656F7574E4
:1094500055733A20746F2041434B27732073796E04
:10946000632D6465746563741F0000004469736153
:10947000626C65206175746F2D41434B2E205573CE
:1094800065206175746F41636B436F6E6669672019
:10949000746F207265656E61626C652E000000005D
:1094A000536574207468652041434B207061796C6A
:1094B0006F616420746F207472616E736D69742EB5
:1094C0000000000053657420686F77206D75636835
:1094D000206461746120746F206C6F616420696E18
:1094E000746F2074686520545841434B20464946A8
:1094F0004F2E00005072696E742074686520637589
:109500007272656E7420545841434B207061796CBF
:109510006F6164206461746120616E64206279749B
:1095200065206C656E6774682E00000047657420C6
:109530007468652063757272656E742073746174EB
:1095400065206F66206175746F2D41434B696E67AE
:109550002E0000005061757365206F722052657394
:10956000756D65206175746F2D41434B696E6700A1
:10957000313D5061757365527820303D5265737589
:109580006D6552781F313D50617573655478203098
:109590003D526573756D6554781F0000436F6E749E
:1095A000726F6C206175746F2D41434B207265732F
:1095B000706F6E736520666F72206A7573742074A5
:1095C0006865206E65787420726563656976652EBE
:1095D00000000000313D63616E63656C41636B2088
:1095E000303D73656E6441636B1F313D7573655427
:1095F0007842756620303D757365547841636B42DF
:1096000075661F005365742061204750494F2070D4
:10961000696E2064617461206F7574206269742EB4
:10962000000000006770696F506F72743A207374A5
:109630006172742066726F6D20273027206F722050
:10964000276127206F72202741271F6770696F509D
:10965000696E1F73746174653A20302F311F0000EA
:109660004765742074686520696E646578206F664C
:10967000207468652063757272656E74206D756CF8
:1096800074692D50485920726164696F20636F6E50
:109690006669672E0A2020202020202020202020FC
:1096A000202020202020202020536565207468651C
:1096B00020656E747269657320696E202A63686123
:1096C0006E6E656C436F6E666967735B5D2E2053CB
:1096D00074617274207769746820696E646578209B
:1096E000302E000041637469766174652061206DDD
:1096F000756C74692D50485920726164696F2063DC
:109700006F6E66696775726174696F6E2E0A2020CC
:109710002020202020202020202020202020202049
:1097200020205365652074686520656E74726965D4
:109730007320696E202A6368616E6E656C436F6E7C
:10974000666967735B5D2E2053746172742077695C
:10975000746820696E64657820302E006D756C74B5
:1097600069506879496E6465781F000053657420FC
:109770007468652076616C7565206F662048465870
:109780004F204354554E452E205468652072616425
:10979000696F206D7573742062652049444C452EB5
:1097A000000000006374756E651F0000476574203B
:1097B0007468652076616C7565206F662048465830
:1097C0004F204354554E45005365742074686520FE
:1097D00076616C7565206F66204846584F2043546B
:1097E000554E452064656C746100000064656C74BE
:1097F000611F0000476574207468652076616C7590
:1098000065206F66204846584F204354554E4520EA
:1098100064656C7461000000536574207468652091
:1098200050414354554E452076616C756520666FF6
:109830007220545820616E642052582E000000009F
:10984000747850614374756E651F7278506143740B
:10985000756E651F00000000436F6E74726F6C20A0
:10986000504120706F7765722063616C696272612C
:1098700074696F6E2E000000436F6E6669677572C3
:109880006520636869702073706563696669632029
:109890006465627567206F75747075742E0A202078
:1098A00020202020202020202020202020202020B8
:1098B000202055736520277365744465627567536E
:1098C00069676E616C2068656C70206D6527206625
:1098D0006F72206D6F72652064657461696C732EA0
:1098E0000000000070696E1F7369676E616C1F7302
:1098F00069676E616C4F7074696F6E731F00000052
:10990000436F6E74726F6C204465627567206D6F73
:10991000646520776869636820616C6C6F77732079
:10992000667265714F766572726964652E0000001B
:109930005365742074686520726164696F20667273
:10994000657175656E63792E2052657175697265F2
:1099500073206465627567206D6F64652E0000007A
:1099600066726571487A3A204F6E6C7920736D612A
:109970006C6C20646576696174696F6E73206672C1
:109980006F6D207468650A20202020202020202070
:1099900020202020202020202020202020202020C7
:1099A000202020202020202020202020637572727B
:1099B000656E7420636F6E66696775726174696F36
:1099C0006E2061726520737570706F727465642E9D
:1099D0001F000000436F6E666967757265206469D9
:1099E00072656374206D6F646500000073796E6347
:1099F00052783A20303D44697361626C6520313D94
:109A0000456E61626C651F73796E6354783A2030DD
:109A10003D44697361626C6520313D456E61626CE5
:109A2000651F646F7574506F72741F646F75745026
:109A3000696E1F64636C6B506F72741F64636C6B30
:109A400050696E1F64696E506F72741F64696E5046
:109A5000696E1F646F75744C6F630A20202020208C
:109A60002020202020202020202020202020205BBB
:109A700075696E74386F70745D2064636C6B4C6FC5
:109A8000630A2020202020202020202020202020A9
:109A90002020202020205B75696E74386F70745D03
:109AA0002064696E4C6F631F00000000436F6E748A
:109AB000726F6C20646972656374206D6F64652ECB
:109AC00000000000436F6E74726F6C205458206960
:109AD0006E20646972656374206D6F64652E00008A
:109AE000537461727420612054582074686174202A
:109AF00077696C6C2062652063616E63656C6C6570
:109B0000642E000064656C617955733A207768654E
:109B10006E20746F2063616E63656C2069741F73BF
:109B2000746F704D6F64653A205B303D5241494C13
:109B30005F49646C655D203E303D5241494C5F5346
:109B4000746F704D6F64655F741F0000436F6E66C5
:109B50006967757265732074686520746865726DD5
:109B60006973746F722070696E2E00005374617295
:109B70007473206120746865726D6973746F7220EC
:109B80006D6561737572656D656E742E0000000001
:109B9000476574732074686520746865726D6973B5
:109BA000746F7220696D706564616E63652E00006C
:109BB000436F6D7075746520746865204846584F12
:109BC0002050504D20646576696174696F6E2E0A6D
:109BD0002020202020202020202020202020202085
:109BE000202020204D7573742062652063616C6CA9
:109BF0006564206166746572206120636F6D706CAE
:109C000065746520746865726D6973746F72206D18
:109C10006561737572656D656E740A202020202061
:109C200020202020202020202020202020202069EB
:109C30006520616674657220676574546865726D2D
:109C40006973746F722E00004765742072616E64D0
:109C50006F6D20646174612066726F6D2074686539
:109C600020726164696F2E006C656E67746842795A
:109C70007465731F5B303D73686F77207468656D22
:109C80005D20313D68696465207468656D1F000062
:109C9000436F6E74726F6C20545820756E646572D9
:109CA000666C6F7773206279206E6F74206C6F61C1
:109CB00064696E6720746865205458204649464F91
:109CC0002E000000313D466F72636520756E64653D
:109CD00072666C6F777320303D44697361626C65A6
:109CE0001F000000436F6E74726F6C205258206F1B
:109CF000766572666C6F77732062792064656C613B
:109D000079696E6720696E20746865206576656E76
:109D1000742068616E646C65722E0000303D446989
:109D20007361626C6520313D456E61626C651F64D4
:109D3000656C617955733A205B305D1F000000004F
:109D4000436F6E74726F6C2063616C6962726174D0
:109D5000696F6E732E00000053657420746865206F
:109D60005458207374617465207472616E736974E1
:109D7000696F6E732E0000007478537563636573AA
:109D8000733A202769646C65272F277278271F7420
:109D9000784572726F723A202769646C65272F27A5
:109DA0007278271F000000005365742074686520D6
:109DB0005258207374617465207472616E73697493
:109DC000696F6E732E00000072785375636365735C
:109DD000733A202769646C65272F277278272F270D
:109DE0007478271F72784572726F723A20276964FF
:109DF0006C65272F277278272F277478271F00007C
:109E000047657420746865205458207374617465C4
:109E1000207472616E736974696F6E732E00000036
:109E200047657420746865205258207374617465A6
:109E3000207472616E736974696F6E732E00000016
:109E4000536574206E657874207472616E736D69E9
:109E5000742773206175746F6D6174696320726516
:109E60007065617420636F756E742E006E756D621F
:109E70006572206F66206175746F2D726570656103
:109E8000746564207472616E736D697473206166A9
:109E9000746572207468652066697273741F6465E6
:109EA0006C6179557320696E7465722D7472616E80
:109EB000736D6974206F7220686F702064656C61C7
:109EC000790A20202020202020202020202020204F
:109ED0002020202020205B75696E7433326F7074EF
:109EE0005D206368616E6E656C2028696620686F0E
:109EF0007070696E67290A202020202020202020F1
:109F000020202020202020202020207265706561E4
:109F1000742064656C6179557320616E6420636898
:109F2000616E6E656C20666F72206164646974692D
:109F30006F6E616C20686F70732E1F006E756D629E
:109F40006572206F66206175746F2D726570656132
:109F5000746564207472616E736D697473206166D8
:109F6000746572207468652066697273741F646515
:109F70006C6179557320696E7465722D7472616EAF
:109F8000736D6974206F7220686F702064656C61F6
:109F9000790A20202020202020202020202020207E
:109FA0002020202020205B75696E7433326F70741E
:109FB0005D20706879207261696C4368616E6E65BE
:109FC0006C206C6F676963616C4368616E6E656C71
:109FD00020616363657373416464726573730A20FF
:109FE0002020202020202020202020202020202071
:109FF000202020286120686F70277320636F6E66B1
:10A0000069672C207265706561742066726F6D20BF
:10A0100064656C6179557320666F72206164646950
:10A0200074696F6E616C20686F7073291F00000087
:10A030005365742064657369726564205458207494
:10A04000696D657374616D7020706F736974696F89
:10A050006E2E00005241494C5F5061636B65745431
:10A06000696D65506F736974696F6E5F741F00006E
:10A070005365742064657369726564205258207456
:10A08000696D657374616D7020706F736974696F49
:10A090006E2E0000536574205241494C2073746148
:10A0A0007465207472616E736974696F6E2074696F
:10A0B0006D696E67732028757365202D3120746F6C
:10A0C000206B6565702073616D65292E00000000AE
:10A0D00069646C65546F527855731F7478546F526D
:10A0E0007855731F69646C65546F547855731F728B
:10A0F00078546F54785573205B305D0A20202020FF
:10A10000202020202020202020202020202020204F
:10A110005B696E7433326F70745D20727853656161
:10A1200072636854696D656F75745573205B305D3B
:10A130000A20202020202020202020202020202035
:10A1400020202020205B696E7433326F70745D2094
:10A150007478546F527853656172636854696D65A1
:10A160006F7574205B305D0A202020202020202085
:10A170002020202020202020202020205B696E74B9
:10A1800033326F70745D207478546F5478205B3074
:10A190005D1F0000466F7263652061205241494C8B
:10A1A00020617373657274207769746820746865C0
:10A1B00020676976656E206572726F7220636F64C6
:10A1C000652E00005241494C5F41737365727445BE
:10A1D00072726F72436F6465735F741F00000000DA
:10A1E000476574207468652063757272656E7420AB
:10A1F0005241494C74657374204170704D6F6465B1
:10A200005F74206D6F64652E000000004765742048
:10A210007468652063757272656E74205241494C92
:10A220005F526164696F53746174655F7420726119
:10A2300064696F2073746174652E000056657269DD
:10A24000667920726164696F206D656D6F72792027
:10A25000636F6E74656E74732E00000064757261B6
:10A2600074696F6E55733A2074696D65206C696D01
:10A2700069741F303D526573756D65206966207085
:10A28000726576696F75736C79206469646E277482
:10A290002066696E69736820313D5265737461721E
:10A2A000741F303D63757272656E742072616469EB
:10A2B0006F20636F6E66696720313D6578746572E3
:10A2C0006E616C20726164696F20636F6E6669678E
:10A2D0001F303D4E6F2063616C6C6261636B203197
:10A2E0003D557365205241494C43625F436F6E6632
:10A2F0006967566572696669636174696F6E1F008C
:10A30000476574207468652063757272656E742089
:10A31000726164696F206368616E6E656C2E000007
:10A320005365742074686520726164696F20636886
:10A33000616E6E656C2E00006368616E6E656C1FE9
:10A3400000000000506572666F726D2061207265BA
:10A35000626F6F74206F662074686520636869702F
:10A360002E000000526573657276656420666F7218
:10A370002053696D706C69636974792053747564D6
:10A38000696F20757365206F6E6C792E0000000078
:10A390001F1F1F1F000000001F1F1F005365742098
:10A3A00074686520524620706174682E00000000B9
:10A3B000303D506174683020313D50617468311F08
:10A3C0000000000053686F772F436F6E66696775F2
:10A3D0007265207072696E74696E67206F662052B4
:10A3E00041494C206576656E7473206173207468F2
:10A3F0006579206F636375722E0000007072696E5C
:10A40000744576656E74733C33313A303E20707219
:10A41000696E744576656E74733C36333A33323EFA
:10A420000A20202020202020202020202020202042
:10A4300020202020205B75696E7433326F70745D4C
:10A44000206D61736B3C33313A303E206D61736B2C
:10A450003C36333A33323E1F0000000044697370CB
:10A460006C6179205241494C206665617475726552
:10A470007320737570706F727465642061742063EB
:10A480006F6D70696C6520616E642072756E7469A1
:10A490006D652E005265616420636F756E742033A4
:10A4A000322D62697420776F7264732073746172E5
:10A4B00074696E6720617420616464726573732EC1
:10A4C00000000000616464726573731F636F756ED2
:10A4D000741F000057726974652033322D626974ED
:10A4E0002076616C756573207374617274696E6730
:10A4F00020617420616464726573732E0000000033
:10A50000616464726573731F76616C756530207663
:10A51000616C756531202E2E2E1F00005468726FFD
:10A5200075676870757420746573742E0000000080
:10A530006E756D626572206F66207061636B657405
:10A54000731F000053657473207468652052535361
:10A5500049206F66667365742E0000006F6666732F
:10A56000657444626D1F00004765747320746865EC
:10A570002052535349206F666673657428732920EF
:10A58000696E2064426D2E005B303D726164696FBC
:10A5900020616E642070726F746F636F6C2D7370C6
:10A5A0006563696669635D20313D726164696F202E
:10A5B0006F6E6C791F0000005365747320746865BA
:10A5C0002052535349206465746563742074687223
:10A5D0006573686F6C642E00525353492064657430
:10A5E000656374207468726573686F6C6420286991
:10A5F0006E2064426D292E20282D31323820646966
:10A600007361626C657320646574656374696F6EF1
:10A61000291F0000476574732074686520525353E6
:10A620004920646574656374207468726573686F2B
:10A630006C6428696E2064426D292E005472616E2C
:10A64000736D69742061207061636B65742061743F
:10A650002061206365727461696E2074696D652E76
:10A660000000000074696D653A20706572206D6F9E
:10A6700064651F5B27616273273D4162736F6C7570
:10A6800074655D202772656C273D52656C61746945
:10A6900076650A2020202020202020202020202035
:10A6A000202020202020205B737472696E676F70F9
:10A6B000745D202761626F7274272052582069668A
:10A6C000205458206F636375727320647572696ECD
:10A6D00067207061636B65742052580A2020202027
:10A6E000202020202020202020202020202020206A
:10A6F000202020202020202020202020202020205A
:10A700006F74686572776973652054582069732087
:10A7100064656C6179656420746F20656E64206F78
:10A72000662052581F0000004765742F536574203F
:10A73000746865206672657175656E6379206F66F1
:10A74000667365742061646A7573746D656E742ECA
:10A75000000000006F6666736574487A1F00000091
:10A76000436F6E74726F6C20686F6C64696E6720E3
:10A770006F66207265636569766564207061636BDE
:10A780006574732E000000005B303D50726F63658E
:10A790007373207061636B65747320696D6D65649C
:10A7A000696174656C795D20313D486F6C6420701F
:10A7B00061636B6574731F0053757370656E6420FD
:10A7C00070726F63657373696E67206F6620434CA8
:10A7D0004920696E70757420666F722061207768F9
:10A7E000696C652E000000007761697454696D65BD
:10A7F00055731F5B2772656C273D52656C617469E8
:10A8000076655D2027616273273D4162736F6C75C9
:10A8100074651F00436C6561722074686520736302
:10A820007269707420656E74657265642076696102
:10A8300020656E7465725363726970742E00000037
:10A840005B303D52414D5D20313D466C6173681F68
:10A85000000000005072696E742074686520736394
:10A860007269707420656E746572656420766961C2
:10A8700020656E7465725363726970742E000000F7
:10A88000456E7465722073637269707420656E74AE
:10A890007279206D6F64652E0A20202020202020F0
:10A8A00020202020202020202020202020436F6EE8
:10A8B000636C75646520656E747279206D6F646574
:10A8C000207769746820746578742027656E6453F6
:10A8D0006372697074272E005B303D52414D5D20DC
:10A8E000313D466C6173682D7363726970742077B3
:10A8F000696C6C2072756E206F6E20626F6F741FB2
:10A900000000000052756E207468652073637269E0
:10A91000707420656E746572656420766961206567
:10A920006E7465725363726970742E00436F6E7437
:10A93000726F6C20726574696D65206F7074696FD9
:10A940006E732E006F7074696F6E4269744D61731F
:10A950006B3A20313D4846584F207C20323D4846D6
:10A9600052434F207C20343D44434443207C2038D4
:10A970003D4C43441F00000020456E61626C652021
:10A980005369676E616C204964656E7469666965B8
:10A990007220322E3447687A203830322E31352EEC
:10A9A00034207369676E616C2064657465637469D3
:10A9B0006F6E000020456E61626C65205369676EA2
:10A9C000616C204964656E74696669657220666FA2
:10A9D0007220424C45207369676E616C2064657417
:10A9E000656374696F6E00004D6F646520303D448F
:10A9F000697361626C6520313D424C45314D627036
:10AA00007320323D424C45324D6270731F0000008E
:10AA10002047657420746865206D6178696D756D77
:10AA20002076616C6964206368616E6E656C436F4B
:10AA30006E66696720696E6465782C20746865208D
:10AA40006D6178696D756D2076616C6964206368ED
:10AA5000616E6E656C436F6E666967456E74727980
:10AA600020696E64657820696E207468652073655E
:10AA70006C6563746564206368616E6E656C436FBA
:10AA80006E66696720616E6420706172616D6574C5
:10AA9000657273206F66207468652073656C6563EA
:10AAA000746564206368616E6E656C436F6E666981
:10AAB00067456E74727900006368616E6E656C4301
:10AAC0006F6E66696720696E6465781F6368616E82
:10AAD0006E656C436F6E666967456E747279206946
:10AAE0006E6465781F0000005F5F5F5F5F5F5F5FA0
:10AAF0005F5F5F5F5F5F5F5F5F5F5F5F5F5F5F5F66
:10AB00005F5F5F5F5F5F5F5F5F0000005F5F5F5F72
:10AB10004170706C69636174696F6E5F436F6E66DC
:10AB2000696775726174696F6E5F5F5F5F000000D7
:10AB30007365744576656E74436F6E666967000071
:10AB40007265736574436F756E746572730000008F
:10AB50007365745065726970686572616C456E6189
:10AB6000626C65007365744E6F74696669636174C5
:10AB7000696F6E73000000006765744C6F674C6509
:10AB800076656C73000000006765745665727369C2
:10AB90006F6E000067657456657273696F6E5665F7
:10ABA00072626F736500000073657450746950724F
:10ABB0006F746F636F6C0000676574507469000098
:10ABC0007365745072696E74696E67456E61626C0C
:10ABD000650000005F5F5F5F5F5F5F5F5F5F5F5F9C
:10ABE0005F5F5F5F5F5F5F5F5F5F5F5F5F5F5F5F75
:10ABF000000000005F5F5F5F526563656976655FB7
:10AC0000616E645F5472616E736D69745F5F5F5FE4
:10AC100000000000727800007278417400000000AB
:10AC200073657452784F7074696F6E730000000022
:10AC3000636F6E66696752784F7074696F6E7300E8
:10AC4000747800007478576974684F7074696F6E17
:10AC500073000000747841667465725278000000D9
:10AC6000636F6E66696754784F7074696F6E7300B6
:10AC700073657454784F7074696F6E7300000000D0
:10AC800073657446697865644C656E677468000026
:10AC9000736574506F7765720000000067657450CB
:10ACA0006F77657200000000736574506F7765728E
:10ACB000436F6E6669670000676574506F776572F1
:10ACC000436F6E6669670000676574506F776572E1
:10ACD0004C696D6974730000656E61626C655061EA
:10ACE0004175746F4D6F646500000000636F6E66A0
:10ACF000696750614175746F4D6F646500000000B5
:10AD000073776565705478506F7765720000000046
:10AD10006F66667365744C716900000067657452F4
:10AD2000737369007377656570506F7765720000A3
:10AD30007374617274417667527373690000000026
:10AD40006765744176675273736900007365745464
:10AD500078546F6E65000000736574547853747294
:10AD600065616D0073746174757300006669666F68
:10AD700053746174757300007365745478486F6C14
:10AD8000644F666600000000736574547844656C17
:10AD900061790000676574547844656C61790000DE
:10ADA00073657454785061796C6F616400000000C1
:10ADB00073657454785061796C6F6164517569651D
:10ADC0007400000073657454784C656E6774680095
:10ADD0007072696E7454785061636B657400000022
:10ADE0007065656B0000000067657454696D6500EF
:10ADF00073657454696D650064617461436F6E6658
:10AE00006967000073657452784669666F000000D8
:10AE100073657454784669666F5468726573686FB9
:10AE20006C64000073657452784669666F5468728A
:10AE30006573686F6C6400006669666F4D6F64656A
:10AE4000546573744F7074696F6E730072784669DD
:10AE5000666F4D616E75616C526561640000000043
:10AE600074784669666F4D616E75616C4C6F616494
:10AE7000000000006669666F52657365740000002B
:10AE800061626F727452785061636B657400000088
:10AE90007072696E74547841636B7300636F6E6691
:10AEA00069675278486F7070696E6700636F6E668D
:10AEB000696752784368616E6E656C486F7070693F
:10AEC0006E670000656E61626C655278486F7070E5
:10AED000696E6700656E61626C6552784368616E89
:10AEE0006E656C486F7070696E670000636F6E66A8
:10AEF00069675278486F7070696E674F707473003D
:10AF0000636F6E6669674368616E6E656C486F70EB
:10AF100070696E674F7074696F6E7300636F6E66F1
:10AF2000696752784D756C7469486F700000000055
:10AF3000636F6E6669674368616E6E656C486F70BB
:10AF400070696E674D756C746900000067657452B6
:10AF500078486F7070696E67527373690000000003
:10AF60006765744368616E6E656C486F7070696E7A
:10AF70006752737369000000737065637472756D56
:10AF8000416E616C797A657200000000636F6E66D5
:10AF900069675278447574794379636C6500000081
:10AFA000656E61626C655278447574794379636C3F
:10AFB0006500000067657444656661756C7452785D
:10AFC000447574794379636C65436F6E6669670095
:10AFD0007365745478416C74507265616D626C6510
:10AFE0004C656E00636F6E66696753796E63576F69
:10AFF0007264730067657453796E63576F7264731C
:10B00000000000007072696E7452784572726F723F
:10B01000730000007072696E745278467265714FE9
:10B0200066667365747300007072696E744461744F
:10B03000615261746573000073746F70496E666964
:10B040006E697465507265616D00000073746F7095
:10B05000496E66696E697465507265616D626C6592
:10B06000547800005F5F5F5F5F5F5F5F5F5F5F5FA0
:10B070005F5F5F5F5F5F5F5F5F5F5F5F5F5F5F5FE0
:10B080005F5F5F5F5F5F5F005F5F5F5F456E657221
:10B0900067795F4D6F6465735F616E645F52465F91
:10B0A00053656E73696E675F5F5F5F00736C6565A4
:10B0B00070000000726673656E736500636F6E6684
:10B0C0006967526653656E736557616B657570008D
:10B0D000636F6E666967526653656E736557616B21
:10B0E0006575705068790000736574526653656EBB
:10B0F000736554785061796C6F6164005F5F5F5F66
:10B100005F5F5F5F5F5F5F5F5F5F5F5F5F5F5F5F4F
:10B110005F5F5F5F5F0000005F5F5F5F416464725D
:10B120006573735F46696C746572696E675F5F5FB4
:10B130005F000000636F6E666967416464726573E7
:10B140007346696C746572007365744164647265FA
:10B15000737346696C746572696E670067657441E4
:10B1600064647265737346696C746572696E6700B6
:10B170007072696E74416464726573736573000004
:10B180007365744164647265737300007365744120
:10B190006464726573734D61736B00007365744111
:10B1A000646472657373456E61626C6500000000D3
:10B1B0005F5F5F5F5F5F5F5F5F5F5F5F5F5F5F5F9F
:10B1C0005F5F5F5F5F5F5F5F5F5F00005F5F5F5F4D
:10B1D0004572726F725F526174655F546573746912
:10B1E0006E675F5F5F5F00007065725278000000FD
:10B1F00070657253746174757300000073657442F6
:10B200006572436F6E666967000000006265725286
:10B2100078000000626572537461747573000000F9
:10B220005F5F5F5F5F5F5F5F5F5F5F5F5F5F5F5F2E
:10B230005F5F5F5F5F5F5F5F5F5F5F5F5F5F0000DC
:10B240005F5F5F5F4C697374656E5F4265666F72C6
:10B25000655F54616C6B5F4C42545F5F5F5F0000E1
:10B260007365744C62744D6F646500006765744C5F
:10B270006274506172616D73000000007365744CFC
:10B280006274506172616D73000000007365743800
:10B2900030323135344363614D6F64650000000026
:10B2A0005F5F5F5F5F5F5F5F5F5F5F5F5F5F5F5FAE
:10B2B0005F5F5F5F5F0000005F5F5F5F3830325F3E
:10B2C00031355F345F4D6F64655F5F5F5F00000025
:10B2D000656E61626C6538303231353400000000D3
:10B2E000636F6E66696732703447487A383032313E
:10B2F00035340000636F6E6669673836334D487ABF
:10B300003830323135340000636F6E666967393129
:10B31000354D487A38303231353400007365743831
:10B320003032313534650000736574383032313570
:10B330003467000073657438303231353446704DEF
:10B340006F6465006163636570744672616D6573F7
:10B350000000000073657450726F6D697363756FE0
:10B3600075734D6F6465000073657450616E436F53
:10B370006F7264696E61746F72000000736574505F
:10B38000616E49643830323135340000736574536E
:10B39000686F727441646472383032313534000041
:10B3A0007365744C6F6E6741646472383032313546
:10B3B000340000007365744164647265737365736F
:10B3C0003830323135340000736574446174615231
:10B3D00065714C6174656E63790000007365743843
:10B3E00030323135345048520000000074726967C1
:10B3F0004D6F64655377697463685478000000008A
:10B400006D6F64655377697463684C6966650000A5
:10B410005F5F5F5F5F5F5F5F5F5F5F5F5F5F5F5F3C
:10B42000000000005F5F5F5F424C455F4D6F6465E9
:10B430005F5F5F5F00000000736574426C654D6F75
:10B4400064650000676574426C654D6F646500005B
:10B45000736574426C654368616E6E656C506172B1
:10B46000616D7300736574426C65506879537769D8
:10B47000746368546F527800736574426C654164FC
:10B48000766572746973696E670000007365744253
:10B490006C65314D62707300736574426C65324D3A
:10B4A00062707300736574426C65436F64696E67A4
:10B4B00000000000736574426C6553696D756C73B0
:10B4C00063616E005F5F5F5F5F5F5F5F5F5F5F5FD6
:10B4D0005F5F5F5F5F5F5F005F5F5F5F5A5F5761E6
:10B4E00076655F4D6F64655F5F5F5F007365745A7B
:10B4F000576176654D6F6465000000006765745A9A
:10B50000576176654D6F6465000000007365745A7D
:10B5100057617665526567696F6E00006765745A9A
:10B5200057617665526567696F6E00006C69737468
:10B530005A57617665526567696F6E730000000047
:10B540006765745A576176654261756452617465C6
:10B55000000000007365745A576176654E6F64652C
:10B56000496400007365745A57617665486F6D656C
:10B57000496400007365745A576176654F70746949
:10B580006F6E73007365745A576176654C6F7750B0
:10B590006F776572000000006765745A57617665C1
:10B5A0004C6F77506F776572000000007A77617694
:10B5B00065526563656976654265616D00000000EE
:10B5C0007365744D666D4D6F646500006765744DFD
:10B5D000666D4D6F646500005F5F5F5F5F5F5F5F1B
:10B5E0005F5F5F5F5F5F5F5F5F5F00005F5F5F5F29
:10B5F0005241494C5F54696D65725F5F5F5F000047
:10B6000073657454696D65720000000074696D653E
:10B610007243616E63656C007072696E7454696D1B
:10B620006572537461747300656E61626C654D750B
:10B630006C746954696D6572000000007365744D27
:10B64000756C746954696D65720000006D756C7479
:10B650006954696D657243616E63656C000000003A
:10B660006765744D756C746954696D657253746166
:10B67000747300007072696E744D756C74695469EE
:10B680006D657253746174730000000064656C61D1
:10B69000795573005F5F5F5F5F5F5F5F5F5F5F5FF5
:10B6A0005F5F5F5F5F5F5F5F000000005F5F5F5F26
:10B6B0004175746F5F41434B5F696E675F5F5F5FAA
:10B6C000000000006175746F41636B436F6E6669C3
:10B6D000670000006175746F41636B446973616258
:10B6E0006C65000073657441636B5061796C6F61C8
:10B6F0006400000073657441636B4C656E67746829
:10B70000000000007072696E7441636B5061636B7E
:10B71000657400006765744175746F41636B000068
:10B720006175746F41636B50617573650000000053
:10B73000736574547841636B4F7074696F6E7300F6
:10B740005F5F5F5F5F5F5F5F5F5F5F5F5F5F5F5F09
:10B750005F5F5F5F5F5F00005F5F5F5F4750494F04
:10B760005F46756E6374696F6E735F5F5F5F000045
:10B770007365744770696F4F757450696E0000008F
:10B780005F5F5F5F5F5F5F5F5F5F5F5F5F5F5F5FC9
:10B790005F5F5F5F5F5F5F5F5F5F5F005F5F5F5F18
:10B7A000446961676E6F737469635F616E645F544F
:10B7B0006573745F5F5F5F00676574436F6E666992
:10B7C00067496E6465780000736574436F6E6669DF
:10B7D00067496E64657800007365744374756E65BF
:10B7E000000000006765744374756E65000000001A
:10B7F0007365744374756E6544656C746100000014
:10B800006765744374756E6544656C74610000000F
:10B8100073657450614374756E650000656E616296
:10B820006C65506143616C00736574446562756753
:10B830005369676E616C0000736574446562756777
:10B840004D6F646500000000667265714F76657229
:10B850007269646500000000636F6E666967446921
:10B86000726563744D6F6465000000006469726501
:10B8700063744D6F64650000646972656374547825
:10B8800000000000747843616E63656C0000000086
:10B89000636F6E6669674846584F546865726D6994
:10B8A00073746F7200000000737461727454686581
:10B8B000726D6973746F7200737461727454686529
:10B8C000726D6973746F724D6561737572656D65C4
:10B8D0006E740000676574546865726D6973746F87
:10B8E00072000000676574546865726D6973746FE7
:10B8F00072496D706564616E6365000067657448C8
:10B9000046584F50504D4572726F720067657452C1
:10B91000616E646F6D0000007365745478556E64D9
:10B920006572666C6F77000073657452784F766548
:10B9300072666C6F7700000073657443616C6962B6
:10B94000726174696F6E73007365745478547261B8
:10B950006E736974696F6E730000000073657452D2
:10B96000785472616E736974696F6E7300000000C1
:10B9700067657454785472616E736974696F6E731D
:10B980000000000067657452785472616E736974C8
:10B99000696F6E73000000007365744E65787454AF
:10B9A00078526570656174007365744E6578744291
:10B9B0006C655478526570656174000073657454E9
:10B9C0007854696D65506F730000000073657452A0
:10B9D0007854696D65506F7300000000736574548E
:10B9E000696D696E67730000666F7263654173739A
:10B9F000657274006765744170704D6F6465000016
:10BA0000676574526164696F537461746500000006
:10BA1000766572696679526164696F00676574431F
:10BA200068616E6E656C00007365744368616E6E6C
:10BA3000656C00007265736574000000777269744C
:10BA400065526D725374727563747572650000008F
:10BA5000757064617465436F6E66696750747200D7
:10BA6000757064617465436F6E6669677572617441
:10BA7000696F6E506F696E74657200007265636FF6
:10BA80006E6669677572654D6F64656D00000000D4
:10BA90007365745266506174680000007072696E5C
:10BAA000744576656E7473007072696E744368696C
:10BAB0007046656174757265730000006765746D2A
:10BAC000656D77007365746D656D77007468726F6E
:10BAD0007567687075740000736574527373694F8D
:10BAE0006666736574000000676574527373694F0E
:10BAF00066667365740000007365745273736944FD
:10BB000065746563745468726573686F6C64000073
:10BB100067657452737369446574656374546872BD
:10BB20006573686F6C6400007478417400000000F5
:10BB3000736574467265714F6666736574000000C4
:10BB4000686F6C64527800007761697400000000CF
:10BB5000636C656172536372697074007072696EB0
:10BB60007453637269707400656E746572536372A6
:10BB70006970740072756E536372697074000000AE
:10BB8000736574526574696D654F7074696F6E008A
:10BB9000656E61626C653830323135345369676E79
:10BBA000616C4964656E74696669657200000000C5
:10BBB000656E61626C65426C655369676E616C4964
:10BBC00064656E7469666965720000006765744338
:10BBD00068616E6E656C436F6E666967456E747200
:10BBE00079000000298E0100AF1E0100AF1E010088
:10BBF000FF000000298E0100AF1E0100AF1E0100F2
:10BC0000FF00000045F20200B85F0000D05F0000B6
:10BC1000020212FF658401003C600000AF1E0100BB
:10BC2000FF00000035D802005C600000806000006A
:10BC300000FF00008DD8020098600000D86000006E
:10BC400000FF0000F9D70200F0600000AF1E010005
:10BC5000FF000000E37F010028610000AF1E01002B
:10BC6000FF000000F17F010044610000AF1E0100F1
:10BC7000FF0000005D80010068610000906100002D
:10BC800000FF0000FF7F0100C8610000AF1E01003F
:10BC9000FF0000002DE20200E0610000D86000001B
:10BCA00000FF0000298E0100AF1E0100AF1E010041
:10BCB000FF000000298E0100AF1E0100AF1E010031
:10BCC000FF00000035A3010010620000D8600000F2
:10BCD00000FF000059A40100286200004862000033
:10BCE0000206020610FF0000CDA50100E062000080
:10BCF0001463000012FF00009F9F010044630000D6
:10BD00007063000002FF0000B99F0100A4630000FF
:10BD10007063000002FF000029A10100D46300004D
:10BD20000864000002FF0000EF9F01001C64000097
:10BD30005064000012FF000069710200806400007E
:10BD4000AC64000001FF00000DEC0200C8640000BC
:10BD5000F86400000516FF00E1EB020040650000FA
:10BD6000AF1E0100FF00000015EB0200646500003B
:10BD700084650000000101FF0FEA0200A4650000D5
:10BD8000AF1E0100FF0000005DEA0200C865000070
:10BD9000F865000010FF0000D9F4020004660000FE
:10BDA0004066000000FF000055F3020054660000EA
:10BDB0008C6600000015FF00B3EC0200C4660000B2
:10BDC000AF1E0100FF0000008B8001000067000033
:10BDD0003867000005FF0000CD8001009C6700006F
:10BDE000D867000012FF0000898301000C68000082
:10BDF00048680000050502FF7B81010078680000AB
:10BE0000946800000211FF00FB810100D06800006F
:10BE1000AF1E0100FF000000BFA60100F068000097
:10BE20000C6900000212FF003FA7010068690000D2
:10BE3000886900000212FF00E97D0100FC69000032
:10BE4000AF1E0100FF000000DD7E0100206A00003F
:10BE5000AF1E0100FF0000008DA101004C6A000030
:10BE60004066000002FF00006DA10100806A000032
:10BE7000AC6A000002FF000055A10100C06A00008A
:10BE8000AF1E0100FF000000696F0200F86A0000A9
:10BE90002C6B00000110FF00836F0200446B000058
:10BEA0002C6B00000110FF002B7002006C6B000077
:10BEB000FC6B000001FF0000CD6E02000C6C000066
:10BEC000AF1E0100FF00000049770200406C000037
:10BED0006C6C00000111FF0085840100886C00007B
:10BEE000AF1E0100FF0000009D840100B46C000043
:10BEF000D06C000002FF0000C5710200D86C000089
:10BF0000006D0000060610FF2D730200A86D0000F2
:10BF1000C86D000001FF0000C9F10200F06D0000D3
:10BF2000186E000001FF000011F20200486E0000D0
:10BF3000706E000001FF0000D5730200A06E0000CB
:10BF4000CC6E00000000FF0051740200086F00007A
:10BF5000446F0000000110FFEB760200A86F0000A4
:10BF6000AF1E0100FF00000083760200D86F0000C2
:10BF7000007000000000FF00297702002C70000014
:10BF80006470000002FF000021E1020074700000F4
:10BF90008060000000FF0000E1ED010098700000EB
:10BFA000C470000012FF0000C3F0010080710000A7
:10BFB000B47100000010FF0049EF0100EC710000B7
:10BFC00024720000000013FFE5EF0100647200001E
:10BFD000A07200000002020202FF00003FF1010017
:10BFE000E87200001473000000FF0000A5F40100D7
:10BFF000207300005C7300000011FF00A7F1010036
:10C000004C7400007874000002050515FF00000064
:10C01000EFF3010010750000407500000010FF00F4
:10C0200099F3010088750000AF1E0100FF000000B9
:10C03000D3A10100B8750000F475000001FF0000F5
:10C04000AFA20100047600003C760000000212FF5F
:10C0500061A2010074760000AF1E0100FF00000025
:10C0600079E10200A47600008060000000FF00007B
:10C07000BFE10200CC7600008060000000FF0000FD
:10C08000E1D80200F8760000AF1E0100FF000000BA
:10C0900011A2010024770000AF1E0100FF00000084
:10C0A000298E0100AF1E0100AF1E0100FF0000003D
:10C0B000298E0100AF1E0100AF1E0100FF0000002D
:10C0C00039A90100507700008C7700000612FF00AC
:10C0D000C9AC010064780000787800000212FF000B
:10C0E000B36C020014790000AF1E0100FF000000D5
:10C0F000BB6F0200507900008C7900000002FF0045
:10C10000298E0100AF1E0100AF1E0100FF000000DC
:10C11000298E0100AF1E0100AF1E0100FF000000CC
:10C12000C9C80200D8790000F87900000210FF00A9
:10C1300093C90200647A00004066000000FF00001E
:10C14000C1C90200807A0000AF1E0100FF0000009C
:10C1500021CA0200AC7A0000AF1E0100FF000000FF
:10C16000ABCA0200DC7A0000047B0000000010FF74
:10C1700099CA0200447B00006C7B00000010FF00A5
:10C18000ABCB0200807B0000B47B0000000000FF0E
:10C19000298E0100AF1E0100AF1E0100FF0000004C
:10C1A000298E0100AF1E0100AF1E0100FF0000003C
:10C1B000F9E90100E47B00001C7C00000202FF00A2
:10C1C00091EA0100387C0000AF1E0100FF00000072
:10C1D000D1EA01006C7C0000987C000002FF0000A6
:10C1E0006DEB0100C07C00004066000000FF000015
:10C1F000EDEB0100DC7C0000AF1E0100FF00000041
:10C20000298E0100AF1E0100AF1E0100FF000000DB
:10C21000298E0100AF1E0100AF1E0100FF000000CB
:10C2200039E702004C7D0000747D000016FF00001D
:10C23000E7E70200887D0000AF1E0100FF0000005C
:10C2400017E80200A87D0000BC7D0000000000058A
:10C25000010102FF95C70100FC7D0000147E000073
:10C2600000FF0000298E0100AF1E0100AF1E01007B
:10C27000FF000000298E0100AF1E0100AF1E01006B
:10C28000FF000000D9B401005C7E0000807E000049
:10C290000601010410FF000095B60100087F0000B0
:10C2A000607F000010FF000053B701002C800000E9
:10C2B000AF1E0100FF000000D1B701008880000020
:10C2C000AF1E0100FF000000F9BC0100E480000087
:10C2D0000481000002FF000075BD01002081000004
:10C2E0004081000002FF0000FBBD01005C810000F6
:10C2F0008C8100000000FF0047B80100D0810000E1
:10C30000F88100000000000010FF0000ABB9010040
:10C31000908200004066000000FF00000BBA0100A0
:10C32000AC820000D882000000FF00006BBA010060
:10C33000E48200000C8300000110FF00BFBA01007E
:10C3400028830000588300000110FF0013BB010088
:10C3500078830000A48300000000000000000000BB
:10C3600010FF000073BB010010840000388400003F
:10C37000010116FFD5BC010098840000C4840000B0
:10C3800002FF0000C9BE0100D08400000886000042
:10C390000010FF0029C10100948800009C89000062
:10C3A000000012FF49C10100988B0000748C00004E
:10C3B00000FF0000298E0100AF1E0100AF1E01002A
:10C3C000FF000000298E0100AF1E0100AF1E01001A
:10C3D000FF000000C1CF0200D08C000040660000CA
:10C3E00000FF000009D00200E48C0000AF1E010035
:10C3F000FF00000089D10200008D0000308D000098
:10C400000012FF004FD30200648D0000E08D000099
:10C410000012FF0077D20200B08E0000D08E000024
:10C4200000FF000039D00200E48E0000048F0000FD
:10C4300010FF000099D00200288F0000048F000038
:10C4400010FF0000F9D00200488F0000648F000048
:10C4500000FF000049D10200808F0000AF1E0100E4
:10C46000FF000000298E0100AF1E0100AF1E010079
:10C47000FF000000298E0100AF1E0100AF1E010069
:10C48000FF0000005D120300A08F0000BC8F0000C1
:10C4900010FF00004D12030000900000AF1E0100CD
:10C4A000FF0000008D120300209000003890000073
:10C4B00000FF00007D12030058900000AF1E010035
:10C4C000FF0000003D12030078900000AF1E010045
:10C4D000FF000000BD12030098900000AF1E010095
:10C4E000FF0000009D120300C8900000DC900000D7
:10C4F00001FF0000AD120300E4900000089100006D
:10C500000200FF006D12030018910000349100003A
:10C5100010FF0000CD12030044910000F8640000F9
:10C520000516FF00DD12030074910000AF1E01002C
:10C53000FF000000ED120300A4910000AF1E0100F7
:10C54000FF000000E1E80200D0910000406600001A
:10C5500000FF0000D1E80200F4910000AF1E0100CE
:10C56000FF000000298E0100AF1E0100AF1E010078
:10C57000FF000000298E0100AF1E0100AF1E010068
:10C58000FF000000EF0E03000C9200002892000054
:10C590000206FF00590F03005C920000AF1E01006D
:10C5A000FF000000950E030084920000AF1E010002
:10C5B000FF00000021100300A89200004066000068
:10C5C00000FF0000CD100300C4920000E4920000C0
:10C5D000000206FF7911030034930000609300000D
:10C5E00000FF00007F0F03008093000060930000B5
:10C5F00000FF0000FBF20200A8930000D4930000AB
:10C6000002FF0000298E0100AF1E0100AF1E0100D5
:10C61000FF000000298E0100AF1E0100AF1E0100C7
:10C62000FF000000D1CC0200E09300001094000055
:10C6300006010101FF00000059CE02006C940000C9
:10C64000AF1E0100FF000000A5700200A0940000D2
:10C650002C6B00000110FF001F710200C494000049
:10C66000FC6B000001FF000089700200F4940000E0
:10C67000AF1E0100FF00000003CE02002C95000059
:10C68000AF1E0100FF000000A1CE02005495000083
:10C69000709500000000FF00F5CE02009C950000A0
:10C6A000D49500000000FF00298E0100AF1E01009C
:10C6B000AF1E0100FF000000298E0100AF1E010027
:10C6C000AF1E0100FF000000B1E50200049600006B
:10C6D00024960000060000FF298E0100AF1E010015
:10C6E000AF1E0100FF000000298E0100AF1E0100F7
:10C6F000AF1E0100FF000000D96B02006096000031
:10C70000AF1E0100FF000000EB6B0200E49600008A
:10C710005C97000000FF0000EBED02006C9700004A
:10C72000A497000001FF0000C1ED0200AC970000DB
:10C73000AF1E0100FF00000051EE0200C89700008C
:10C74000EC97000001FF000031EE0200F4970000BA
:10C75000AF1E0100FF00000071EE020018980000FB
:10C76000409800000000FF00D5EE0200589800003D
:10C770004066000000FF000045DD020078980000E0
:10C78000E4980000060611FF75D50200009900002C
:10C790004066000002FF0000F1D402003099000062
:10C7A0006099000002FF0000EBA70100D49900008F
:10C7B000EC990000000000000000000010FF0000E5
:10C7C00001A80100AC9A00004066000000FF0000D4
:10C7D0001DA80100C49A00004066000000FF000090
:10C7E0005DD70200E09A0000049B00000510FF00E6
:10C7F000A9D702004C9B0000AF1E0100FF00000003
:10C80000BDD702006C9B0000AF1E0100FF000000BE
:10C81000D1D70200909B0000AF1E0100FF00000076
:10C82000E5D70200B09B0000AF1E0100FF00000032
:10C8300009D90200489C0000689C00000110FF001C
:10C84000A3D60200909C0000C49C000000FF0000E2
:10C85000CBD60200E49C00001C9D00000012FF00EB
:10C860001BD70200409D00004066000000FF000052
:10C870004FEF0200589D0000789D00000606FF0063
:10C88000C9EF0200A89D0000C89D00000606FF0039
:10C89000AFF00200009E0000AF1E0100FF0000008C
:10C8A00061F00200209E0000AF1E0100FF000000AA
:10C8B00009F80100409E00006C9E00000112FF007C
:10C8C00011F90100409E00003C9F00000112FF0092
:10C8D00075AD010030A0000054A0000000FF000072
:10C8E000BDAD010070A0000054A0000000FF0000DA
:10C8F000FDF0020094A00000D0A000000505051581
:10C90000FF00000065DF020094A10000C4A1000048
:10C9100002FF00006DE20200E0A10000AF1E010076
:10C92000FF00000091E202000CA20000AF1E010017
:10C93000FF00000011E302003CA200005CA2000026
:10C9400002000000FF000000F1E8020000A3000068
:10C95000AF1E0100FF00000029E9020020A3000033
:10C9600038A3000001FF0000D3D8020044A3000058
:10C97000AF1E0100FF0000009F16030064A300002B
:10C9800090A3000000010012FF0000005F170300E9
:10C9900064A3000098A30000000100FFD517030066
:10C9A00064A30000AF1E0100FF0000001713030086
:10C9B0009CA30000B0A3000002FF0000B1DF020052
:10C9C000C4A30000FCA3000012FF00006185010069
:10C9D0005CA40000AF1E0100FF000000BBD50200F8
:10C9E00094A40000C4A400000212FF0031D602008B
:10C9F000D4A4000000A500000212FF00DFEC01003B
:10CA00001CA5000030A5000002FF000051820100BB
:10CA100044A500005CA5000005FF00009D82010008
:10CA200068A5000088A5000010FF00003783010002
:10CA3000B8A50000D8A5000003FF00000183010095
:10CA400014A60000AF1E0100FF000000A3A001001B
:10CA50003CA6000064A600000216FF007FE9020069
:10CA600028A7000054A7000015FF000019AE010020
:10CA700060A7000088A7000000FF0000D50B03009E
:10CA8000B8A70000E8A700000216FF00F10C0300A1
:10CA900014A8000040A8000010FF0000630D030070
:10CAA00054A8000040A8000010FF0000730C030011
:10CAB00080A80000D8A8000010FF0000E90D0300C6
:10CAC00004A90000D8A8000010FF000049F50200EA
:10CAD0002CA9000044A9000000FF0000D5C70100F8
:10CAE00078A900004066000000FF000077D4020033
:10CAF000B4A90000E8A9000000FF0000FD6B0200DF
:10CB000010AA0000B8AA00000000FF00E8AA000078
:10CB1000E4BB0000000000000CAB0000F4BB000010
:10CB20000000000030AB000004BC0000000000006A
:10CB300040AB000014BC00000000000050AB00003F
:10CB400024BC00000000000064AB000034BC000006
:10CB50000000000078AB000044BC000000000000B2
:10CB600088AB000054BC00000000000094AB000043
:10CB700064BC000000000000A8AB000074BC000012
:10CB800000000000B8AB000084BC00000000000002
:10CB9000C0AB000094BC000000000000D4AB00005B
:10CBA000A4BC000000000000F4AB0000B4BC000016
:10CBB0000000000014AC0000C4BC00000000000035
:10CBC00062060100C4BC00000100000018AC0000B7
:10CBD000D4BC00000000000020AC0000E8BC000055
:10CBE0000000000030AC0000E8BC000001000000C4
:10CBF00040AC0000F8BC000000000000E61A010094
:10CC0000F8BC00000100000044AC000008BD0000BA
:10CC10000000000054AC000018BD0000000000003F
:10CC200060AC000028BD00000000000070AC0000F7
:10CC300028BD00000100000080AC000038BD0000ED
:10CC40000000000090AC000048BD000000000000A3
:10CC50009CAC000058BD000000000000A8AC000023
:10CC600068BD000000000000B8AC000078BD000006
:10CC700000000000C8AC000088BD000000000000FB
:10CC8000D8AC000098BD000000000000ECAC000033
:10CC9000A8BD00000000000000AD0000B8BD00000D
:10CCA0000000000010AD0000C8BD00000000000042
:10CCB0001CAD0000D8BD00000000000024AD000045
:10CCC000E8BD00000000000030AD0000F8BD00002D
:10CCD0000000000040AD000008BE000000000000A1
:10CCE0004CAD000018BE00000000000058AD000070
:10CCF00028BE00000000000064AD000038BE000047
:10CD0000000000006CAD000048BE00000000000004
:10CD100078AD000058BE00000000000088AD0000A3
:10CD200068BE00000000000094AD000078BE000066
:10CD300000000000A0AD000088BE00000000000060
:10CD4000B0AD000098BE000000000000C4AD0000BF
:10CD5000A8BE000000000000D0AD0000B8BE00007A
:10CD600000000000E0AD0000C8BE000000000000B0
:10CD7000E8AD0000D8BE000000000000F0AD0000EB
:10CD8000E8BE000000000000F8AD0000F8BE0000A2
:10CD90000000000004AE000008BF0000000000001A
:10CDA00010AE000018BF00000000000024AE00001C
:10CDB00028BF00000000000038AE000038BF0000AF
:10CDC000000000004CAE000048BF00000000000062
:10CDD00060AE000058BF00000000000074AE00000C
:10CDE00068BF00000000000080AE000078BF0000B7
:10CDF0000000000090AE000088BF000000000000AE
:10CE00009CAE000098BF000000000000ACAE000027
:10CE100098BF000001000000C4AE0000A8BF0000E1
:10CE200000000000D4AE0000A8BF00000100000018
:10CE3000ECAE0000B8BF00000000000000AF000032
:10CE4000B8BF0000010000001CAF0000C8BF000018
:10CE50000000000030AF0000C8BF0000010000006B
:10CE60004CAF0000DCBF00000000000060AF00001D
:10CE7000DCBF00000100000078AF0000ECBF000044
:10CE8000000000008CAF0000FCBF000000000000AC
:10CE9000A0AF000010C0000000000000B4AF000010
:10CEA00020C0000000000000D0AF000030C0000033
:10CEB00000000000E4AF000040C0000000000000DF
:10CEC000F4AF000050C000000000000004B00000FB
:10CED00060C000000000000014B0000070C000003E
:10CEE0000000000028B0000080C00000000000002A
:10CEF00038B0000090C00000000000004CB00000FE
:10CF000090C000000100000064B00000A0C000005C
:10CF10000000000088B00000B0C000000000000069
:10CF2000ACB00000C0C0000000000000B4B00000C1
:10CF3000D0C0000000000000BCB00000E0C0000055
:10CF400000000000D0B00000E0C0000001000000C0
:10CF5000E8B00000F0C0000000000000FCB00000DD
:10CF600000C100000000000018B1000010C1000066
:10CF70000000000034B1000020C1000000000000EB
:10CF800048B1000030C10000000000005CB10000AA
:10CF900040C100000000000070B1000050C100005E
:10CFA0000000000080B1000060C10000000000002F
:10CFB0008CB1000070C10000000000009CB10000B6
:10CFC00080C1000000000000B0B1000090C100006E
:10CFD00000000000CCB10000A0C100000000000073
:10CFE000E8B10000B0C1000000000000F0B1000096
:10CFF000C0C1000000000000FCB10000D0C1000072
:10D00000000000000CB20000E0C1000000000000C1
:10D0100014B20000F0C100000000000020B20000C7
:10D0200000C200000000000040B2000010C200007A
:10D030000000000060B2000020C2000000000000FC
:10D040006CB2000030C20000000000007CB20000A2
:10D0500040C20000000000008CB2000054C200007A
:10D0600000000000A0B2000064C200000000000048
:10D07000B8B2000074C2000000000000D0B200008E
:10D0800084C2000000000000E0B2000098C200006E
:10D0900000000000F4B20000A8C200000000000080
:10D0A00008B30000B8C20000000000001CB300007C
:10D0B000C8C200000000000028B30000D8C2000071
:10D0C0000000000034B30000E8C2000000000000CF
:10D0D00044B30000F8C200000000000054B3000098
:10D0E0000CC300000000000068B300001CC3000077
:10D0F000000000007CB300002CC300000000000012
:10D100008CB300003CC3000000000000A0B300008E
:10D110004CC3000000000000B4B3000064C3000072
:10D1200000000000C8B3000074C30000000000004D
:10D13000DCB3000084C3000000000000ECB300007A
:10D1400094C300000000000000B40000A4C300006D
:10D150000000000010B40000B4C300000000000094
:10D1600024B40000C4C300000000000038B4000074
:10D17000D4C300000000000044B40000E4C3000079
:10D180000000000050B40000F4C3000000000000E4
:10D1900064B4000004C400000000000078B4000083
:10D1A00014C40000000000008CB4000024C400007F
:10D1B0000000000098B4000034C40000000000002B
:10D1C000A4B4000044C4000000000000B4B4000097
:10D1D00054C4000000000000C4B4000064C4000097
:10D1E00000000000D8B4000074C40000000000007B
:10D1F000ECB4000084C4000000000000FCB4000097
:10D2000094C40000000000000CB50000A4C400009D
:10D21000000000001CB50000B4C4000000000000C5
:10D220002CB50000C4C400000000000040B50000A0
:10D23000D4C400000000000054B50000E4C40000A5
:10D240000000000064B50000F4C40000000000000D
:10D2500074B5000004C500000000000084B50000A3
:10D2600014C500000000000098B5000024C50000AF
:10D2700000000000ACB5000034C500000000000054
:10D28000C0B5000044C5000000000000CCB500009F
:10D2900054C5000000000000D8B5000064C50000BF
:10D2A00000000000ECB5000074C5000000000000A4
:10D2B00000B6000084C50000000000000CB60000AD
:10D2C00094C500000000000018B60000A4C50000CE
:10D2D0000000000028B60000B4C5000000000000F7
:10D2E0003CB60000C4C50000000000004CB60000C1
:10D2F000D4C500000000000060B60000E4C50000D6
:10D300000000000074B60000E4C500000100000049
:10D310008CB60000F4C500000000000094B60000C8
:10D3200004C6000000000000ACB6000014C60000F7
:10D3300000000000C4B6000024C600000000000089
:10D34000D4B6000038C6000000000000E4B60000BB
:10D3500048C6000000000000F4B6000058C60000F7
:10D360000000000004B7000068C6000000000000D4
:10D3700014B7000078C600000000000020B70000CD
:10D3800088C600000000000030B7000098C600000A
:10D390000000000040B70000A8C600000000000028
:10D3A00058B70000B8C600000000000070B70000C9
:10D3B000C8C600000000000080B70000D8C600000A
:10D3C000000000009CB70000E8C60000000000005C
:10D3D000B8B70000F8C6000000000000C8B70000A1
:10D3E00008C7000000000000D8B7000018C7000000
:10D3F00000000000E4B7000028C7000000000000A3
:10D40000F0B7000038C700000000000000B80000BE
:10D4100048C700000000000010B8000058C7000016
:10D42000000000001CB8000068C7000000000000F9
:10D4300028B8000078C700000000000038B80000DD
:10D4400088C700000000000048B8000098C700002E
:10D450000000000058B80000A8C70000000000004D
:10D460006CB80000C0C700000000000078B80000E1
:10D47000D0C700000000000084B80000E0C7000032
:10D480000000000090B80000F0C70000000000009D
:10D49000A8B8000000C8000000000000B8B80000F4
:10D4A00000C8000001000000D4B8000010C800004F
:10D4B00000000000E4B8000010C8000001000000F7
:10D4C000FCB8000020C80000000000000CB90000FB
:10D4D00030C800000000000018B9000040C800007B
:10D4E0000000000028B9000050C800000000000043
:10D4F00038B9000060C800000000000048B9000012
:10D5000070C80000000000005CB9000080C8000086
:10D510000000000070B9000090C80000000000008A
:10D5200084B90000A0C800000000000098B9000005
:10D53000B0C8000000000000A8B90000C0C800008A
:10D5400000000000BCB90000D0C8000000000000CE
:10D55000CCB90000E0C8000000000000DCB9000009
:10D56000F0C8000000000000E8B9000004C9000095
:10D5700000000000F4B9000014C900000000000021
:10D5800000BA000024C900000000000010BA00002A
:10D5900034C90000000000001CBA000048C90000A7
:10D5A0000000000028BA000058C900000000000078
:10D5B00034BA000068C90000000000003CBA000056
:10D5C00078C900000000000050BA00008CC90000BB
:10D5D0000000000060BA00008CC9000001000000DB
:10D5E0007CBA00009CC900000000000090BA000056
:10D5F000ACC90000000000009CBA0000BCC90000DB
:10D6000000000000A8BA0000CCC900000000000023
:10D61000BCBA0000DCC9000000000000C4BA000071
:10D62000ECC9000000000000CCBA0000FCC90000FA
:10D6300000000000D8BA00000CCA00000000000082
:10D64000E8BA00001CCA000000000000F8BA0000A0
:10D650002CCA00000000000010BB00003CCA000003
:10D660000000000028BB00004CCA000000000000C1
:10D6700030BB00005CCA00000000000040BB00009E
:10D680006CCA00000000000048BB00007CCA00001B
:10D690000000000050BB00008CCA00000000000029
:10D6A0005CBB00009CCA00000000000068BB0000DA
:10D6B000ACCA00000000000074BB0000BCCA00003F
:10D6C0000000000080BB0000CCCA00000000000089
:10D6D00090BB0000DCCA000000000000B0BB0000EE
:10D6E000ECCA000000000000CCBB0000FCCA000037
:10D6F000000000000000000000000000000000002A
:10D70000434C4920696E7374616E636520696E7362
:10D7100074300000656E64536372697074000000B9
:10D7200072616D5F73746F726167653E0000000027
:10D73000050000000000000000C20100000500001C
:10D7400000100000000000000000000000800550F4
:10D750002100050006000402010000000B0C00007F
:10D7600060660020200000000100000015B60200E5
:10D7700000000000000000000000000000000000A9
:10D78000880E00200000000080010000D010002062
:10D79000FFFFFFFFFFFFFFFFFFFFFFFF0000000095
:10D7A0000000000000000000000000000000000079
:10D7B00000000000F10B0200730C0200810C02005B
:10D7C000B90C0200CF0C0200699801006D980100AD
:10D7D0007198010075980100799801000398010083
:10D7E000319801003B9801004B98010043980100DB
:10D7F0006FAF0100ABAF0100CDAF0100E3AF01009F
:10D8000009B0010064000100780001008C000100F3
:10D81000A000010068050100540501006805010031
:10D82000540501004870180E4470860D30702412A3
:10D8300002989A153870020E3470260E3070080F58
:10D840002C70080F2870761024708E102070100E27
:10D850001C7036111870B2111470080EB1100860E7
:10D8600001D80A7104B87F78020C7E78641000C673
:10D87000981F00A01DB8707803B018600F3027B350
:10D880000F330111C04806986A0229B0086001D818
:10D89000087109DD047109BB11101660A048086009
:10D8A00004100112FF3221500860D048086000883F
:10D8B0000698C21200C4401F00A000BA03DF107116
:10D8C00009DF0672029824031DB8507800A04413A3
:10D8D000281441158110086002D814711088069828
:10D8E000141700C014C000B806986C19009106986F
:10D8F00080020160B83020D806711EBC637C784D70
:10D900005412F03240DE0472404804DB08720DDD30
:10D910000C72044BEF3014480698BA0400C4E0407F
:10D9200000544412086201322140087C811140D920
:10D930001C72B1123032CF4A013AB1DA107208D8F3
:10D94000067104D80871804C237C4470684C4412E2
:10D95000FF328722047580B8E84C81D8367140D9EF
:10D960000472237C084B0698BA0404BA1CB9767971
:10D9700000C1204001B835797F216121007906B9C5
:10D9800006A901D806710298FE01804C307C0298ED
:10D99000520208D86A7100C1544000B8141110D95D
:10D9A0005E71584C441280BDA26DFF25784C441224
:10D9B000FC22513A2814104C00C20CC101B82412A8
:10D9C0002814086228140862281408622814304CAD
:10D9D000304C00C11C4000B814111814086100C577
:10D9E000284001B85415FF35047110491814B04C83
:10D9F000441208620132067102980401804C08D872
:10DA00000C7107BA24D8047106BA187004D80C71C6
:10DA100001BA40D80E7102BA0A7005BA20D8047251
:10DA200003BA204C4411C04C181408611814911109
:10DA3000383111429111186110D90472EF3200C1CE
:10DA4000084001B8141110311E6111422814A111AF
:10DA50000861181406985219181400C1084001B83A
:10DA600014111861FF31181400C1448001B8141159
:10DA70001814086118143088024806987E03009331
:10DA800008DB047101F800A027B00F3000A0108857
:10DA9000B111186180D90A7100C1884000B808111D
:10DAA000009100A000C4704000B8441000A000C065
:10DAB0008840005004118261041082601050F0729E
:10DAC00000A05415504512710698C40406985A04D3
:10DAD00007B8707802B841781EBA5B7A5C7A5D7AD2
:10DAE00000C220C001B8241206981E1700C5441FAA
:10DAF00000A05415511400C3FF010000313D09641A
:10DB00007F3406988A02015851280475015841282B
:10DB10000E758111086102D90472FF0FCC7007B82D
:10DB2000727800F8EBBD00C0401F00A00411113D49
:10DB300010D91271FF33186300C1781002B8381180
:10DB400007B97479581000A006988002184C0D305F
:10DB50000472044800C11CC101B8141100C3D01ED6
:10DB600000A0911504351A7218131CBB08D8047153
:10DB70006C7B04D804716A7B1DBB2F7C5B7B1670A9
:10DB8000044B18131CBB08D804716F7B04D80471B4
:10DB90006D7B217C0C3002600698460406982E0BA3
:10DBA00000B8B111186140D906720298200401BC76
:10DBB00000C2084001B800DC0A7124150265604A01
:10DBC0000A702C4A241508654C4A043508D904719A
:10DBD000202400C1381F00A0141200DC327120D8AC
:10DBE000067101B80C70F0DA0C720CDB087102B827
:10DBF00006984E04482400C3384101B834138F7B83
:10DC00000E7102B9911308DB047203B9067004495E
:10DC1000141100C3884000B8FFB8012011410871F9
:10DC2000014118130824014200C1284000B8141112
:10DC300001411C655141911520351E655141181354
:10DC40002813481300C3844000B8341003D8167159
:10DC5000073005DC1071B1108F780A7200C384C4DC
:10DC60000350217B1DB8507800B800C1381F00A0B8
:10DC700014121C602150F0300152281100A04024E1
:10DC8000076400C0FFFF0100013C17B002200158EB
:10DC90004028067518AC01EC00A0208800C020C008
:10DCA00001B8041217B4211304123052F871196428
:10DCB000402400C3701F00A03410141106986E0D8C
:10DCC0001961009211592129067600BB1159069855
:10DCD0004E0D8762313B0472215A412A00A000C2D6
:10DCE000704000B8317A00A0308801B9116100C3DA
:10DCF0000000C0FF3110312800BC002D0C751154FC
:10DD000018AC01EC312DF470196451134155312CCC
:10DD1000009300A000C3C00FFEFF50B2313A014291
:10DD200050AA00A006980A07FFB0867808715CB870
:10DD30006B786E7800C2548001B800C0D81F00A074
:10DD400004100812B822217A237A52B8417801B817
:10DD50000C6021A809B819604CA800C0FFD1C1FF10
:10DD60004FB2013A00C0002E300001424FAA24B841
:10DD70006E78ACB9FFB004D804714CB923A90698E9
:10DD80006A0500C0139001000698F00400A000C0CE
:10DD9000541F00A017B118100698C40400C01890B2
:10DDA00001000698F00449BC21B952B849B207DE17
:10DDB0002A7105DE0871627C607C1D0C61796778D0
:10DDC00064786B786278657863786078617C010C40
:10DDD000010C6878020C69786C78020C00C22C8007
:10DDE00001B8277A287A267A6A78050C41790A0CD4
:10DDF000B11040D8067102987C06784A2B7A327AA4
:10DE0000584A247A00C400011100404A00C010841E
:10DE100000000812508800C584100100FBAD10BD41
:10DE200001BB8A6B21B9FAA9C44A1812217A227A55
:10DE300000C0341F00A00410FCA8826441103030E0
:10DE40000129F9A9F8ADFBB08260FBA80330A065F9
:10DE50002110044820EC237A0410037A184A241174
:10DE6000DC4A01580029241004753150F8B11150D2
:10DE700081632A71514031400812FCB18461FCA9D0
:10DE80000F310E7117B0112817B111591028FA76F9
:10DE9000C44AF9B11812217A227AA07000950812AA
:10DEA00000C20C8001B8207A844A00B80812020C23
:10DEB000A44A087A020C21B84178784A0B7A127A7F
:10DEC00000C2C81F00A0FFB008D80472184A24106E
:10DED00000DC0A7140A80422241041A806988A0296
:10DEE00000C2441F00A02410015100C4FF01000023
:10DEF00041391150081200A006980A0700BC00C260
:10DF00000C8001B8217A52B84978020C4878020C8A
:10DF100049B8417852AC21AC204A087A067A077A8F
:10DF200049AC00C05C1F00A017B1181000A059B880
:10DF300040785AB101D9FC72427857B8407858B14C
:10DF400001D9FC72427800A000C20C8001B8217A8D
:10DF5000227A21B8547852B8BC4A241199791271A6
:10DF600007B915614CA9617800BB03BC0C6414703F
:10DF700009B919614CA9417801BB126300C4002E94
:10DF8000300000C0FFD1C1FF4FB1013941414FA95D
:10DF9000E44AC8B8081224AB4CB823A806986A050E
:10DFA00000C0681F00A017B1181000C00490010045
:10DFB0000698F00400C08009004040A809B8FFB1ED
:10DFC00008D9047103B853A8B11004D80C7156BB1A
:10DFD000607B57BA627A607A02D80C7156BB607B5C
:10DFE00059BA627A607A04B86E783DB8607800C039
:10DFF0005638000000C1B08001B814119979087238
:10E0000000C0D604000000C124C000B814119F79DC
:10E01000047208484CA82EB8FFB108D906714AA866
:10E0200004704BA80FB834A800C00C5E000046B2C4
:10E03000014246AA00C12C4001B814110861063102
:10E04000087100B90698F60F0698C812B11101D9E7
:10E050000E710698781902D906720698000C069877
:10E06000C212511406985A0400C0641F00A017B1D0
:10E0700018100298D00F00B84CA84AA84BA800C0AE
:10E08000F321FFFF46B1013946A904B86F7800A01B
:10E0900000C0581F00A017B11810FABC1964415CE9
:10E0A000512C00C06C1F00A00410012C06750698AE
:10E0B0005A0406983A0EB110186007D8347140BA65
:10E0C000069898121DBC7F7C04B86578911004D81E
:10E0D00016711CB86E7800C0684000B821780698A8
:10E0E0001E1001400872427C0698D4120298C80A99
:10E0F0001DB8717804B86C7841B842786378447878
:10E10000FFB104D9067202987E0900C00490010094
:10E110000698F00400C32C1F00A000C274C000B811
:10E120002414481300BC48121C4B1C4A24144813E6
:10E1300000BC48124ABA447A427A4BBA447A427ACC
:10E14000617A4CBA647A657A3DBA607A4DB942B860
:10E150003FBB5B7966796179020C6479050C637960
:10E160006079050C627965795A7900C2340102B888
:10E17000241305B819603140081242B86A78020CBD
:10E180004A78020C40BCFFB208DA06714ABA06703F
:10E190004BBA627A657A677A667A6A79667B0298A0
:10E1A000460A00C32C1F00A000C274C000B824148B
:10E1B00048131C4B1C4A241448133FBC48121C4AE9
:10E1C00000BC48124ABA647A627A4BBA647A627ABC
:10E1D000617A4CBA647A657A3DBA607A01D94E7137
:10E1E000647800C1708001B800C080000800081188
:10E1F0000698F00A42B861784DB97F797E796A78DD
:10E2000068786278020C7B790F0C7A79140C747937
:10E21000417860787579050CFFB208DA06714AB862
:10E2200004704BB8657801BC1664407002D93C712B
:10E230000698F00A42B84DB96878407841787F79FD
:10E240007E797B790F0C7A79140CFFB208DA0871A9
:10E2500071794ABA067070794BBA7279657A6A78C0
:10E26000020C4A78050C01BC1664020C4179407915
:10E270000C0C00C04C0102B848100698BA045114A6
:10E2800000C06C1F00A00410012C17B0011187689A
:10E29000015841280E7605218769415C412D112DD9
:10E2A000067006985A0400C0681F00A017B1181025
:10E2B00042B84DBB7C7B6478020C29B86878511455
:10E2C0004044067506985A0442B84478FFB101D913
:10E2D0000C7100C1548001B8CBB8081100C0601F98
:10E2E00000A017B11810911004D8147100C0A81E16
:10E2F00000A0041080D8067107B8537800F807B85A
:10E3000000C1CC1E00A000C220C001B824122811F8
:10E31000767800F8B1109478387106988A02E4B9DA
:10E3200011591128067600B80C70A0B911590129AD
:10E330000475A0B8826000C3C01F00A03413012B75
:10E34000341000C3FFFF00FF42B13139114042A831
:10E3500000A01DB09178FA7142B86478020C00BA3E
:10E3600029AA00C4548001B842B84DB900C3C040C6
:10E3700001B83413977B047240EC020C44785C794A
:10E3800053AA0A0C281442B84DB9FFB301DB267119
:10E39000244C00C3FF0FFF013814547940784178B2
:10E3A0005579020C5B795A79140C5F795E794A7859
:10E3B0004278347002DB1471527951795079020C31
:10E3C0005B795A795F795E791E7004DB1A7100C43B
:10E3D000FF07000000C3342102B848133FBB467B4F
:10E3E000020C5B795A793DBB407B4CBB447B457B3F
:10E3F00000C3301F00A03414403C167100C068C038
:10E4000000B8481028131C4B1C483414481028131B
:10E410004AAA4BAA04B86D781DB851785CB84B78FD
:10E420004E7800A000C074C000B80411108800B974
:10E43000181068480411108801B90B6118102C4895
:10E4400004111088008800C1231C000018104AB86D
:10E4500064784BB86478260C28B000C1FFFF0FF039
:10E46000113871B90B61114028A828B973797479F2
:10E4700000C21010303045AA54790E0C00C0E8409C
:10E4800001B8041100C23030101045AA0E0C04105F
:10E49000008810880698C20C0091009020888F6137
:10E4A0008F600698C20C0090886A21400112906A21
:10E4B000035800C13F3F00001138FFBC022441282F
:10E4C0001138014245AA28B953794AB844784BB863
:10E4D000447800900091181000912C481810009179
:10E4E0006848181000A09168436091694361115B0E
:10E4F000012B112841603128315B00BA30280676A3
:10E500003128204A4163302806763128104A416379
:10E51000302806763128084A4163302806763128AB
:10E52000044A4163302806763128024A4163302884
:10E530000476014A00A0115910D9067108600860DC
:10E5400008D90471086004D90471046002D9047107
:10E55000026001D90471016000A01088041102302A
:10E5600006710861086100C0FFFF000011380091CA
:10E5700000A000BA01D806710148112A1F6101608C
:10E5800001D8F6720138F67200A000C220C001B8AE
:10E59000241211592129127300210E7100C238C0B2
:10E5A00001B824120121212900A002B020D8147141
:10E5B00000C0B41E00A0041002B9457906981C12D0
:10E5C000EA7003B09F78087200B806A800F80698B1
:10E5D0000A0700C5781F00A050880C4D1CBC00C065
:10E5E000B81E00A0811101D91E71407C0095011553
:10E5F000044D50887C4DFFBB1863315B04110698B5
:10E60000660D3129F875069868185415069878191A
:10E6100001D908720698240706700698C2071CBB29
:10E62000547B009500F8069852080E7006982E0B41
:10E6300006985208069818110698D406211900C0A9
:10E640002C4001B80A78097800F810B901BA069888
:10E650008E120698D00F00C5781F00A000F8911206
:10E6600003321CB900C3A81E00A0341300C4B0407C
:10E6700000541DB84278707903DE067144783E700C
:10E680007179A11020D80A71069824070298140FF6
:10E6900080DB1C7102D8187205B80814A110103064
:10E6A0000248081400B808149110086008141DB836
:10E6B0006278A11000DC0676517900BA9111203100
:10E6C0001D61911004D80E7200C14C1F00A01411DE
:10E6D00001D90A7120880698F60F009200C12040E7
:10E6E00000B80533054B1872084C03DE0471904CDA
:10E6F000441400C3FF1F0000413BFF23381194491D
:10E7000000C3384101B83413086380DB0C7103BACD
:10E7100018620698FC0E087018620698FC0E0C49E8
:10E720000879097914102140081100A000BD06984D
:10E73000640210B903DC047100B901BA06988E12A4
:10E7400002D9067100404E7203B118610F3106986C
:10E750001E10FFD82872811008D8187106DD0A71C2
:10E760000698640203DC0C72069862100698D412B4
:10E770000C7006DD107106986810487020B804A867
:10E7800006DD1072069852080698D40601F840B8C3
:10E7900004A800F800C0A81E00A00413086301DB51
:10E7A000227191100111186111381DB910D808712A
:10E7B00044790298140F02DBFA72A11328DBF47279
:10E7C00003BD0698C40F0698520800C57C1F00A020
:10E7D0000698640200BA03DC0472FC4D5415212D26
:10E7E0000698000502986C089110015503355150A8
:10E7F000011900A000C1481F00A0141001D84271E7
:10E8000001480860FE200E75811020D8087100C1F3
:10E810004C1F00A0141101D9287100C02C4001B870
:10E820000412215108610F3118611152281000C0E3
:10E83000084001B8041191122151203111522119BF
:10E8400000A0811380DB067201B800A000C314C0D1
:10E8500001B8341006302E726C4B34121C4B34103D
:10E86000186002302072811080D8DE713410014AA5
:10E8700008620460803021508C480A717F234D2348
:10E880003410013000A000BD0698C40F1CB84778B2
:10E890004578437802B8447800A006985208069854
:10E8A000621000C5841F00A0541506980005029848
:10E8B0006C08B1138F7B0A7200C384C40350017BC0
:10E8C0000698C81200C1384101B814118F790E7131
:10E8D00000C1B84000B800BA0698FC0E50BA0698BD
:10E8E000981206981E10FFD84A71911004D84872E9
:10E8F000811008601CD8407220D938721112FF3282
:10E900002151347180218021111400C0D81E00A033
:10E910000413FFBA3151113A215111531DB9381066
:10E920007B7940440E7200B900C2B01E00A01812DC
:10E93000067004B860780698C21200F800B900C2E8
:10E94000A44000541812644A0AB918121CBA507A2A
:10E95000517A1DB942795F7900A00698640207DCFC
:10E960001072911000200A75069818110298320E44
:10E970000698D40601B9911004D8047100B910BAF0
:10E9800006988E1200BA0040347100C0A81E00A084
:10E990000411086101D9127104D9E2728110086072
:10E9A00001D8DA711DB8647800C11CC101B806989D
:10E9B000760401B81160002A047600BA069818118E
:10E9C00000C5881F00A05415212D0698240700C5F6
:10E9D0008C1F00A000F800BC811108D9167280D9E4
:10E9E000207201B910BA06988E1200400E7101BC57
:10E9F0001070069862100698D41220B804A800F887
:10EA00000698181181110231127100B900C2144028
:10EA100000541812244A02B918120698621000C550
:10EA2000901F00A054150698F01802986C08041165
:10EA3000012114711CBA737A0420041228110420D5
:10EA400004110121F47200A00698BA0401F8911093
:10EA500010D8287100C51CC101B854110698660D64
:10EA600000C5C81E00A054155129EA7507B875786D
:10EA70001DB8447801B804A800F8B110186010D887
:10EA80002E7100C05040005400C3084000B831143B
:10EA9000984C44113411086101D9FA7144122810BC
:10EAA000086228100862281008622810E87002988E
:10EAB0009E0206988002113804721E6202BB00C1D9
:10EAC000D81E00A0141120390C72911210DA0672AF
:10EAD000417B00A00698C81200C2A81E00A0241204
:10EAE00020DA0472617B1CBA527A00A01CBA727AD6
:10EAF000811204DAFC7200A01CB86B7800C0684078
:10EB000000B82F7800A010631EB9637900B902EC39
:10EB100000CD114502EC00CC01DB087100BB02986E
:10EB2000C61603B841110731FA211C76062191124D
:10EB300010DA087102DD10721E7020B80698120DEE
:10EB40003038147208B80698460400C02C4000B84B
:10EB50002978207800F8056020D8067102985614AC
:10EB600002EC00CA05B823DA187104DBDA7120DA86
:10EB7000D67110DAD2721EB8617800B801DA067266
:10EB800002EC00C8911110D9267100C1BC1E00A072
:10EB900014111150FF300C720761A1101150023096
:10EBA0000A7180DB0A720AB89E701DB97C79186000
:10EBB000911111402111C031114001191EB84111AC
:10EBC00008D90471667820D904726578A11002D83A
:10EBD0000672C0DA1E711EB8273123DD087210DB01
:10EBE0001072607825DD0A7121DD087208DB04717E
:10EBF000627803B8411107310872A1152035AA7156
:10EC000002DD2072A11120D9A07102D91672CCDACE
:10EC10009872411140D9927206B8054D5A72029805
:10EC2000F81221114049C0D94C71A031411540352D
:10EC3000026551410461086308DA1E7204DA367213
:10EC40001049A1150235067110DB0E7201340A71EC
:10EC500008DB22711EB86778CC3211101A300ADC3A
:10EC60000872CCDE0471FD3100C00D0F0C0D216067
:10EC700001D85C7207B80298221300BA411108D972
:10EC80000C7102EC00CA05B830DAEC720734F031CE
:10EC9000036101DA0471014900C0F300A3E32160BC
:10ECA00001D8D27100C098144068216040300144FE
:10ECB00040DA0471204C04320262204A11100630FE
:10ECC0001F60014218311D61114202984013204A11
:10ECD00000C00517085021601130014220880DDA6C
:10ECE000527100C1DE1B250180BC04DA107208DA03
:10ECF0000A7200C120841000E024A024FFBB086336
:10ED00004143026401DA06711E49024B00C0201F14
:10ED100000A008633810BC2002DA127101B9115941
:10ED2000A11380DB087100C100FCFF0118100298DC
:10ED3000521600C4A81E00A0441080D87E71009214
:10ED40000462DDDA0871A11180D992721EBD437D83
:10ED5000EFBD06980203DDDA8472A11105D95C715A
:10ED600000C24040005424121024281401D9067215
:10ED700002D9327140D91E7102EC00CA211018323A
:10ED80000471FA2220D804720822FE22087502ECCF
:10ED900000C8F87001D90E7102EC00C802D90672E1
:10EDA00004DC187200C0A81E00A004101D6001D869
:10EDB00006711EB8647807B873780298C616641096
:10EDC00000C6981F00A0C3B806986A0200C4401F7E
:10EDD00000A014BA281400B8011AB1108F780A7272
:10EDE00000C084C40350017891101030011905BA95
:10EDF0000698981202D9067101B804A800C0A81E8E
:10EE000000A0041380DB06710298E2121DBA7C7A1E
:10EE100001DB5E7100C2241F00A024111114FF3415
:10EE200002EC00C8FF24FA7608610698220D0461FE
:10EE300011380F3004611114011141100698220D90
:10EE400001D8087203B8029822130C4A02DB16712B
:10EE50002410112811280698360D00C2204000B851
:10EE6000FF200812411008600698220D01D87C711D
:10EE700020BC1033767100BB00C1201F00A0141508
:10EE8000C021112C511218620F320E71408851149A
:10EE90000698EE1641430094511208651C620F3229
:10EEA0000E71411151140698EE161C644143086519
:10EEB000513B00C1DC1E00A01411111231100F30A3
:10EEC000127100BA056101D80471114201600FD8B6
:10EED000F472311003601E30047201B8003A0872F7
:10EEE00004B80298221302980E1500C0384101B8E8
:10EEF00004118F7914717F20692004110861303169
:10EF000010DD06711DBA637A06980A100698000390
:10EF100000F830885088FF34087102ECFF24F87044
:10EF200002EC00CD1410595001440421FF22F2726A
:10EF30000F4C0095009300A000C1AC1E00A014115E
:10EF400000A03088069828198111086102D906723C
:10EF5000029806181CBB557B086120D906710298DF
:10EF6000F6170088A11018600698141708211415C8
:10EF7000FC251EBB5C7B5D7B00C1084001B8141101
:10EF80000731FE21307608D82A725113FC2334133E
:10EF900004DB20711863FF33315B00C110C000B87F
:10EFA0001411086180490C71FF31302960751EBB56
:10EFB0007B7B1C707B7B7C7B00DD04717D7B01BBDC
:10EFC0003815811318634033067107BB717BEC253C
:10EFD000541300DF5471042505DF547154152111B9
:10EFE00020880698660D009251293E7500C10840A0
:10EFF00001B8141102DB0C710731315B31292A761B
:10F000000C7004DF0872016180D91E720698141713
:10F0100000C010C000B806986C1906981417141197
:10F02000FFD9607202984C180090009300A054150C
:10F03000A111186110D9A672082508D8A071082559
:10F0400010D89A71208821110698660DFC2554125B
:10F05000112AF82554110C2520D80871F0255411D7
:10F060001025202904762159181500920298B81706
:10F0700007B97179811010D80A711CB8447802B8A8
:10F0800041781CB9747904B9677900F88110A0D867
:10F0900008711CB9497900A0086002D8FA71069875
:10F0A000141710880698C812106210DA0871082127
:10F0B0001415F025541100C20020FEFF20291275FE
:10F0C0000698781901D90A72069852080698D4064B
:10F0D00000941CBB41100C2006980A124111082113
:10F0E000141006980A123128441111120861FF31D8
:10F0F000FF320122105210721861181404244413B4
:10F10000042438140C7018612141181408240814C0
:10F110000298C2124044147100C1B01E00A0141520
:10F1200051131C630FDB0C7219650698C40441155A
:10F1300000A00698D4060698C81208BB5114069879
:10F14000B0184415FC255415029800051CB900C3DD
:10F15000A81E00A03413086308DB1A718113A0DB1A
:10F160000671497910706979086302DB087204B985
:10F17000677900F800A08111086102D910711CB9EB
:10F180007579069814171411FF3100A0FFB900A07B
:10F19000041008211411F421081100A0811110613C
:10F1A00010310E710698141708211411F82114114A
:10F1B00000A0000064060000193F010604100100D1
:10F1C0000001000202000000000500010100000033
:10F1D000000000000000000000000000000000002F
:10F1E0000D0000000000000000000000B8F1000069
:10F1F000D4F100000000000058E58500A864B501C6
:10F20000E803000001020000B40B1002000000003F
:10F2100000000000000000000000000000000000EE
:10F22000E703000000000000000000000D000000E7
:10F230000000000000000000B8F10000D4F1000060
:10F240000000000058E58500A864B501E80300004F
:10F2500001020000D30B10020000000000000000BB
:10F26000000000000000000000000000E7030000B4
:10F2700000000000000000000D0000000000000081
:10F2800000000000B8F10000D4F100000000000010
:10F2900058E58500A864B501E803000001020000FC
:10F2A000860B1002000000000000000000000000BB
:10F2B0000000000000000000E70300000000000064
:10F2C000000000000D000000000000000000000031
:10F2D000B8F10000D4F100000000000058E58500FE
:10F2E000A864B501E8030000010200003C0B100215
:10F2F000000000000000000000000000000000000E
:10F3000000000000E7030000000000000000000013
:10F310000C400200000000000040000020400200FD
:10F320000F0000000000000030400400000000005A
:10F330000000000000000000000000004840010044
:10F340000007000050400100000000005C40020087
:10F350000000000000000000A840010000000000C4
:10F36000B4400400FF40000000000000FF41000026
:10F370000000000008C00100000000001CC00110D7
:10F3800000F807001CC001300002002020C005006A
:10F39000001300000A61000000A8A802000000009D
:10F3A0000000000050C00400873181000E3707D6EE
:10F3B00043050608116D030064C00800E53700002E
:10F3C00040201006C8F248181FE8F600BD4B721521
:10F3D00011A3180510325476980A000088C0010065
:10F3E00000000000080001014407000018000101AE
:10F3F000000000002000010101A000001C400801E5
:10F40000100000009101000001C001060050000042
:10F4100000000000000000030000002000000000C9
:10F420005C400501410C0000300144001000000068
:10F430000000000000000000804002010000EC0815
:10F44000000000008C4009010000000000000000E6
:10F4500000000000000000000000000000000000AC
:10F46000000000000000000000000000E040020179
:10F470003300000000000000EC40070193E8A68C78
:10F4800000000000640483078813C83A90200A0033
:10F4900000612000B75635121041020120300429C6
:10F4A00088BB400024410201000000000000000071
:10F4B000304111016406660C0C010000E853FA00AB
:10F4C000000000000000000000000000000000003C
:10F4D000000000000000000001000000000000002B
:10F4E000000000000000000000000000640483072A
:10F4F0008813820000000000304204010000000078
:10F500000000000E00000000000000004442010165
:10F510000000000010800101030000003C80010198
:10F520000100000088800101000000009C800301B0
:10F530000000000070780300D0000000A8800111D6
:10F54000F0010000A88001310542CB01AC8001111F
:10F55000F0010000AC800131053EFD00B0800201E9
:10F5600000030002370000018800020200000004CE
:10F570004C0000009400010200000000D0000202D4
:10F580000E00000090029608E40001023D094204CA
:10F59000F400010200000000180101020000000454
:10F5A000FFFFFFFFFC1F0103E0F1000040400200ED
:10F5B00000000000000000005840010180700600BB
:10F5C00088400101160300000C4101016E46100045
:10F5D00038800101B40B1000FFFFFFFFFC1F010387
:10F5E0002CF200004040020000000000000000007B
:10F5F00058400101546F06008840010116030000C5
:10F600000C4101016A46100038800101D30B100043
:10F61000FFFFFFFFFC1F010378F2000040400200E3
:10F620000000000000000000584001014272060086
:10F6300088400101150300000C4101016E461000D5
:10F6400038800101860B1000FFFFFFFFFC1F010344
:10F65000C4F2000040400200000000000000000072
:10F660005840010130750600884001011503000073
:10F670000C4101016D461000388001013C0B100067
:10F68000FFFFFFFFA4F500008008089240420F0032
:10F69000000000000000FF7FB00F0020000000000D
:10F6A00000000000DCF500008008089240420F00D6
:10F6B000000001000100FF7FB00F002000000000EB
:10F6C0000000000014F600008008089240420F007D
:10F6D000000002000200FF7FB00F002000000000C9
:10F6E000000000004CF600008008089240420F0025
:10F6F000000003000300FF7FB00F002000000000A7
:10F700000000000010F300000000000084F600007C
:10F710000400000000000000193F01060410010071
:10F720000001010600102700000C0000000000008E
:10F730000000000050C300001C250000C4090000A8
:10F7400050C300007C150000DC050000F5DA020063
:10F7500070170000B80B0000E5BF00007017000034
:10F76000B80B00000D000000000040000000000089
:10F7700018F7000034F7000000000000082F860092
:10F780000048E80140420F00010100001149500209
:10F790000000000000000000000000000000000069
:10F7A000000000002A420F000000000000000000DE
:10F7B0000D000000000080000000000018F70000AD
:10F7C00040F7000000000000004786000048E80104
:10F7D00080841E0001010000114950020000000059
:10F7E0000000000000000000000000000000000019
:10F7F00054841E0000000000000000000D00000006
:10F80000000080000000000018F700004CF7000026
:10F8100000000000802596000048E80140420F00EB
:10F820000108000011495002000000000000000023
:10F830000000000000000000000000003D420F003A
:10F8400000000000000000000D000000000080002B
:10F850000000000018F7000058F70000000000004A
:10F86000802596000048E80140420F000102000098
:10F8700011495002000000000000000000000000DC
:10F8800000000000000000003D420F0000000000EA
:10F89000000000000C400200018101000041000056
:10F8A0002040020000000000010000003040030082
:10F8B000000000000000000000000000A84001005F
:10F8C00007000000B8400300FF4C0000FF4D00009F
:10F8D000FF4D000008C00100000000001CC0011026
:10F8E00000F807001CC00130F502080020C0050028
:10F8F00000130000EC80B3034375A8020000000071
:10F900002E02000050C001008741300C58C0020098
:10F9100054060708D1B6020064C008000430000095
:10F9200040201006C8F248181FE8F600BD4B7215BB
:10F9300011A3180510325476980A000088C00100FF
:10F940000000000008000101080700001800010184
:10F95000AAAAAA00200001010060DA001C400101EF
:10F960001000000030400301000000030000000010
:10F97000000000006840020129417671000000008B
:10F98000E040020133000000000000000C410101D2
:10F99000B855120024410101000000005441050146
:10F9A0000100000000000000000000000000000056
:10F9B00000000000384202010000000000000000CA
:10F9C000444201010000000010800101030000001A
:10F9D00038800201114910000100000088800101F7
:10F9E000000000009C800101EB400200B080020199
:10F9F000000300023700000188000202000C00042E
:10FA00004C0000009400010200040000D00002023B
:10FA10000E00000090029608E40001023D09420435
:10FA2000F400010200000000180101026000510210
:10FA3000FFFFFFFFFC1F010364F700003C400400D0
:10FA4000000000000000000000000000A00700000F
:10FA500050400100000000005C4002000000000077
:10FA600000000000B4400100FF4C000054C0010041
:10FA70000E2D09E620400401000000861FC0010091
:10FA800000600000008000005840040118000500DC
:10FA900080080000090000009100040080400C0173
:10FAA0008C000C000000000012002200000000008A
:10FAB000000000000002050E1C2F435362696861BC
:10FAC0005543320416E4B8C68A674533224A920485
:10FAD000EC40070190382CAC000000005A10080AD6
:10FAE000D007CA4A51104800F9541E804737414A8E
:10FAF0001041020130194A0589BB4000284101012B
:10FB0000FFFF000030410901F15004430C010000E7
:10FB1000E853FA000000080010161C22282E343A80
:10FB2000404621436587A90B0000C0B4684103012A
:10FB30005A10080AD0074104C103000030420201F4
:10FB40008993A30F5EC25D0EA0800201707803004E
:10FB5000D0000000A8800111F0010000A880013150
:10FB60000542CB01AC800111F0010000AC800131F5
:10FB7000053EFD00FFFFFFFFFC1F0103B0F7000083
:10FB80003C400400000000000000000000000000F5
:10FB9000A007000050400100000000005C4002008F
:10FBA0000000000000000000B4400100FF4C000015
:10FBB00054C001000A2D09E620400401000000069F
:10FBC0001FC000000060000000D032005840040157
:10FBD0006402FF008008000001000000110008001E
:10FBE00080400C010804000000000000D90322003E
:10FBF00000000000000000000102071121374B5AED
:10FC0000676962544029150500008020434433335E
:10FC10002392A424EC40070190382CAC0000000093
:10FC2000640483078813C83A9D200A00016120807C
:10FC30004737414A104102012A144A0289BBC00ACF
:10FC400028410101FFFF0000304109016406660CF4
:10FC50000C010000E853FA000000080012181E24EE
:10FC60002A30363C424821436587A90B0000E0C496
:10FC7000684103016404830788138200C1080000FF
:10FC80003042020145966B105C22670EA080020193
:10FC900070780300D5C00000A8800111F0010000B9
:10FCA000A88001310542CB01AC800111F0010000B8
:10FCB000AC80013105228D00FFFFFFFFFC1F010317
:10FCC000FCF700003C4004001000000000000000B1
:10FCD0000000000020070000504001000004000068
:10FCE0005C4002000D0F000001010000B440010063
:10FCF00003C0010054C001000E2D09E6204004019C
:10FD0000300000461FC801000020001000800000E5
:10FD100058400401180005004008000009000000D8
:10FD200091000A0080400C018C002C0200000000B1
:10FD3000120012005B808C1B000000000002050E08
:10FD40001C2F4353626968615543320416E4B8C6F8
:10FD50008A674533224A9204EC40070180B0B18C97
:10FD600000000000640483078813C83A9C200A003E
:10FD700001612080B756351210410201A01B0429F1
:10FD800008884000284101010000000030410901BD
:10FD90006406660C0C0100004CD4E83B04196F307B
:10FDA000080E141A20262C32383E10325476980A47
:10FDB0001D5F00006841030164048307881382000B
:10FDC0000000000030420201000000000008000EA8
:10FDD000A080020170380300D0000000A88001114B
:10FDE000F0010000A8800131055AFD01AC8001112D
:10FDF000F0010000AC800131053EFD00FFFFFFFF78
:10FE0000FC1F010348F800003C4004001000000003
:10FE1000000000000000000020170000504001001A
:10FE2000010400005C4002000D0F00000101000011
:10FE3000B440010003C0010054C001000E2D09E6CA
:10FE400020400401300000461FC8010000200010BF
:10FE50000080000058400401180005004008000020
:10FE60000900000091000A0080400C018C002C0267
:10FE700000000000120012005B808C1B00000000DC
:10FE80000002050E1C2F435362696861554332041A
:10FE900016E4B8C68A674533224A9204EC4007014B
:10FEA00080B0B18C00000000640483078813C83A56
:10FEB0009C200A0001612080B756351210410201D2
:10FEC000A01B04290888400028410101000000000F
:10FED000304109016406660C0C0100004CD4E83B7B
:10FEE00004196F300A10161C22282E343A401032A2
:10FEF0005476980A1D5F80A4684103016404830757
:10FF0000881382000000000030420201000000005F
:10FF10000008000EA080020170380300D00000002D
:10FF2000A8800111F0010000A8800131055AFD01EF
:10FF3000AC800111F0010000AC800131053EFD00F4
:10FF4000FFFFFFFF34FA0000809C2B8F80841E008F
:10FF5000000000002700FF7FB80F00200000000015
:10FF60000000000078FB0000809C2B8F80841E0026
:10FF7000000000002200FF7FB80F002000000000FA
:10FF80000000000078FB0000809C2B8F80841E0006
:10FF9000000023002300B600B80F0020000000007E
:10FFA0000000000078FB0000809C2B8F80841E00E6
:10FFB0000000240024009D00B80F00200000000075
:10FFC0000000000078FB0000809C2B8F80841E00C6
:10FFD0000000250025007D00B80F00200000000073
:10FFE0000000000078FB0000809C2B8F80841E00A6
:10FFF0000000260026005300B80F0020000000007B
:020000040001F9
:100000000000000078FB0000809C2B8F80841E0085
:10001000000027002700FF7FB80F0020000000002D
:1000200000000000BCFC0000809C2B8F80841E0020
:10003000000000002700FF7FB80F00200000000034
:100040000000000000FE0000809C2B8F80841E00BA
:10005000000000002700FF7FB80F00200000000014
:100060000000000094F800000000000044FF0000C1
:10007000010000000000000094F8000000000000F3
:1000800064FF0000060000000000000094F800007B
:10009000000000002400010001000000000000003A
:1000A00094F800000000000044000100010000007E
:1000B00000000000193F01060410010000010106C4
:1000C00000102700000900000000000000000000F0
:1000D000E1190000E1190000000000000D0000001F
:1000E0006666660000000000B4000100D000010058
:1000F000000C0000001A9A00005A620280841E0060
:10010000042000001149500200000000000000001F
:10011000000000000000000000000000B0841E008D
:1001200000000000000000000D0000006666660090
:1001300000000000B4000100D00001000000000039
:10014000001A9A00005A620280841E0004200200F5
:1001500011495002000000000000000000000000F3
:100160000000000000000000B0841E00000000003D
:10017000000000000C400200018014007F400000DD
:100180002040020000000000000000003040040099
:10019000000000000000000000000000000000005F
:1001A00050400100000000005C4002000000000020
:1001B00000000000A840010007000000B440040057
:1001C00000400000FF4C000000410000FF4D000017
:1001D00008C001000000000020C00500004300002E
:1001E000EC80B3034375A802000000002E0200005B
:1001F00054C003000E2D09E654060708D1B60200CC
:1002000064C008000430000040201006C8F24818FE
:100210001FE8F600BD4B721511A318051032547675
:10022000980A000088C001000000000008000101D9
:100230000407000018000101000000002000010177
:10024000088400001C4002011000000020F9130483
:100250005C4005014108000001000000B0070800F3
:10026000A7000000000000009440070101011030C9
:1002700050707F7F000000000000000000000000C0
:100280000000000000000000E04002013300000018
:10029000000000000041020100612000B756351245
:1002A0000C410301F95412002030042988BB40009E
:1002B000304103016406660C0C010000E853FA00AB
:1002C0006841030164048307881382000000000072
:1002D00030420301000000000000000E000000009A
:1002E00044420101000000001080010103000000F1
:1002F00038800201114910000100000088800101CE
:10030000000000009C800301EB40020070780300B5
:10031000D5C00000A8800111F0010000A8800131C3
:100320000542CB01AC800111F0010000AC8001312D
:1003300005228D00B0800201000300023700000199
:1003400088000202000C00044C000000940001022E
:1003500000040000D00002020E0000009002960887
:10036000E40001023D094204F40001020000000023
:100370001801010260005102FFFFFFFFFC1F010393
:10038000DC0001004040030000000000000000000D
:10039000A00700001CC0011000F807001CC00130BD
:1003A000F502080050C001008741300C24400601CE
:1003B00007C0520000000000000000000000000321
:1003C0000000000000000000584001016402FF002E
:1003D000804005014B01A0089BC34A74F003000054
:1003E0000000000000000000EC4005017DA8D98B52
:1003F00000000000640483078813C83A9C200A00A8
:100400002441020100000000031000003C410B01E8
:1004100000000000000000000000000000000000DC
:1004200000000000000000000100000000000000CB
:100430000000000000000000000000003C4201013C
:1004400000000000FFFFFFFFFC1F01032801010067
:10045000404003000000000000000000A007000072
:100460001CC0011000F807001CC001301402080075
:1004700050C001008741300424400601070062009B
:100480003870000000000000000000030068010F49
:1004900040B8244058400101FC006900804005013B
:1004A0002363E0119BC34A74F00300000380000043
:1004B000BE0A0000EC4005017DA8D98B590B000055
:1004C000640483078813C83A90200A00244102017B
:1004D00000000000001E00003C410B0100148C00D5
:1004E000141A21282E343B42495043557698BA0CB1
:1004F00028690000010000000721286414171A0071
:100500002004C869A1203A093C42010129000000E9
:10051000FFFFFFFF7C0301004063598F404B4C00FD
:100520000B000B001A00FF7FC00F0020000000002E
:1005300000000000480401004063598F404B4C000C
:100540000B000B001A00FF7FC00F0020000000000E
:10055000000000007401010000000000140501000B
:100560000100000000000000740101000000000014
:1005700034050100010000000000000010B5040077
:100580002100C9B2002000F052F810BD00000101A6
:1005900038B5040000F05DF8050009480460280043
:1005A00000F05BF8002032BD70B5002400F051F877
:1005B000060003480568300000F04FF8280070BDC1
:1005C0003429002070B504000D001600002C02D163
:1005D000FFF7EAFF0400002C08D06068002805D06F
:1005E0003200290020686368984700E0232070BD2E
:1005F0002DE9FC4104000E0017001D00E846002C08
:1006000002D1FFF7D1FF0400002D00D0A846002C36
:100610000AD0A068002807D043463A00310020687D
:10062000D4F808C0E04700E02320BDE8F68113B508
:100630000400012201A92000FFF7C4FF16BD38B550
:1006400004000D000023012229002000FFF7D0FF45
:1006500032BDEFF3108072B67047002800D162B649
:10066000704772009A4200D2885470477047F8B5BC
:1006700004000D0016001F002000C0B2002803D0A7
:100680002000C0B2FFF77AFFF1BD03001A78002AFC
:1006900005D00A00511E002A01D05B1CF6E7181A8B
:1006A00070470100C9B2302904DBC0B23A2801DA30
:1006B000012000E00020C0B2704738B504000025DA
:1006C00020680078FFF7EDFF002808D02068411C63
:1006D00021600A210078303801FB0505F0E7280089
:1006E00032BD2DE9F84F05000E00170098460B9C0F
:1006F000DDF83090DDF834A000971AF0030F0BD12D
:10070000A346CB4508D243463A0031002020A847F3
:100710007F1C1BF1010BF4E7002C08D0641E43463C
:100720003A0031000A98005DA8477F1CF4E75FEAB1
:100730008A700AD50098381A484506D243463A00CE
:1007400031002020A8477F1CF4E73800BDE8F28F75
:100750002DE9F74F84B01F00DDF84080119C129EF8
:10076000DDF84C90DDF850A0159DDDF858B05FEA3B
:100770008B7021D4002D0AD05FEACB7007D53000F2
:10078000C0B2002802D11BF00C0F00D06D1E5445E2
:1007900006D2202C04D2302008F80400641CF6E7AE
:1007A0005FEACB7008D5AC4206D2202C04D23020B0
:1007B00008F80400641CF3E75FEACB6038D55FEA11
:1007C0004B500CD4002C0AD0544501D0AC4206D179
:1007D000641E002C03D0B9F1100F00D1641EB9F1D2
:1007E000100F09D15FEA8B6006D4202C04D2782048
:1007F00008F80400641C15E0B9F1100F09D15FEA94
:100800008B6006D5202C04D2582008F80400641C04
:1008100008E0B9F1020F05D1202C03D2622008F8BC
:100820000400641C202C03D2302008F80400641C4F
:10083000202C17D23000C0B2002804D02D2008F898
:100840000400641C0EE05FEA4B7004D52B2008F80E
:100850000400641C06E05FEA0B7003D5202008F852
:100860000400641CCDF80CB002950194CDF8008012
:100870003B00069A05990498FFF733FF07B0BDE8DF
:10088000F08F2DE9F74F90B01E001C9C1D9D1E9F00
:10089000DDF87C80DDF88090DDF884B05FF0000A40
:1008A000002C01D13BF0100B5FEA4B5001D5002C1E
:1008B0001ED0B4FBF7F007FB1040514611F1010ABE
:1008C0000200D2B20A2A02DA10F1300207E05FEA2F
:1008D0008B6201D5412200E0612282180A3A07ABFF
:1008E0005A54B4FBF7F4002C02D0BAF1200FE0D335
:1008F000CDF818B0CDF81490CDF8108003972800EB
:10090000C0B20290CDF804A007A800903300129A5C
:1009100011991098FFF71CFF13B0BDE8F08F2DE977
:10092000FF4F8FB0DDE91C45DDE92089DDF88CB093
:10093000249F0026002000218D4203D1844201D152
:1009400037F01007780505D5002000218D4201D130
:10095000844229D02000290042464B4600F084FF03
:1009600092463000461C5146C9B20A2902DA1AF1F1
:10097000300107E0B90601D5412100E061211AEB01
:1009800001010A3907AA11542000290042464B46AA
:1009900000F06AFF04000D00002000218D4201D10B
:1009A000844201D0202ED5D30697CDF814B02298DA
:1009B0000490CDF80C809DF878000290019607A86D
:1009C0000090129B119A10990F98FFF7C1FE13B077
:1009D000BDE8F08F000000002DE9F74F2DED088BEA
:1009E0008EB09B46B0EE408AF0EE608A229EDDF823
:1009F0008C80DDF8909000279FEDBE9B53EC182B68
:100A000051EC180B01F048F80ED0CDF80C90CDF851
:100A1000088003200190B5A000905B46189A1799B2
:100A20001698FFF75EFE5CE151EC180B5FF0FF32A9
:100A30007FF4801301F040F80FD2CDF80C90CDF880
:100A4000088004200190DFF8380600905B46189A71
:100A500017991698FFF745FE43E151EC180B002259
:100A6000DFF8203601F040F819D85FEA497001D567
:100A7000042000E003205FEA497102D5DFF8081680
:100A800000E09BA1CDF80C90CDF80880019000917A
:100A90005B46189A17991698FFF723FE21E151EC4F
:100AA000180B0122DFF8E43501F01EF807D951ECEC
:100AB000180B0022DFF8D83500F0FEFF0FD2CDF87A
:100AC0000890CDF804800096B0EE480AF0EE680A6F
:100AD0005B46189A1799169800F010F901E100206A
:100AE0008DF8100051EC180B0022002300F0E4FFF9
:100AF00008D201208DF8100051EC180B91F0004144
:100B000041EC180B5FEA495001D406200600202F63
:100B100007D20A2E05D3302005A9C8557F1C761EA2
:100B2000F5E751EC180B00F0F7FF0500DFF864A5BE
:100B3000280001F00FF802000B0051EC180B01F037
:100B400037F80AEBC602D2E9002301F0DFF841ECE6
:100B50001B0B51EC1B0B01F0ABF90400200001F062
:100B6000BBF902000B0051EC1B0B01F021F841EC2A
:100B70001A0B51EC1A0B0122DFF8443C00F0B4FFD1
:100B80000ED8641C200001F0A7F90AEBC602D2E9D6
:100B9000002300F0A9FF10D8002004006D1C0CE019
:100BA00051EC1A0B0022DFF8183C00F085FF04D34B
:100BB000002C01D0E00700D5641C002E1ED12800B7
:100BC00000F0C8FF02000B0051EC180B00F0F0FF22
:100BD00041EC1A0B51EC1A0B0022DFF8E43B00F059
:100BE0006BFF07D251EC1A0B0122DFF8D43B00F067
:100BF0007BFF26D8E80724D56D1C22E03100202F8A
:100C00000ED2491E0A20B4FBF0F200FB1240303035
:100C100005AAD0557F1C0A20B4FBF0F4002CEED1BD
:100C2000202F08D20800411E002804D0302005AA39
:100C3000D0557F1CF4E7202F03D22E2005AAD055D3
:100C40007F1C202F0DD20A2095FBF0F100FB1150E4
:100C5000303005A9C8557F1C0A2095FBF0F5002D02
:100C6000EFD119F00300012814D1B8F1000F08D01A
:100C70009DF81000002802D119F00C0F01D0B8F136
:100C80000108474506D2202F04D2302005A9C855B7
:100C90007F1CF6E7202F17D29DF81000002804D003
:100CA0002D2005A9C8557F1C0EE05FEA497004D5C8
:100CB0002B2005A9C8557F1C06E05FEA097003D503
:100CC000202005A9C8557F1CCDF80C90CDF80880D0
:100CD000019705A800905B46189A17991698FFF798
:100CE00000FD0EB0BDEC088BBDE8FE8F6E616E009E
:100CF000666E690000000000000000002DE9FE4F54
:100D00002DED068B8AB08046B0EE408AF0EE608A08
:100D10001C9D1E9F53EC182B51EC180B00F0BCFED1
:100D20000FD151EC180B0022D64B00F0DDFE08D994
:100D300051EC180B5FF0FF327FF4801300F0BCFE23
:100D40000ED202971D9801900095B0EE480AF0EE81
:100D5000680A129B119A10994046FFF73DFE8AE1FE
:100D600051EC180B0022002300F0A6FE02D25FF027
:100D7000010A01E05FF0000A5046C0B2002805D029
:100D800051EC180B91F0004141EC180B780501D49F
:100D9000062005008DED068BDDE90601080D00211A
:100DA00004006405640DA4F2FF34DDE906235FF05E
:100DB000FF30DFF8101A02400B400020DFF8081A5D
:100DC00010431943CDE90601200000F0C3FEDFF80F
:100DD000FC29DFF8FC3900F099FFDFF8F829DFF88B
:100DE000F83901F087F8CDE90001DDE9062300209C
:100DF000DFF8E81901F07EF8DFF8E429DFF8E439DC
:100E000000F084FFDDE9002301F074F800F084FEB7
:100E10000600300000F09EFEDFF8CC29DFF8CC3968
:100E200000F074FF0022DFF8983901F063F800F059
:100E300073FE0890300000F08DFEDFF8B429DFF873
:100E4000B43900F063FFCDE90001089800F082FE9C
:100E5000DFF8A429DFF8A43900F058FF02000B00E6
:100E6000DDE9000100F0A4FE41EC190B53EC192B55
:100E700051EC190B00F04AFF41EC1A0B089800F2F4
:100E8000FF30C11701050020CDE9060153EC192BF5
:100E900000205FF0804100F039FFCDE90201002021
:100EA0005FF0804153EC192B00F082FECDE9000188
:100EB00051EC1A0B0022DFF8483901F0D9F8002272
:100EC000DFF8403901F016F802000B0051EC1A0B64
:100ED00001F0CEF80022DFF8303901F00BF8020003
:100EE0000B0051EC1A0B01F0C3F8DDE9002301F00F
:100EF00001F802000B00DDE9020101F0B9F800225F
:100F0000DFF8C43800F0F6FFDDE9062300F0FEFE4E
:100F1000CDE9060151EC180BDDE9062300F0CCFD0C
:100F200009D2761EDDE906010022DFF8D83801F08B
:100F30009FF8CDE90601642E04DA16F1630F01DB98
:100F4000042400E00524380523D551EC180BDFF804
:100F5000BC28DFF8BC3800F0C7FD15D851EC180BE1
:100F60000022DFF8B03800F0A7FD0DD2AE4202DA61
:100F7000AD1B6D1E01E00020050057F480670020C6
:100F800004000020060004E0002D02D0780500D502
:100F90006D1E1D981D998C4202D2001B814601E0F6
:100FA0005FF00009B80703D5002C01D0002081466E
:100FB000002E07D051EC180BDDE9062301F058F89C
:100FC00041EC180B119809905046C0B2002806D089
:100FD00051EC180B91F0004141EC100B03E0B0EE26
:100FE000480AF0EE680A37F400600290CDF80490E9
:100FF0000095129B119A10994046FFF7EDFC83462D
:10100000002C37D05A46501C1190B80601D5452007
:1010100000E06520129B1099C0B2C047002E01D598
:10102000012000E00020002E01D5714200E03100D7
:1010300005220592621E0492002203920A22029265
:10104000C0B201900091129B119A10994046FFF78F
:1010500018FC8346B8070DD50998BBEB00001D9915
:10106000884207D2129B5A4610992020C0471BF194
:10107000010BF1E758460AB0BDEC068BBDE8FE8FC8
:10108000980100000000F07FA001000065CDCD4177
:1010900065CDCDC1480100002DE9FB4F90B00400A3
:1010A00092461C9F00251198002802D1DFF868079E
:1010B000040012980078002800F039831298007814
:1010C00025280AD053462A00119912980078A04783
:1010D0006D1C1298401C1290EBE71298401C129065
:1010E000002006001298007820281FD0232825D041
:1010F0002B2813D02D2809D0302827D156F00106EF
:101100001298401C129001200A9021E056F002062D
:101110001298401C129001200A9019E056F0040623
:101120001298401C129001200A9011E056F0080617
:101130001298401C129001200A9009E056F0100607
:101140001298401C129001200A9001E000200A90A1
:101150000A980028C6D10020099012980078FFF75D
:10116000A0FA002804D012A8FFF7A7FA099010E00F
:10117000129800782A280CD138683F1D002804D521
:1011800056F002064142099100E009901299491C6B
:10119000129100208046129800782E281ED156F415
:1011A00080661298401C129012980078FFF779FA26
:1011B000002804D012A8FFF780FA80460EE01298AB
:1011C00000782A280AD138683F1D012801DB8046B3
:1011D00001E05FF000081299491C12911298007802
:1011E000682817D06A282AD06C2804D0742820D008
:1011F0007A282AD02FE056F480761298401C12905C
:10120000129800786C2804D156F400761298401C8D
:10121000129020E056F080061298401C129012980E
:101220000078682804D156F040061298401C1290AD
:1012300011E056F480761298401C12900BE056F4A0
:1012400000761298401C129005E056F480761298B1
:10125000401C1290FFE712980078252800F0528277
:10126000452800F07581462800F05681472800F097
:101270006F8158281ED062281CD0632800F092810C
:10128000642817D0652800F06381662800F0448147
:10129000672800F05D8169280CD06F280AD070287B
:1012A00000F0F681732800F0A981752802D0782813
:1012B00040F0328212980078782803D01298007893
:1012C000582802D15FF0100911E0129800786F28B9
:1012D00002D15FF008090AE012980078622802D172
:1012E0005FF0020903E05FF00A0936F01006129879
:1012F0000078582801D156F0200612980078692805
:1013000005D012980078642801D036F00C067005DC
:1013100001D57608760012980078692804D01298D2
:101320000078642840F09C80B00543D5FF1D37F05D
:101330000707D7E900010837CDE90C01DDE90C23E7
:10134000002000218B4205DC01DB824202D25FF0EB
:10135000010C01E05FF0000CDDE90C23012000210D
:101360008B4207DB01DC824204D3DDE90C01CDE9CD
:101370000E0106E0DDE90C01404271EB4101CDE9CF
:101380000E01089609980790CDF81880484600216C
:10139000CDE904015FFA8CFCCDF808C0DDE90E014F
:1013A000CDE9000153462A0011992000FFF7B7FA52
:1013B0000500ADE0F00521D5D7F800B03F1DBBF129
:1013C000000F01D5012000E00020BBF1010F01DB7F
:1013D000594601E0DBF100010596099A0492CDF827
:1013E0000C80CDF80890C0B20190009153462A00BD
:1013F00011992000FFF745FA050089E0700605D530
:10140000D7F800B03F1D5FFA8BFB0AE0300605D528
:10141000D7F800B03F1D0FFA8BFB02E0D7F800B001
:101420003F1DBBF1000F01D5012000E00020BBF102
:10143000010F01DB594601E0DBF100010596099A35
:101440000492CDF80C80CDF80890C0B201900091C4
:1014500053462A0011992000FFF713FA050057E0C0
:10146000B0051AD5FF1D37F00707D7E90023083765
:10147000089609980790CDF8188048460021CDE9D4
:10148000040100200290CDE9002353462A0011995F
:101490002000FFF744FA05003AE0F00513D538685C
:1014A0003F1D059609990491CDF80C80CDF8089060
:1014B00000210191009053462A0011992000FFF766
:1014C000E0F9050024E0700605D5D7F800B03F1D0F
:1014D0005FFA8BFB0AE0300605D5D7F800B03F1D58
:1014E0001FFA8BFB02E0D7F800B03F1D0596099864
:1014F0000490CDF80C80CDF8089000200190CDF834
:1015000000B053462A0011992000FFF7BAF90500F0
:101510001298401C1290CCE512980078462801D110
:1015200056F02006FF1D37F0070797ED000B083730
:10153000029609980190CDF8008053462A0011992F
:101540002000FFF749FA05001298401C1290B0E500
:1015500012980078672803D012980078472801D1A4
:1015600056F4006612980078452803D01298007847
:10157000472801D156F02006FF1D37F0070797EDE9
:10158000000B0837029609980190CDF80080534669
:101590002A0011992000FFF7B1FB05001298401CAA
:1015A000129086E55FF00109B0070CD4484610F1AF
:1015B00001090999884206D253462A001199202030
:1015C000A0476D1CF2E738683F1D53462A00119969
:1015D000C0B2A0476D1CB0070CD5484610F10109F8
:1015E0000999884206D253462A0011992020A04723
:1015F0006D1CF2E71298401C12905AE5D7F8009043
:101600003F1DB8F1000F01D0414601E05FF0FF310E
:101610004846FFF73AF88346700502D5C34500D324
:10162000C346B0070CD4584610F1010B0999884203
:1016300006D253462A0011992020A0476D1CF2E7DC
:1016400099F80000002810D0700504D54046B0F18C
:101650000108002809D02A00551C5346119999F811
:101660000000A04719F10109EAE7B0070CD5584678
:1016700010F1010B0999884206D253462A001199AC
:101680002020A0476D1CF2E71298401C129010E534
:101690000820099056F021065FF000094846C0B2C4
:1016A000002818D03A683F1D089609980790CDF891
:1016B000188010200021CDE90401002002901000C4
:1016C0000021CDE9000153462A0011992000FFF7BF
:1016D00026F9050012E038683F1D05960999049126
:1016E000CDF80C8010210291002101910090534609
:1016F0002A0011992000FFF7C4F805001298401C39
:101700001290D6E453462A0011992520A0476D1C5B
:101710001298401C1290CCE453462A00119912985A
:101720000078A0476D1C1298401C1290C1E45545EA
:1017300001D22A0001E0BAF10102534611990020BA
:10174000A047280013B0BDE8F08F0EB43CB50400EC
:1017500005AD009523005FF0FF3201A92F48FFF788
:101760009BFC36BC5DF810FB0CB47CB504000D008E
:1017700006AE00962B005FF0FF3221002848FFF7ED
:101780008BFC76BC5DF80CFB08B4FCB504000D00C6
:10179000160007AF009733002A0021002048FFF70A
:1017A0007BFCF6BC5DF808FB3EB504000D0000951F
:1017B00023005FF0FF3201A91848FFF76DFC3EBD22
:1017C0000000E03FFFFF0F000000F03FFB799F505B
:1017D0001344D33FB3C8608B288AC63F0000F8BFCC
:1017E00061436F63A787D23F71A379094F930A4082
:1017F0001655B5BBB16B0240EF39FAFE422EE63FFB
:1018000000002C4000002440000018402D431CEB39
:10181000E2361A3F80842E416D0601006F060100FA
:101820006506010013F0004C03D55B42524263F1A0
:1018300000039CEA210C00F0178010B5644603D326
:101840004942404261F1000100F00EF8640004D307
:101850004942404261F10001244203D55B425242B9
:1018600063F1000310BD0000BBBBE1B1B2F5803FE6
:1018700080F07E80022A1ED98C46B1FBF2F102FB79
:1018800011C31B0443EA1043B3FBF2FC02FB1C33FD
:1018900080B240EA0343B3FBF2F002FB103240EAAD
:1018A0000C4000237047022A05D98446B0FBF2F0B1
:1018B00002FB10C270474AB105D100F0010249088D
:1018C0005FEA3000704700220023704700F0F4BC4C
:1018D0000B000200002100207047904271EB030CC6
:1018E000F6D3B3F5803F2FD2F0B5B3FA83F7B1FA50
:1018F00081F4A7F10F0E3D1B5340CEF1200602FAF2
:101900000EF2F3415340B5F10F0746D80F3C2C447B
:101910004140C4F12006A040F1414140B1FBF3F643
:1019200003FB1611A2FB0645001BA94102D2761E3D
:101930008018594180EA010221FA0EF362FA0EF290
:1019400000215A403046F0BD30B4B1FBF3FC03FB3C
:101950001C11A2FB0C45001BA94103D2ACF1010CE8
:101960008018594130BC02460B4660460021704742
:10197000B2F1807F65D3F0B5B2FA82F7B1FA81F4A3
:10198000C7F10F063D1B22FA06F307F1110EF241D3
:1019900020355A40B5F10F07B8D94140C4F12006AF
:1019A000A040F1414140B1FBF3FC03FB1C11A2FB41
:1019B0000C45001BA94103D2BCF1010C8018594110
:1019C0000F2F12D30F3FC90341EA5041B1FBF3F689
:1019D00003FB1611A2FB0645D4EBC030A94102D28D
:1019E000761E8018594146EACC3C07B34140C7F106
:1019F0002006B840F1414140B1FBF3F603FB16115C
:101A0000A2FB0645001BA94102D2761E801859414F
:101A100080EA010221FA0EF3C7F1200462FA0EF205
:101A20000CFA07F05A402CFA04F13043F0BD80EA7A
:101A3000010221FA0EF3002162FA0EF260465A40CA
:101A4000F0BD8C46B1FBF2F102FB11C31B0243EA6D
:101A50001063B3FBF2FC02FB1C331B024CEA0020B8
:101A600043EA1063B3FBF2FC02FB1C331B024CEA9B
:101A7000002043EA1063B3FBF2FC02FB1C331B02A1
:101A80004CEA002043EA1063B3FBF2FC02FB1C3279
:101A90004CEA00200023704790420CD141EA030C2D
:101AA00050EA4C0C07D0994205D14FF4001C1CEBB6
:101AB000410F38BF894270474FF4001C1CEB410FA7
:101AC00094BF1CEB430F09E041EA030C50EA4C0CB5
:101AD00052EA0C0C03D2994208BF9042704714BFDF
:101AE0008B428242704774004FF4001C1CEB410F84
:101AF00094BF1CEB430F09E041EA030C50EA4C0C85
:101B000052EA0C0C03D28B4208BF8242704714BFCA
:101B10009942904270470202C1F30A5340F2FE32EA
:101B20009B1A14DDD3F120034FEAE17208DDC902EC
:101B300041EA505141F00040D84080185040704771
:101B400003F2E13010B1D24382F000407047002030
:101B500070470202C11768B14840401AB0FA80F2DB
:101B60009040D21CC907C2F5846241EA025202EBDE
:101B7000D0214005704730B4002513E050F8042B05
:101B8000D30744BFA9F101039A18091F042942F899
:101B9000045BFAD213468C0744BF15809B1CC9070F
:101BA00048BF1D7050F8041B0029E7D130BC7047B6
:101BB00070B44FF0004591EA030F40F1A3816B40F0
:101BC000841A71EB030603D2001BB1411219734151
:101BD0004FF4001C1CEB410F34BF7CEB430442E08C
:101BE0000C0DA4EB1356352E4FDC45EAC323DB0A5C
:101BF00045EAC121C912B6F120050DDD63FA05F6EB
:101C0000EB4086EA0305124218BF45F00105C018F3
